:020000040800F2
:1000000000000220293401083197000833970008C6
:10001000359700083797000839970008000000005E
:100020000000000000000000000000003B970008F6
:100030003D970008000000003F9700084197000826
:100040006D3401086D3401086D3401086D34010808
:100050006D3401086D3401086D3401086D340108F8
:100060006D3401086D3401086D340108297A0008E7
:100070006D3401086D3401086D3401086D340108D8
:100080006D3401086D3401086D3401086D340108C8
:100090006D3401086D3401086D3401087199000850
:1000A0006D3401086D3401086D3401086D340108A8
:1000B0003D9900086D3401086D3401086D34010864
:1000C0006D3401086D3401086D3401086D34010888
:1000D0006D3401086D340108859A00086D340108FB
:1000E0006D3401086D340108459700086D3401082E
:1000F0006D3401086D3401086D3401086D34010858
:100100006D3401086D3401086D3401086D34010847
:100110006D3401086D3401086D3401086D34010837
:100120006D3401086D3401086D3401086D34010827
:100130006D3401086D3401086D3401086D34010817
:100140006D3401086D3401086D340108759700089D
:100150006D3401086D3401086D3401086D340108F7
:100160006D3401086D3401086D3401086D340108E7
:100170006D3401086D3401086D3401086D340108D7
:080180006D3401086D34010823
:1001880024B8050800000020300C0020300C0020A6
:10019800D43C002008B5074B186809F063FA0EF044
:1001A800DFF8054B054806221A70BDE8084001F043
:1001B800C8BC00BF40260020CD250020A80F002085
:1001C80008B5034801F0BDFC024B00221A7008BDB7
:1001D800FC170020CD25002008B5054B0122002082
:1001E8001A7005F0E1FE0348BDE8084001F0A9BC1B
:1001F800582C00206C1500202DE9F041144C2046A5
:1002080004F055F800201349134A03F007FE134978
:10021800134A0746002003F001FE1249124A064617
:10022800002003F0FBFDD22105463A4623460A206A
:1002380003F00CFFD22132462346FA2003F006FFD2
:100248005A20D2212A462346BDE8F04103F0FEBEDB
:100258008013002056A40508C90100085FA40508FA
:10026800E101000867A405089D01000808B5054BD1
:10027800012200201A7005F097FE0348BDE80840E7
:1002880001F05FBC582C00206C15002008B503480D
:1002980001F057FC024B00221A7008BDFC17002021
:1002A800CD25002008B5054B07221A700EF058F826
:1002B8000348BDE8084001F044BC00BFCD2500203C
:1002C800801300202DE9F041144C204603F0EFFF85
:1002D80000201349134A03F0A1FD1349134A0746A6
:1002E800002003F09BFD1249124A0646002003F045
:1002F80095FDD22105463A4623460A2003F0A6FE7C
:10030800D221324623465A2003F0A0FEAA20D22149
:100318002A462346BDE8F04103F098BEA80F002006
:1003280056A405089502000870A40508AD02000847
:1003380079A4050875020008014801F002BC00BF55
:100348009411002010B5094C204603F0B0FF00209E
:100358000749084A03F062FDD221024623464FF4BA
:100368008270BDE8104003F071BE00BFB4160020D3
:1003780082A405084103000870B50C4C0C4D206898
:100388004FF6E076314603F08DF82068294603F0F1
:1003980037F86068314603F085F86068294603F04D
:1003A8002FF8BDE8704004F0BBB900BF300C002046
:1003B80078AA050838B52B4CFFF7DEFF002005F0BA
:1003C800F3FD237A23B90A203221274A05F0FAFEE1
:1003D800637A23B90A206421244A05F0F3FE214CEC
:1003E800A37A23B90A209621214A05F0EBFEA37AC5
:1003F8001C4DFBB16B7AEBB12B7ADBB100232B726E
:100408006B72AB721B4B286801221A704FF6E071B1
:1004180003F048F82868184902F0F2FF686817499D
:1004280002F0EEFF0BF033FC04F07AF9144804F004
:10043800BBF90DE00B4C4FF47841206803F032F81B
:100448002068104902F0DCFF60680F4902F0D8FF0D
:10045800FFF792FF00200BF0DDFB0C48BDE83840A9
:1004680001F06FBB300C002089A4050897A405088B
:10047800A6A40508CD250020B4A4050879AA050876
:1004880080969800C8A405087BAA0508FC170020D8
:1004980008B500200BF0BEFB0248BDE8084001F09B
:1004A80050BB00BFFC17002038B5FFF765FF0DF003
:1004B8006FFF3C213F220023DF2005F065FE4FF44B
:1004C80080600EF0A3FC124C3E223C21DF2000236A
:1004D80005F05AFE012323720E4B4FF6E07518689B
:1004E80009F0C0F82068294602F0DCFF20680A49B4
:1004F80002F086FF6068294602F0D4FF6068074969
:1005080002F07EFF04F00CF9054B00221A7038BD8A
:10051800300C002040260020DAA40508EDA40508C8
:10052800CD25002038B5FFF727FF0DF031FF6E21EC
:100538003F220023DF2005F027FE4FF486400EF00F
:1005480065FC124C3E226E21DF20002305F01CFEC4
:10055800012363720E4B4FF6E075186809F082F8B4
:100568002068294602F09EFF20680A4902F048FFE9
:100578006068294602F096FF6068074902F040FF6C
:1005880004F0CEF8054B00221A7038BD300C00205C
:100598004026002000A5050811A50508CD25002046
:1005A80010B5FFF7E9FE0DF0F3FEA0213F2200236E
:1005B800DF2005F0E9FD4FF402400EF027FC114C56
:1005C8003E22A021DF20002305F0DEFD0123A372D7
:1005D8000D4B186809F046F820684FF6E07102F0F4
:1005E80061FF2068094902F00BFF6068084902F0C2
:1005F80007FF04F095F864200BF0D8F9054B0022AA
:100608001A7010BD300C00204026002022A50508D5
:1006180079AA0508CD2500202DE9F74F3A4D3B4E24
:100628000024284603F043FE224623464FF6FF7176
:1006380037480094019402F0F9FE4FF6E078042759
:10064800F06041462246234632480097019402F062
:10065800EDFE23463060414622462F48009701941C
:1006680002F0E4FE2D4970602D4A204603F0D6FBC7
:100678002C492D4A0746204603F0D0FB2B492C4A2B
:100688008046204603F0CAFB2A492B4A8146204669
:1006980003F0C4FB29492A4A8346204603F0BEFBDF
:1006A80021468246F2682B46204603F0CFFC5A21A9
:1006B80032682B460A2003F0C9FC6E2172682B466B
:1006C8000A2003F0C3FC9B213A462B46FA2003F08C
:1006D800BDFC692142462B46FA2003F0B7FC3721BE
:1006E8004A462B46FA2003F0B1FCC82152462B4655
:1006F800AA2003F0ABFCF020C8215A462B4603B0D1
:10070800BDE8F04F03F0A2BC24140020300C0020F8
:1007180036A505083EA5050851A5050860A50508E4
:10072800A905000868A505082D05000858A50508AD
:10073800B104000870A505089904000877A5050804
:10074800BD03000838B50C4C4FF6E0752068294603
:1007580002F0A8FE2068094902F052FE60682946A6
:1007680002F0A0FE6068064902F04AFE03F0D8FFD6
:10077800BDE8384003F0D4BF300C00203EA5050882
:100788007EA5050870B52DED028B9FED248A88B0F3
:100798000A26F0EE488A03E0B0EE608AF0EE418A5D
:1007A8000CF043FD8DED000ACDED010A9DE8030034
:1007B80004AB83E80300F0EE680AB0EE480A9DED4A
:1007C800041ADDED051A8DED028ACDED038A0CF0D1
:1007D800CDFACDED010A8DED000A9DE8030002ADCA
:1007E80085E80300013E6C46DDED020A9DED031A23
:1007F800D2D19FED0B0A0CF00FFD8DED000ACDED67
:10080800010A9DE8030085E80300DDED030A9DED7C
:10081800020A08B0BDEC028B70BD00BF00000000EA
:10082800CDCCCC3D2DE9F74F564D574CDFF86491B0
:10083800DFF864814FF6E07005F08AFB286811F054
:10084800F7FC064668680F4611F0F2FC3246CDE91F
:1008580000013B464946204616F07CFB2246002311
:100868000520372105F0AEFC2869484F484E11F0A5
:10087800DFFC824668698B4611F0DAFC5246CDE906
:1008880000015B463946204616F064FB22460023E9
:100898000520692105F096FC286B11F0C9FC8246F9
:1008A800686B8B4611F0C4FC5246CDE900015B46EB
:1008B8004146204616F04EFB002305209B21224688
:1008C80005F080FC31462A6C204616F043FB224690
:1008D80000239B21A22005F075FC4FF4FC6005F075
:1008E80037FBA86811F0A4FC8246E8688B4611F033
:1008F8009FFC5246CDE900015B464946204616F06A
:1009080029FB224605205021002305F05BFCA8693D
:1009180011F08EFC8246E8698B4611F089FC52463C
:10092800CDE900015B463946204616F013FB224606
:1009380000230520822105F045FCA86B11F078FC06
:100948008246E86B8B4611F073FC5246CDE90001F4
:100958005B464146204616F0FDFA00230520B421E7
:10096800224605F02FFC31466A6C204616F0F2FA52
:10097800A220B4212246002303B0BDE8F04F05F0C1
:1009880021BC00BF603A0020400C0020A3A5050848
:10099800C6A5050891A50508B5A5050808B5002050
:1009A80005F002FB0A4B1B780B2B0BD8DFE803F092
:1009B8000A0A0A0A0A0A08060A0A0A0A054802E08E
:1009C800054800E00548BDE8084001F0BAB800BF96
:1009D800CD25002080130020A80F0020FC17002040
:1009E8002DE9F14F2D4C204603F061FC00202C49E5
:1009F8002C4A03F013FA2C492C4A8146002003F0B4
:100A08000DFA2B492B4A0746002003F007FA2A491A
:100A18002A4A0646002003F001FA2949294A0546D0
:100A2800002003F0FBF92849284A8046002003F0FB
:100A3800F5F92749274A8246002003F0EFF9D22129
:100A480083464A462346E62003F000FB28203A4620
:100A58002346014603F0FAFA462132462346282067
:100A680003F0F4FA64212A462346282003F0EEFA1C
:100A7800822142462346282003F0E8FA52462346BC
:100A88002820A02103F0E2FA28205A46BE21234656
:100A980001B0BDE8F04F03F0D9BA00BF6C150020D3
:100AA800CBA50508A5090008D4A505083514000834
:100AB800DFA5050811140008E9A50508ED130008CD
:100AC800F4A50508C9130008FFA50508A513000823
:100AD80009A6050881130008023810B50A2800F293
:100AE8003484DFE810F00B000F00D0003A01250233
:100AF800BB01D002EA0232049903ED03BDE81040BD
:100B08000BF032B900204FF6E0710BF083FA642045
:100B18004FF6E0710BF07EFAC8204FF6E0710BF04B
:100B280079FA4FF6FF7005F013FA00237D20DC21D7
:100B3800B14A05F047FB4EF29C7005F009FAAF4B3D
:100B48001C78022C32D0052C6CD0012C40F0FD838F
:100B5800B4204FF4F0610BF05DFA05202146A84A55
:100B6800002305F02FFB05205221A64A002305F09B
:100B780029FBB621A44A0023052005F023FB4FF4E6
:100B8800F06005F0E5F940F2131021469C4A002375
:100B980005F018FB40F2131052219B4A002305F080
:100BA80011FB40F21310B621984A2CE0A0204FF414
:100BB800F0610BF02FFA05200121924A002305F07D
:100BC80001FB05205221924A002305F0FBFAB621C9
:100BD8008D4A0023052005F0F5FA4FF4F06005F082
:100BE800B7F940F213100121864A002305F0EAFA0A
:100BF80040F213105221844A002305F0E3FA854A93
:100C080040F21310B621002305F0DCFA4EF29C7076
:100C180005F09EF90520A2217F4A0023BDE8104077
:100C280005F0D0BA64204FF4F0610BF0F3F92046D8
:100C380001217A4A002305F0C5FAB621724A002339
:100C4800204605F0BFFA4FF4F06005F081F940F254
:100C580013100121714A002305F0B4FA40F2131071
:100C68005221694A002305F0ADFAB62140F213106B
:100C78006B4A002305F0A6FA4EF29C7005F068F95D
:100C880020465221C8E700204FF6E0710BF0C2F968
:100C980031204FF6E0710BF0BDF963204FF6E0719B
:100CA8000BF0B8F995204FF6E0710BF0B3F9C720B7
:100CB8004FF6E0710BF0AEF94EF29C7005F048F972
:100CC800052001210023574A05F07CFA0520202140
:100CD8000023554A05F076FA052052210023534A8D
:100CE80005F070FA052084210023514A05F06AFABC
:100CF800B6210520444A002305F064FA4FF4F06059
:100D080005F026F9012140F213100023454A05F0A9
:100D180059FA40F213102021464A002305F052FAEE
:100D280040F213105221384A002305F04BFA40F2E2
:100D380013108421404A002305F044FAB6213F4AA3
:100D480040F21310002305F03DFA4FF6FF7005F04E
:100D5800FFF87D20DC213A4A5FE700204FF6E0717A
:100D68000BF058F927204FF6E0710BF053F94F209C
:100D78004FF6E0710BF04EF977204FF6E0710BF06B
:100D880049F99F204FF6E0710BF044F9C7204FF660
:100D9800E0710BF03FF94EF29C7005F0D9F8052090
:100DA80001210023184A05F00DFA05201621002319
:100DB800244A05F007FA05203E210023224A05F0BF
:100DC80001FA052066210023204A05F0FBF98E214F
:100DD800002305201E4A05F0F5F905201D4AB62115
:100DE800002305F0EFF94FF6FF7005F0B1F87D200C
:100DF800DC21194A11E700BFDFA505081C03002004
:100E08000FA6050818A60508E3AB05080EA60508F1
:100E180013A6050817A605084AA605081DA605086D
:100E28001CA6050836A6050821A6050831A605084A
:100E380026A605082BA6050830A6050835A6050828
:100E4800E9A5050839A605083DA6050841A605082F
:100E580045A6050849A605084DA6050800204FF631
:100E6800E0710BF0D7F831204FF6E0710BF0D2F8B3
:100E780063204FF6E0710BF0CDF895204FF6E07146
:100E88000BF0C8F8C7204FF6E0710BF0C3F84EF22C
:100E98009C7005F05DF8052001210023BF4A05F08C
:100EA80091F9052020210023BD4A05F08BF9052082
:100EB80052210023BB4A05F085F90520842100232F
:100EC800B94A05F07FF9B6210520B84A002305F094
:100ED80079F94FF4F06005F03BF8012140F2131066
:100EE8000023B34A05F06EF940F213102021B14AED
:100EF800002305F067F940F213105221AB4A002392
:100F080005F060F940F213108421AB4A002305F084
:100F180059F9B621A94A40F21310002305F052F9F5
:100F28004FF6FF7005F014F87D20DC21A44A74E622
:100F3800A44B1C78022C32D0052C5DD0012C40F03B
:100F48008B8000204FF6E0710BF064F834204FF6E8
:100F5800E0710BF05FF864204FF6E0710BF05AF87F
:100F68004FF6E07198200BF055F84EF29C7004F0A3
:100F7800EFFF05202146944A002305F023F90520B8
:100F88002021924A002305F01DF905205021904A9E
:100F9800002305F017F9052084218E4A59E0002026
:100FA8004FF6E0710BF036F852204FF6E0710BF077
:100FB80031F890204FF6E0710BF02CF84FF6E07105
:100FC800B4200BF027F84EF29C7004F0C1FF052006
:100FD8000121814A002305F0F5F805203E217C4ACD
:100FE800002305F0EFF805207C217A4A002305F05C
:100FF800E9F80520A0212BE000204FF6E0710BF066
:1010080009F82E204FF6E0710BF004F87F204FF618
:10101800E0710AF0FFFF4FF6E071AD200AF0FAFF29
:101028004EF29C7004F094FF204601216B4A002385
:1010380005F0C8F820463221654A002305F0C2F8B9
:1010480020466B21634A002305F0BCF8204699210D
:10105800634A002305F0B6F84FF4F06004F078FF17
:10106800604A00230520B62105F0ACF84FF4FC6176
:10107800C8200AF0CFFF4FF6FF7004F069FF872001
:10108800DC21594AC9E500204FF6E0710AF0C2FF99
:1010980063204FF4FC610AF0BDFF4FF6E071C720F2
:1010A8000AF0B8FF4FF6FF7004F052FF002005F079
:1010B80051F8A520D7214D4AAFE5042005F04AF89C
:1010C80000204FF6E0710AF0A5FF31204FF6E071DD
:1010D8000AF0A0FF63204FF6E0710AF09BFF95200D
:1010E8004FF6E0710AF096FFC7204FF6E0710AF05C
:1010F80091FF4EF29C7004F02BFF05200121002384
:101108003B4A05F05FF8052020210023314A05F00D
:1011180059F8052052210023364A05F053F80520D6
:1011280084210023344A05F04DF80520B621334ABE
:10113800002305F047F84FF6E07004F009FF40F28D
:101148000B1001212E4A002305F03CF840F22B1029
:1011580020212C4A002305F035F840F223105221B3
:10116800294A002305F02EF840F21B108421274A53
:10117800002305F027F8B621254A002340F2131072
:1011880005F020F84FF6FF7004F0E2FE002004F0AE
:10119800E1FF6E20D2211F4ACFE000BF59A6050803
:1011A8005DA605087AA6050861A60508E3AB05084B
:1011B8006AA6050866A6050865A6050869A60508BD
:1011C8006EA605081C0300201DA6050842A60508F2
:1011D8003AA6050889A605084AA605083EA60508F0
:1011E80079A60508FAAC050809A6050891AA050814
:1011F8007DA6050888A605088BA605088FA60508FC
:1012080094A6050836A605089BA605089FA6050806
:10121800A4A60508AAA60508042004F09BFF002040
:101228004FF6E0710AF0F6FE27204FF6E0710AF05B
:10123800F1FE4F204FF6E0710AF0ECFE77204FF6F2
:10124800E0710AF0E7FE9F204FF6E0710AF0E2FE37
:10125800C7204FF6E0710AF0DDFE4EF29C7004F0F4
:1012680077FE052001210023384A04F0ABFF052052
:1012780016210023364A04F0A5FF05203E2100234D
:10128800344A04F09FFF05206621334A002304F006
:1012980099FF05208E21314A002304F093FFB621DF
:1012A8002F4A0023052004F08DFF4FF6FF7004F04D
:1012B8004FFE002004F04EFF6420D221294A3CE072
:1012C800042004F047FF00204FF6E0710AF0A2FE68
:1012D80043204FF6E0710AF09DFE85204FF6E0713D
:1012E8000AF098FE4FF6E071C7200AF093FE4EF21E
:1012F8009C7004F02DFE052001211B4A002304F0F8
:1013080061FF05204521194A002304F05BFF0520F1
:101318008721134A002304F055FFB621144A0023FD
:10132800052004F04FFF4FF6FF7004F011FE002077
:1013380004F010FF0F4A7D20D221002304F042FF61
:101348000420BDE8104004F005BF10BDB0A6050894
:1013580066A605086BA60508B5A60508B8A605087B
:101368004AA60508BBA60508C4A605081DA60508C3
:10137800E3AB050857AB050810B5064C064806232D
:10138800237000F0DEFB2078FFF7A6FBBDE81040D5
:101398000DF00ABD582C00205817002010B5064C37
:1013A80006480723237000F0CCFB2078FFF794FB56
:1013B800BDE810400DF0F8BC582C0020581700204C
:1013C80010B5064C06480523237000F0BAFB2078B8
:1013D800FFF782FBBDE810400DF0E6BC582C00205A
:1013E8005817002010B5064C06480423237000F057
:1013F800A8FB2078FFF770FBBDE810400DF0D4BCC7
:10140800582C00205817002010B5064C0648032316
:10141800237000F096FB2078FFF75EFBBDE81040D4
:101428000DF0C2BC582C00205817002010B5064CEF
:1014380006480223237000F084FB2078FFF74CFB5A
:10144800BDE810400DF0B0BC582C00205817002003
:1014580038B5094C05464FF6E071206802F022F8CD
:1014680020680DB1054900E0054901F0C9FFBDE854
:10147800384003F055B900BF5C0C0020C8A6050829
:10148800DBA60508194B10B51C78012C05D006D32E
:10149800022C0CBF3024002402E0002400E01024B9
:1014A80004F1C80006F012FB11490246114815F074
:1014B80051FD04F1CC0006F009FB0D4902460E4827
:1014C80015F048FD04F1D00006F000FB084902467B
:1014D8000A4815F03FFD04F1D40006F0F7FA044974
:1014E80002460748BDE8104015F034BD1C0E002028
:1014F800C6A5050810260020342600204A2C002006
:10150800FC25002010B5E82006F0E0FA0F4C024652
:1015180021460F4815F01EFDEC2006F0D7FA2146AB
:1015280002460C4815F016FDF02006F0CFFA2146C9
:101538000246094815F00EFDF42006F0C7FA0246E7
:1015480006482146BDE8104015F004BDC6A50508AB
:1015580010260020342600204A2C0020FC250020DC
:101568000E4A012310B513700D4A002414700D4A59
:10157800204613700AF04EFB204604F015FD0A4B76
:1015880003221A700AF0A4FE0BF0E9FB074B084887
:101598001C70BDE8104000F0D4BA00BF582C0020E1
:1015A800770D0020750D0020CD250020343800204F
:1015B8003812002038B50D4B0D4D00241C700D4B12
:1015C80028681C700C4B4FF6E0711C7001F06AFF24
:1015D80028680A4901F014FF03F0A2F8204604F035
:1015E800E3FC0748BDE8384000F0ABBAD40D002052
:1015F8005C0C0020770D0020CD2500207DAA050871
:10160800FC17002007B50E4B0E481A78D2F10102DC
:1016180038BF00221A700C4B05221A7000F091FA9C
:10162800022201238DE80C00B02060211022322311
:101638000DF05EFD03B05DF804EB03F071B800BF78
:10164800D40D0020F0100020CD2500202E4A0023C4
:1016580010B513702D4A13700DF09EF9044600283A
:1016680042D02B4C4FF6E071206801F01BFF206838
:10167800284901F0C5FE60684FF6E07101F012FFDD
:101688006068254901F0BCFEA0684FF6E07101F0E2
:1016980009FFA068214901F0B3FE03F041F84FF4B7
:1016A8007A600AF083F920684FF6E07101F0FAFEDB
:1016B80020681B4901F0A4FE60684FF6E07101F054
:1016C800F1FE6068164901F09BFEA0684FF6E071D4
:1016D80001F0E8FEA068124901F092FE03F020F83C
:1016E800BDE8104003F01CB80CF03AFE204604F0A8
:1016F8005BFC0C4B0C4804221A7000F022FABDE87F
:101708001040FFF71FB800BFD40D0020770D002050
:101718005C0C0020EEA6050802A7050812A705081C
:101728007CAA0508CD250020241400202DE9F04FBF
:101738006A4DDFF8F4916A4E85B000244FF6FF78C1
:10174800284602F0B4FD41462246234665480094E7
:10175800019401F06BFE042703904146224623467C
:1017680048460097019401F061FE414630602246E8
:10177800234648460097019401F058FE41467060A0
:101788002246234648460097019401F04FFEA8F5EB
:101798000048B060414622462346534800970194CA
:1017A80001F044FE4146F060224623464F48009728
:1017B800019401F03BFE41463061224623464C48E5
:1017C8000097019401F032FE23467061414622469B
:1017D80048480097019401F029FE4749B061474AFB
:1017E800204602F01BFB4649464A8046204602F046
:1017F80015FB4549454A8246204602F00FFB4449FD
:10180800444A0746204602F009FB4349434A8146B9
:10181800204602F003FB4249424A8346204602F032
:10182800FDFA21468446039ACDF808C02B46204687
:1018380002F00CFC052132682B46A02002F006FCC1
:10184800692172682B46782002F000FC7D21B2687D
:101858002B46782002F0FAFB2821F2682B46052057
:1018680002F0F4FB4B2132692B46052002F0EEFB17
:10187800052072696E212B4602F0E8FB9121B269BE
:101888002B46052002F0E2FBD2213A462B460520E2
:1018980002F0DCFBD22142462B46602002F0D6FB48
:1018A800D2214A462B46B02002F0D0FBD221524624
:1018B8002B464FF4807002F0C9FBB4215A462B46E0
:1018C800052002F0C3FBDDF808C06020B4216246A1
:1018D8002B4605B0BDE8F04F02F0B8BBC814002095
:1018E8005C0C002022A705082CA7050833A70508CB
:1018F80039A705083FA7050845A705085516000894
:101908004DA70508BD15000855A705080D160008C0
:101918005EA705086915000866A705080D150008E3
:101928006FA705088D14000879AA0508664A0023E0
:101938002DE9F04713700125644ADFF8A881137078
:10194800A842014688F8005003D0022840F0AB8036
:1019580036E04FF4747006F0A0F80AF0DFFB5C4B39
:101968005C4C186810F052FC53A3D3E900230646D8
:101978000F4610F037FF10B1022323700BE03046FA
:1019880039464FA3D3E9002310F018FFD0F1010026
:1019980038BF00202070012005F054FA0120FFF71D
:1019A80057FD4C4B1978012906D002D302297AD168
:1019B80002E04020002100E0402007F061FA72E0D8
:1019C800C82006F083F80446CC2006F07FF80746C6
:1019D800D02006F07BF80646D42006F077F881463A
:1019E8000AF09CFB3A4B3C491A68A242184602DBB3
:1019F8000B68BB4213DD394B04601E60384B0F6027
:101A0800C3F800900AF0C6F8364B01221A70364A1D
:101A18000520B4210023BDE8F04704F0D3BB94426D
:101A280018D19F4216D12D4B1B689E4212D12C4BC8
:101A38001B6899450ED14FF47470294688F80050F8
:101A480006F02BF8294B00221A60294B4FF07E52E2
:101A58001A6028E0234B02251D7029464FF4747044
:101A680006F01BF81A4B1B6806EE906A1C1BF8EE72
:101A7800E67A06EE904AB8EEE67A1C4B87EE277AAD
:101A8800284683ED007A154B1B6806EE903AB8EEAF
:101A9800E67A174BC7EE277AC3ED007A05F0D2F93C
:101AA8000020FFF7D5FC0AF0D4FABDE8F04702F0B1
:101AB80037BE00BFAFF3008000000000A3E1A141E2
:101AC8000000000080842E41D40D0020770D0020F6
:101AD8004C2600201C0E0020642C0020402C0020E6
:101AE800F8250020C901002078A70508C82500208E
:101AF80008260020AFF3008008B500F053FFFEF77A
:101B08007BFB00F04FF800F06FF8FEF785FDFEF75D
:101B1800D9FBFEF765FF01F055FBFFF707FE01F063
:101B280027F9FEF70FFC01F049FA00F073FB00F00B
:101B380087FD00F091FE00F065FABDE8084000F06E
:101B480033BB10B5044628B90F48104A104B53212F
:101B580003F00EF80F4B1868844213D010B1C36914
:101B680000219847002004F01FFA002004F006FA2C
:101B78004FF6FF7004F0ECF9E3692046012198471D
:101B8800044B1C6010BD00BF8CA705084425040841
:101B9800A8A70508780C00200048D2E7FC17002009
:101BA8000CF0BABE10B5084C204602F080FB0020AD
:101BB8000649074A02F032F9D22102462346FA20A2
:101BC800BDE8104002F042BA600E0020C6A7050822
:101BD800A91B0008024B034801221A70FFF7B1BF86
:101BE800CD250020C81400202DE9F743374D384F84
:101BF800384E0024284602F05AFB2246234647F670
:101C0800FF7135480094019401F010FC4FF6FF78FD
:101C1800814641462246234638460094019401F005
:101C280005FC41463060224623463846009401941C
:101C380001F0FCFB4146706022462346384600947A
:101C4800019401F0F3FB2346B06041462246384632
:101C58000094019401F0EAFB2049F060204A2046F4
:101C680002F0DCF81F49204A0746204602F0D6F861
:101C7800214680464A462B46204602F0E7F93C2199
:101C880032682B46192002F0E1F95A2172682B4676
:101C9800192002F0DBF97821B2682B46192002F0EE
:101CA800D5F99621F2682B46192002F0CFF9D221F6
:101CB8003A462B46EC2002F0C9F99C20D221424634
:101CC8002B4603B0BDE8F04302F0C0B9381200203B
:101CD80079AA05087C0C0020B8A70508C5A705083F
:101CE800DD1B0008CEA70508B91E000870B5474ED1
:101CF800474C327847492DED028B142592B005FBED
:101D080002420C320FA815F025F933780E2B05FB8B
:101D180003F504EB050332D8D3ED016A9B6807EE9F
:101D2800103A6359B8EEE68A06EE903ADFED3A7A51
:101D3800F8EEC78AB8EEE67A88EE278AC8EEA78A50
:101D4800C7EE277A17EE900A10F072FA02460B4691
:101D58006846324915F0FEF818EE100A10F068FAD5
:101D680002460B4605A82E4915F0F4F818EE900A1D
:101D780010F05EFA02460B460AA82A4929E093EDBC
:101D8800017A9B6807EE903A635906EE903AF8EEAE
:101D9800E78AF8EEE67AB8EEC78A17EE900A10F0EE
:101DA80047FA02460B4668461F4915F0D3F818EE65
:101DB800100A10F03DFA02460B4605A81B4915F01B
:101DC800C9F818EE900A10F033FA0B461849024683
:101DD8000AA8184C15F0BEF82068174901F010FB46
:101DE80020680FA901F00CFB6068694601F008FB48
:101DF800A06805A901F004FBE0680AA901F000FB4E
:101E080002F08EFC12B0BDEC028B70BD462600209D
:101E180000000020D7A7050800007A44E2A70508BB
:101E2800F3A7050804A8050815A8050826A80508A5
:101E380037A805087C0C002082AA050808B5144BB1
:101E4800144A1B780D2B01D8012104E00E2B01D177
:101E5800022100E000211170142253430E49C85892
:101E6800CA184FF47A730D4958430860516892684C
:101E78004B430B490B600B4B1A6009F08BFE0A4B66
:101E88000A4801221A70BDE80840FFF75ABE00BF91
:101E9800462600201C0E0020000000204C260020B2
:101EA800642C0020402C0020CD250020C8140020E0
:101EB800C4E700BF4FF6FF7070474FF6FF707047DA
:101EC8001FB5002947D04FF2DE7004F06DF80020EE
:101ED80004F040F90F2004F03BF81F4C1F4A412141
:101EE80001230A2004F06EF9042004F033F9236872
:101EF80028209621042B24DC0123194A04F062F9D6
:101F080003A90DF10E02206804F0E2FB0F2004F093
:101F18001FF8BDF80C00BDF80E1014380F24282245
:101F2800002380B2009404F043F8BDF80E10BDF809
:101F38000C000094143989B22822012304F038F8DF
:101F480009E0084A012304F03DF91E20A521064AAC
:101F5800012304F037F91FBD8C0C002048A80508A0
:101F68005BA8050877A805088DA8050837B51E4C95
:101F78002368042B05462BDC01A80DF1060104F0AB
:101F8800A5FBBDF80630BDF80420184904200DF063
:101F980003FA2368002B04DA1548164A164B592110
:101FA80005E0042B05DD1248124A144B5A2102F0B1
:101FB800DFFD04EB8302BDF8041001339180BDF806
:101FC80006102360052BD18008D1201D04F000FCE9
:101FD80000230B482360FFF7B4FD03E028460121E6
:101FE800FFF76EFF3EBD00BF8C0C0020A4A80508BB
:101FF800E9A80508562504080BA9050822A905081B
:102008001016002037B50B4C204602F050F90A4B49
:102018000A49009300250120094A0A4B019501F05D
:10202800EEFF294602462346284603B0BDE8304065
:1020380002F00CB8DC120020C91E0008BD1E000802
:10204800C31E0008751F00084FF6FF7070474FF653
:10205800FF70704730B54FF6E07087B003F0A4FF0B
:10206800002004F077F80F2003F072FF00212C4ABB
:102078002C4C01230A2004F0A5F8002003F068FF87
:10208800042004F067F80A201921274A012304F0E4
:1020980099F82521254A01230A2004F093F81F20E6
:1020A80003F056FF01230A203721214A04F08AF859
:1020B8002378002B31D001231E2096211D4A04F0DD
:1020C80081F862881C4902A814F044FF01231E20ED
:1020D800A22102AA04F076F8A288184902A814F0EE
:1020E80039FFAE2102AA01231E2004F06BF80F204D
:1020F80003F02EFF6088A188143880B20F252822AB
:102108000023009503F054FFA188608800951439D6
:1021180089B22822012303F04BFF07B030BD00BF6E
:1021280050A90508A40C002062A9050882A9050881
:10213800A2A90508C5A90508D7A90508E4A905089D
:1021480001B187E7704713B50DF1060101A804F046
:1021580071FA144B01221A705988BDF80420891AA3
:102168000E311C2919460AD89C88BDF80600201A89
:102178000E301C2803D899680131996001E00023CA
:102188008B60084B9968012905DD00229A601A7056
:10219800FFF702FD05E05A80BDF806209A80FFF798
:1021A80059FF1CBDA40C002037B50B4C204602F08B
:1021B8007EF80A4B0A49009300250120094A0A4B78
:1021C800019501F01CFF294602462346284603B024
:1021D800BDE8304001F03ABF101600204921000840
:1021E80051200008572000084F21000808B5064B69
:1021F80000221A70054B186814F042FB0448BDE829
:102208000840FFF79EBC00BFCD25002020360020E7
:10221800FC1700202DE9F04F514D524E85B0002497
:10222800284602F044F82246234647F6FF714E48F6
:102238000094019401F0FAF84FF6FF7703903946BD
:102248002246234649480094019401F0EFF83946A4
:1022580030602246234646480094019401F0E6F88F
:102268004FF001087060224623464FF6E07141485E
:10227800CDF80080019401F0D9F82346B0603946C2
:1022880022463D48CDF80080019401F0CFF83B4943
:10229800F0603B4A204601F0C1FD3A493A4A0746F8
:1022A800204601F0BBFD3949394A8046204601F0F5
:1022B800B5FD3849384A8146204601F0AFFD374917
:1022C800374A8246204601F0A9FD3649364A8346F8
:1022D800204601F0A3FD21468446039ACDF808C0A4
:1022E8002B46204601F0B2FE3C2132682B461420D2
:1022F80001F0ACFE3C2172682B46EC2001F0A6FEF2
:10230800B421B2682B460F2001F0A0FED2213A4634
:102318002B46E62001F09AFE642142462B46052012
:1023280001F094FE4A462B460520872101F08EFED7
:1023380052462B460520D22101F088FED2215A466A
:102348002B46502001F082FEDDF808C09B20D221E8
:1023580062462B4605B0BDE8F04F01F077BE00BFDE
:10236800040F0020B00C0020F1A90508FBA90508FE
:1023780075A7050877AA050879AA0508C5A7050855
:10238800F521000858A50508DD23000868A50508FB
:10239800DD24000804AA0508E52500080CAA05089C
:1023A800A125000814AA05085D25000808B50BF04A
:1023B800EFFF4FF441400CF029FD044B186807F07B
:1023C80051F9034B09221A7008BD00BF40260020AE
:1023D800CD25002010B50C4CFFF7E8FF0B4A002371
:1023E800B420052103F0EEFEA0684FF6E07101F07D
:1023F80059F8A068064901F003F80BF0C9FFBDE8D9
:10240800104002F08DB900BFB00C00207FAA05086B
:102418001CAA0508264B2DE9F7431888C00014F0BC
:1024280027FA054628B90520B421224A2B4603F08D
:10243800C9FE214BDFF878801D6000240BF0A8FF4F
:1024480026461E4FDFF8889023E009F0E1F93B6843
:10245800D9F8000045F8083C7B6845F8043C184B5F
:102468001B68C01807F0FEF8164B186809F09EFAAA
:10247800B8F8000094FBF0F080B24FF4FC630093CE
:1024880028210246322303F0EFFC04F59E7401363E
:102498000334B8F800300835B342D6DA0A4B186866
:1024A80007F0E0F8094B09221A70BDE8FE8300BF67
:1024B8002C3A002035AA050820360020EC370020E9
:1024C800C4250020F825002040260020CD25002026
:1024D8002836002010B5094CFFF79CFFA0684FF67E
:1024E800E07100F0DFFFA068054900F089FF0BF0FC
:1024F8004FFFBDE8104002F013B900BFB00C002038
:1025080043AA050810B5074C4FF6E071A06800F023
:10251800C9FFA068044900F073FFBDE8104002F04D
:10252800FFB800BFB00C00205DAA050810B5074C25
:102538004FF6E071A06800F0B5FFA068044900F00C
:102548005FFFBDE8104002F0EBB800BFB00C002000
:1025580073AA050810B50C4C0B2323700B4B0122F2
:102568001A70002002F0EEFF0948FFF7EAFA207817
:10257800FEF7B2FA074B032093ED000A0BF017FFA2
:10258800BDE81040D2E700BF582C0020780D00208D
:10259800581700202403002038B50C4D0C232B704D
:1025A8000B4B01241C70002002F0CCFF0948FFF7F8
:1025B800C8FA2878FEF790FA074B204693ED000AF0
:1025C8000BF0F5FEBDE83840B0E700BF582C0020FE
:1025D800780D0020581700202403002010B50C4C5B
:1025E800092323700B4B01221A70002002F0AAFF66
:1025F8000948FFF7A6FA2078FEF76EFA074B022083
:1026080093ED000A0BF0D3FEBDE810408EE700BF43
:10261800582C0020780D0020581700202403002093
:102628000CF040BA034A044800231370034A13709D
:10263800FFF787BA34380020FC170020CD2500208A
:102648002DE9F743384D394EDFF8FC800024284641
:1026580001F02DFE2246234647F6FF7134480094C8
:10266800019400F0E3FE4FF6FF7781463946224693
:10267800234630480094019400F0D8FE3946306073
:102688002246234640460094019400F0CFFE394686
:1026980070602246234640460094019400F0C6FE2E
:1026A8002346B0603946224640460094019400F023
:1026B800BDFE2149F060214A204601F0AFFB2049C8
:1026C800204A0746204601F0A9FB214680464A4693
:1026D8002B46204601F0BAFC3C2132682B462820C4
:1026E80001F0B4FC5A2172682B46192001F0AEFCA7
:1026F8007821B2682B46192001F0A8FC9621F268CF
:102708002B46192001F0A2FCD2213A462B46EC2098
:1027180001F09CFC0520D22142462B4603B0BDE8BF
:10272800F04301F093BC00BF4C100020C00C002007
:102738008DAA050895AA0508C5A705082D2600082D
:10274800A0AA05082926000879AA050870B5064632
:1027580000200D46144603F0FDFC4FF6FF7003F011
:10276800F7FBF2B273208621002303F00DFDEAB2D5
:102778007320AE21002303F007FDE2B27320D621B7
:102788000023BDE8704003F0FFBC08B5084B2020CB
:102798001860084B1860084B58221A600146FFF76A
:1027A800D5FF0648064B1860BDE8084006F05ABF3A
:1027B800D8010020D4010020D0010020C0E1E400AD
:1027C800EC25002008B5094B20201860084B58213B
:1027D8001960084B02461860FFF7B8FF0648074B18
:1027E8001860BDE8084006F03DBF00BFD8010020D2
:1027F800D4010020D001002080969800EC2500200C
:1028080008B5094B58201860084B20211960084B5F
:102818000A461960FFF79AFF0648074B1860BDE89B
:10282800084006F01FBF00BFD8010020D4010020D7
:10283800D0010020404B4C00EC250020034A0448FE
:1028480000231370034A1370FFF77BB93438002054
:10285800FC170020CD2500202DE9F74F444D454EAB
:10286800DFF83C810024284601F021FD224623465A
:1028780047F6FF7140480094019400F0D7FD4FF6E9
:10288800FF7783463946224623463C480094019404
:1028980000F0CCFD3946306022462346404600947D
:1028A800019400F0C3FD3946706022462346404635
:1028B8000094019400F0BAFD2346B06039462246E0
:1028C80040460094019400F0B1FD2D49F0602D4A76
:1028D800204601F0A3FA2C492C4A0746204601F06D
:1028E8009DFA2B492B4A8046204601F097FA2A493F
:1028F8002A4A8146204601F091FA214682465A46E4
:102908002B46204601F0A2FB3C2132682B461920B9
:1029180001F09CFB5A2172682B46192001F096FBA6
:102928007821B2682B46192001F090FB9621F268B5
:102938002B46192001F08AFBD2213A462B46EC207F
:1029480001F084FB822142462B46192001F07EFBD0
:10295800AA214A462B46192001F078FB1920524635
:10296800D2212B4603B0BDE8F04F01F06FBB00BF8A
:10297800A0180020D00C0020A8AA0508B6AA0508AF
:10298800C5A7050845280008C3AA0508092800089E
:10299800CCAA0508CD270008D5AA05089327000862
:1029A80079AA050810B50B4C204601F080FC0020E0
:1029B8000146224600F09AFD00200749074A01F027
:1029C8002DFAD221024623464FF48270BDE810400A
:1029D80001F03CBB58170020DEAA05080D2A0008A4
:1029E80070B5C9240AE0A8B200223146013502F0C8
:1029F8004BFCF02DF7D10134EF2C02D00025A6B204
:102A0800F1E770BD10B51A4C2378092B08D1194A83
:102A180000231370184A1370FFF7E2FF174823E0EA
:102A28000A2B0ED1164B186813F02AFF154A0023FB
:102A38001370114A1370144A1370FFF7D1FF13482B
:102A480012E0002002F07EFD114A00231360114AB3
:102A580013800D4B02221A700F4B186806F002FE05
:102A680022780E4B0E481A70BDE81040FFF769B87F
:102A7800CD250020780D0020770D0020040F0020C0
:102A880020360020790D0020343800204C1000201A
:102A9800C40D0020D20D002040260020EA25002089
:102AA80094110020034B01224FF4FC601A7003F0CC
:102AB8004FBA00BF770D0020044B054800221A705A
:102AC800044B0C221A70FFF73CB800BF770D0020AA
:102AD800A0180020CD25002007B50A4A002313704E
:102AE80004228DE80C00C6201022232356210CF066
:102AF800FFFA054B05480A221A7003B05DF804EB8B
:102B0800FFF71FB8770D0020CD2500204C100020BE
:102B180007B50A4A0023137004228DE80C00972099
:102B28001022232356210CF0E3FA054B054809220D
:102B38001A7003B05DF804EBFFF703B8770D0020B7
:102B4800CD250020040F002007B50B4B00221A707A
:102B5800082203238DE80C004920102223233D215D
:102B68000CF0C6FA054B064801221A7003B05DF84E
:102B780004EBFEF7E6BF00BF770D0020CD2500204F
:102B8800C814002008B501214FF080400EF0FFFB6B
:102B98000A4B002018700A4B18700A4B18700A4B21
:102BA80008221A70094B187003F0FEF9084B0948FF
:102BB80001221A70BDE80840FEF7C3BFF0250020C7
:102BC800D40D0020770D0020CD250020582C0020A2
:102BD80038360020600E002070B51F4C1F4E20684C
:102BE8004FF6E075294600F05DFC20681C4900F0AE
:102BF80007FC6068294600F055FC6068194900F038
:102C0800FFFBA068294600F04DFCA068164900F0BB
:102C1800F7FB01F085FD4FF47A6008F0C7FE2068E5
:102C2800294600F03FFC2068314600F0E9FB606867
:102C3800294600F037FC6068314600F0E1FBA068E7
:102C4800294600F02FFCA068314600F0D9FBBDE80A
:102C5800704001F065BD00BFE00C00207CAA0508AB
:102C6800EEA6050802A7050812A705080C4B10B523
:102C780000241C700B4B01221A70204608F0CAFF72
:102C8800204603F091F9084B0B221A7009F020FB3B
:102C98000AF065F80548BDE81040FEF752BF00BFCE
:102CA800770D0020582C0020CD2500206C15002021
:102CB8000F4A002310B513700E4A13700BF06CFE08
:102CC800044628B1FFF788FFBDE8104001F028BD91
:102CD80003F06AF909F022FA074B1C70074B072228
:102CE8001A7009F015FA0648BDE81040FEF729BF2A
:102CF800D40D0020770D0020582C0020CD25002071
:102D08008013002010B54FF0804001210EF03FFBEA
:102D1800114A00231370114A1370114A13700BF0F3
:102D28003BFE044628B1FFF757FFBDE8104001F00D
:102D3800F7BC03F039F909F0F1F906F0EFFC094B9B
:102D48001C70094B06221A7009F0E2F90748BDE821
:102D58001040FEF7F6BE00BFF0250020D40D00207D
:102D6800770D0020582C0020CD250020A80F00202A
:102D78002DE9F04F6D4DDFF810928BB000244FF61F
:102D8800FF78284601F093FA4146224623466848D0
:102D98000094019400F04AFB4FF6E0760427049073
:102DA80031462246234663480097019400F03EFBD3
:102DB80031460590224623465F480097019400F06B
:102DC80035FB414606902246234648460097019423
:102DD80000F02CFB594E41463060224623464846B7
:102DE8000097019400F022FB23467060414622467A
:102DF80048460097019400F019FB5149B060514AC8
:102E0800204601F00BF85049504A0746204601F089
:102E180005F84F494F4A8046204600F0FFFF4E49CB
:102E28004E4A8146204600F0F9FF4D494D4A8246F8
:102E3800204600F0F3FF4C494C4A8346204600F0F8
:102E4800EDFF4B494B4A84462046CDF80CC000F0B4
:102E5800E5FF49490790494A204600F0DFFF484905
:102E68000890484A204600F0D9FF21460990049A64
:102E78002B46204601F0EAF82146059A2B46C82041
:102E880001F0E4F80A21069A2B46C82001F0DEF882
:102E9800552132682B46782001F0D8F869217268EC
:102EA8002B46782001F0D2F87D21B2682B46782095
:102EB80001F0CCF805203A4628212B4601F0C6F847
:102EC800D22142462B46052001F0C0F8D2214A46BD
:102ED8002B46562001F0BAF8D22152462B46A6209E
:102EE80001F0B4F8B4215A462B46052001F0AEF89B
:102EF800DDF80CC0B42162462B46562001F0A6F836
:102F0800B421079A2B46A62001F0A0F8B421089A0C
:102F18002B46F62001F09AF8099AF620D2212B4682
:102F28000BB0BDE8F04F01F091B800BFFC170020CE
:102F3800E3AA0508ECAA0508F9AA0508E00C002090
:102F480004AB0508512B00080CAB0508752C0008CC
:102F580015AB05080D2D00081EAB0508B92C000897
:102F680027AB05088D2B000830AB0508192B000886
:102F780039AB0508E12A000842AB0508C12A000858
:102F88004AAB0508AD2A000879AA050807B5032346
:102F980008228DE80C004920102223233D210CF043
:102FA800A7F8044B044801221A7003B05DF804EB3B
:102FB800FEF7C7BDCD250020C81400202DE9F74332
:102FC800314E324F324D0024304601F070F922461E
:102FD800234647F6FF712F480094019400F026FA23
:102FE8004FF6FF78814641462246234638460094EC
:102FF800019400F01BFA41462860224623463846D1
:103008000094019400F012FA414668602246234673
:1030180038460094019400F009FA2346A860414616
:10302800224638460094019400F000FA1A49E860F4
:103038001A4A204600F0F2FE214607464A46334621
:10304800204601F003F83C212A683346192000F095
:10305800FDFF5A216A683346192000F0F7FF7821EE
:10306800AA683346192000F0F1FF9621EA68334632
:10307800192000F0EBFFEC20D2213A46334603B08A
:10308800BDE8F04300F0E2BFF010002079AA05087F
:10309800EC0C002052AB0508C5A70508952F0008C1
:1030A8001C4B1A781C4B10B51A7009F017F91B4BFA
:1030B8001B4A00241C6002202346CA2103F082F820
:1030C800204608F0A7FD174B1C80174B1C70174BA8
:1030D8001B78023B052B1CD8DFE803F003070B1312
:1030E800170FBDE81040FEF7A1B9BDE81040FEF784
:1030F8008BB9BDE81040FEF775B9BDE81040FEF782
:103108004DB9BDE81040FEF75BB9BDE81040FEF7C9
:1031180033B910BDEA250020CD250020C40D0020BC
:1031280078AA05083436002034380020582C0020AE
:1031380008B5084B186806F095FA002002F034FF2D
:1031480009F0C6F8044B05480B221A70BDE8084080
:10315800FEF7F7BC40260020CD2500206C15002086
:10316800114B10B500241C70104B186806F07AFA41
:10317800204602F019FF0E4B1B780B2B0ED8DFE808
:1031880003F006060D0D0D0D0A080D0D0D06094874
:1031980002E0094800E00948FEF7D3FC084B1C7020
:1031A800BDE8104009F094B8582C002040260020B3
:1031B800CD250020FC17002080130020A80F002038
:1031C800343800202DE9F041144C204601F06FF806
:1031D80000201349134A00F021FE1349134A0746F9
:1031E800002000F01BFE1249124A0646002000F09B
:1031F80015FED22105463A462346E62000F026FF72
:103208004B2132462346642000F020FF64206921C8
:103218002A462346BDE8F04100F018BF941100206B
:10322800CBA50508693100085AAB050839310008F3
:1032380066AB0508A930000808B508B143682BB982
:103248000348044A044B9B2101F092FC586908BDCD
:1032580073AB05086825040895AB050808B5FFF7A2
:10326800EBFF8068123080B208BD08B5FFF7E4FFB5
:103278004068063080B208BD2DE9F84F04468846FC
:10328800FFF7DAFF6689E589074606F1030905F1C4
:103298000F0AB8F1000F1FD01F2002F059FE204678
:1032A800FFF7DCFF83462046FFF7DFFF294603468A
:1032B8005FFA8BF2F0B202F08BFE042002F04AFFB4
:1032C8000B364FF6FF70033502F042FEB0B2A9B2DA
:1032D8003A68012302F076FF3D69204641464A4696
:1032E8005346A847BDE8F88F13B504460DF106010B
:1032F80001A803F09FF92046FFF79EFF6389BDF8F8
:103308000410BDF80620C91AE389D21A0339C36824
:103318000F3A204698471CBDF7B5044614200D46C1
:1033280016461F4613F0A4FA089BC7600361064BB4
:103338000649074A80E8700000930190054B002079
:1033480000F05DFEFEBD00BF813200087332000848
:1033580065320008F1320008704708B508B14368C3
:103368002BB90448044A054BAD2101F001FC58690A
:1033780008BD00BFB4AB05088025040895AB050857
:10338800F8B505460E46FFF7E8FF836B04461BB108
:1033980028463146984700E018466F8994F83C3033
:1033A800ED890EB9034310D0208E02F0D1FD608E56
:1033B80002F0E4FD94F8350002F0CCFE94F83430C5
:1033C80038462946224602F0FDFE002384F83C30A8
:1033D800F8BD08B5FFF7C1FF90F83500BDE8084013
:1033E80002F0CDBE38B5FFF7B8FF044613F038FE3B
:1033F800054694F8350002F0BDFE684380B238BD3A
:1034080038B50D46FFF7A9FF29462E22044613F0CA
:1034180057FE50B1204629462E2213F0A3FE002362
:1034280084F82E30012384F83C3038BD2DE9F74369
:10343800074640200E461546984613F019FA0446EA
:1034480028B91148114A124B4E2101F091FB114B3A
:10345800114A12498DE818000020114B00F0CFFDE9
:1034680039468146FFF7CCFF9DF82830268684F838
:1034780035300B9B6586A363002384F8348084F879
:103488003C304846BDE8FE83B4AB050898250408DF
:10349800D2AB050889330008DB330008ED33000898
:1034A8006133000810B50C46FFF757FF0123048667
:1034B80080F83C3010BD00BF4FF4A0707047C820A2
:1034C80070477047074B1B78022B07B508D1064B8E
:1034D8001B78022B04D001A80DF1060103F0AAF80D
:1034E8000EBD00BF34380020582C002073B50A4B9D
:1034F80006460D461446009300200849084A094B21
:10350800019000F07CFD294602462346304602B071
:10351800BDE8704000F09ABDCB340008C134000803
:10352800C7340008CD34000813B502AB03E9060020
:10353800436843B1027C0124082A9C7004D11B69AA
:103548002146984700E01C4620461CBD30B500289F
:103558002BD0058B002425E0036A1A7C012A05D1AB
:103568005B681A888A421BD1187F30BD052A06D1AC
:103578005B681A888A4213D193F82C0030BD032A5D
:1035880006D15B681A888A420AD193F8250030BDB3
:10359800062A05D15B681A888A4201D1D87A30BDDB
:1035A80001340430AC42D7D3002030BD08B1817556
:1035B80001207047F8B504460D46D0B1E175D0F842
:1035C80098309847012D0DD12746002606E0F86966
:1035D80000F10802436906CA98470136238B04376D
:1035E8009E42F4D3D4F898302046294698470120C3
:1035F800F8BDF8BDF8B50546084617460E4613F05F
:103608002FFD013FB84234BF04463C463CB1284632
:103618003146224613F0A6FD00232B55F8BD2C7029
:10362800F8BDF7B5044600200090019000296CD041
:103638000E8B68E000F1080351F823301D7C042D3F
:1036480004D15D682D88954247D0013000F1080308
:1036580051F823301D7C012D04D15D682D889542D9
:103668003BD0013000F1080351F823301D7C052DB3
:1036780004D15D682D8895422FD0013000F10803F0
:1036880051F823301D7C032D04D15D682D889542A7
:1036980023D0013000F1080351F823301D7C022D9E
:1036A80004D15D682D88954217D0013000F10803D8
:1036B80051F823301D7C072D04D15D682D8A954271
:1036C8000BD0013000F1080351F823301D7C062D82
:1036D80008D15D682D88954203D103F10801204681
:1036E80015E0013000F1080351F823502B7C082B1A
:1036F80009D16F683F88974204D105F10801204637
:103708001A4605E00130B04294D3204669460822A3
:1037180013F05EFB2046FEBDF8B505460F4616467B
:10372800002830D04388032B2FD0202013F0A0F896
:10373800044600282BD040F80C5B39460C22FFF7D2
:1037480059FF1820E66113F093F80646B8B1022332
:103758000374012363760F4B446063600E4BA360D0
:10376800002323766B8805EB830201339BB2012B80
:1037780050606B800CD16A685268137608E0204666
:1037880013F07EF804E0064602E0002600E0064654
:103798003046F8BDE4A4040882A1040837B545689A
:1037A80002AB03E906003DB3037C0124042B85F832
:1037B800314022D1688E02F0CBFB95F8300002F040
:1037C800C9FC95F8343043B9BDF80200BDF80610BD
:1037D800AA1C234602F0F6FC0FE0012B03D108488F
:1037E80040F2395104E0022B07D1054840F241511B
:1037F800044A054B01F0BCF92C4620463EBD00BFEB
:10380800E5AB050858700408E3AB0508F8B50446AD
:103818000F46164610B3838A0A2B20D0202013F0B7
:1038280027F80546E8B14460102200F1080039463F
:10383800FFF7E0FE4FF6FF73A08A2B801F236B80F3
:1038480000232B76831D013080B20128EE6144F8F5
:103858002350A08207D1A3691876F8BDF8BD0020CF
:10386800F8BD0120F8BD0120F8BD2DE9F3471D463C
:103878004B1C984282460C461746BDF828600DDD61
:1038880095420BDC01320AF101035B1A521BC8B2E4
:10389800D2B29BB22946009602F092FBAAF1020A24
:1038A8003046C4EB0A0A02F053FB4FF000084FF011
:1038B80001091FFA8AFA0BE0601C08EB050180B2C7
:1038C80089B252460023009602F072FB09F1010901
:1038D8007B1B08F1010899451FFA88F8ECD3BDE86D
:1038E800FC87F8B5C7B2144638461E460D4602F0A6
:1038F80071FB621E92B23846294602F06BFB3046D5
:1039080002F026FB022606E0A21B92B238462946A0
:1039180002F060FB0136A642F6D3F8BD73B5044643
:103928000E4600F11E001546009200233C2280B28C
:103938001E3E02F03DFBB1B220463C220123009519
:1039480002F036FB7CBD73B504460E4601381546B9
:1039580000920023032280B2013E02F029FBB1B29B
:10396800204603220123009502F022FB7CBDF7B517
:10397800089D2E7BEF7A1C463604AB7A06EB0726A9
:10398800F618431A687B06EB00602D18002001909A
:10399800121B08462146009501F002FFFEBD30B516
:1039A800456885B004AB03E906007DB101242C739A
:1039B8006D68BDF80800BDF80A109DF80C209DF848
:1039C8000E300095FFF7D3FF204600E0284605B0EB
:1039D80030BD2DE9F04385B004AB03E90600446827
:1039E800BDF80860BDF80C70002C41D0012384F8A4
:1039F800263094F825300BB9A26800E06268FFB25F
:103A0800BDF80A109DF80E30009230463A46FFF78E
:103A1800AEFF04F10C08022002F09CFB404613F0B4
:103A28001FFB054600B1451E0F3F0024153E1FFA37
:103A380087F90DE002F098FB02F09CFB04FB106193
:103A480089B248462022002302F0D6FB0134E4B2B2
:103A5800AC42EFD3002002F07BFAB8B2B1B24246D2
:103A6800012302F0C9FB002002F074FB012000E0F2
:103A7800204605B0BDE8F0832DE9F04385B004ABDE
:103A880003E906004568BDF80860BDF80C70002D14
:103A98003CD001236B762B7EBDF80A10012B0CBF9E
:103AA8006A68AA689DF80E300092FFB23A4630461E
:103AB800FFF75DFF0C35022002F04CFB284613F09F
:103AC800CFFA0E3F81460024163E1FFA87F80DE014
:103AD80002F04AFB02F04EFB04FB106189B240463B
:103AE8002022002302F088FB0134E4B24C45EFD9D0
:103AF800002002F02DFAB8B2B1B22A46012302F032
:103B08007BFB002002F026FB012000E0284605B0E0
:103B1800BDE8F0832DE9F04F85B00546DDF840900B
:103B2800029148469046039313F09AFADDF838A0BC
:103B3800DDF83CB00646294600242F4611E024B1A2
:103B4800B4420CBF5B46534600E0039B01F10805F5
:103B5800ADB200932846029A4346FFF708FF0134A6
:103B68002946B442EBDD002002F0F2F9022002F00F
:103B7800F1FA7D1D08F10508A8B21FFA88F14A4636
:103B8800012305B0BDE8F04F02F01CBB70B54068DA
:103B980086B006AB03E9060000282ED0012380F882
:103BA8002D308668164BF21A534243EB020390F805
:103BB8002C205AB1002B134D134B144A08BF1D4635
:103BC800134B00F11C0418BF13460AE0002B0D4DDF
:103BD8000D4B0E4A18BF1D460D4B00F10C0408BFD3
:103BE8001346BDF81200BDF81410BDF81620009653
:103BF80001950294FFF78EFF012006B070BD00BF4B
:103C0800C879040804760408AA7B0408E67704083F
:103C18008C7D040870B5446886B006AB03E90600DD
:103C280004B301236377A668104B227FF11A4B4235
:103C380043EB01030AB10BB904E01BB966680C4DEC
:103C48000C4B01E00C4D0D4BBDF81200BDF81410E3
:103C5800BDF8162000960C3401950294FFF75AFF20
:103C6800012000E0204606B070BD00BF148504089E
:103C78005081040832830408EA860408C0880408CE
:103C88002DE9F04385B004AB03E906004468BDF8AC
:103C98000860BDF80A90BDF80C50BDF80E80002CE5
:103CA80000F08C800123A3740220676802F052FAA6
:103CB8004FF6FF7002F062F9002002F049F9EDB208
:103CC8005FFA88F8A6F1160189B230462A464346BB
:103CD8000097FFF74CFE277A002F2ED1A28A2346A1
:103CE80000E00137974204D29969097E043300291C
:103CF800F7D002F039FA02F03DFAA9F116091FFAD5
:103D080089F90E2101FB10914FF6FF7208F10108A5
:103D18005FFA88F389B2009248462A46FFF7A5FD64
:103D2800022002F017FA1F2002F012F9A38A002BD2
:103D380038D0103DE8B2303E2CE0E3685C68A28AD7
:103D48002346013A002700E00137974204D29969D7
:103D5800097E04330029F7D002F006FA02F00AFAC5
:103D68000E2101FB10914FF6FF7208F101085FFA6E
:103D780088F389B2009248462A46FFF776FD02206A
:103D880002F0E8F91F2002F0E3F8A38A53B1103DCE
:103D9800E8B21A3E0637B1B254F827200123083298
:103DA80002F02AFA002002F0D5F94FF6FF7002F06F
:103DB800E5F81F2002F0CCF8012000E0204605B00D
:103DC800BDE8F0832DE9F0410546362088461446C3
:103DD8001F4612F04DFD0646E0B120F8025B414651
:103DE8002E22FFF707FCBDF8183086F8344073869A
:103DF8001820012386F8307086F8313012F038FD2B
:103E0800044618B104234660037404E0304612F0F7
:103E180037FD00E004462046BDE8F081F8B50646C7
:103E280024200F46154612F023FD0446D8B10F4B47
:103E3800068083600E4B39464360102200F10C0067
:103E4800FFF7D8FB01260023182025622377667721
:103E580012F00EFD054610B14460067404E02046D9
:103E680012F00EFD00E005462846F8BD148504084A
:103E78006E7F0408F8B506462C200F46154612F04A
:103E8800F7FC0446E8B120F80C6B39461922FFF715
:103E9800B1FB0D4BA562A3600C4B6360002384F853
:103EA80025301820012384F8263012F0E1FC05465D
:103EB80018B103234460037404E0204612F0E0FCC8
:103EC80000E005462846F8BD209E0408BE9A04086E
:103ED80010B50446142012F0CBFC20B10023438017
:103EE800014B0480036110BD2137000838B5054631
:103EF800442012F0BDFC0446C0B10E4B058243605D
:103F08000D4B0360012383740023037283820B4BE0
:103F18000364182012F0ACFC054618B1072344606E
:103F2800037404E0204612F0ABFC00E00546284686
:103F380038BD00BFB4960408AA92040815380008D2
:103F48002DE9F04105463420884614461F4612F0F4
:103F58008FFC064620B3144B05808360134B414603
:103F68004360102200F10C00FFF744FB214606F1E4
:103F78001C001022FFF73EFB002386F82C30182087
:103F88000123376386F82D3012F072FC044618B10D
:103F980005234660037404E0304612F071FC00E02B
:103FA80004462046BDE8F081C87904082274040854
:103FB8002DE9F041044614200D461646984612F0A5
:103FC80057FC0746B8B1069B048003610023C372FF
:103FD80001234560068180F80A800373182012F0D7
:103FE80047FC044618B106234760037404E03846CA
:103FF80012F046FC00E004462046BDE8F0812DE9B9
:10400800F041044618200D461646984612F030FC3A
:104018000746B8B101238370069B04800361079BA0
:1040280045608660C0F80C804361182012F020FCBF
:10403800044618B108234760037404E0384612F0B8
:104048001FFC00E004462046BDE8F0812DE9F3415D
:1040580098461B8B1D2B05460C4617464FF0000053
:1040680000F2B480B5F5A07F0090019000F2AE8018
:10407800F02900F2AB80127CADF80610511EADF8A5
:104088000250072900F28A80DFE801F045595E04F2
:10409800456A14767B684E4A7A611A8893F83430F8
:1040A8003A80013BDBB2012B7FD8ADF80240ADF876
:1040B80006507AE005F11602ADF8002004F1160268
:1040C800ADF8042002AE434A16E903007A6107F10D
:1040D800080282E8030003F10802013348F822705D
:1040E800A8F818307B681A8A187A3A8000286CD1A8
:1040F800FFF7FCFE3849436859603849DF600126FC
:10410800163D196002461E72A8B2E1B24346FFF797
:104118009DFF30465AE0012A0CBF314B314B78687D
:104128007B6130F80C3B3B8012F09AFF431CDB00AC
:104138001A34ED18ADF80440ADF8005035E07B684E
:10414800294A1B687A6102E0284A7B687A611B88E1
:1041580014353B80ADF800501434ADF8044024E029
:104168007B68234A7A611A883A801A899B7AAD1843
:10417800ADF80050E418F0E77E681E4B7B61338889
:1041880038463B8073689847013D4519ADF80050A3
:10419800B36838469847013C0419DEE71648174AC1
:1041A800174B40F21A3100F0E3FC02AA12E90300AF
:1041B80007F1080383E80300B8F8183003F1080290
:1041C800013348F82270A8F818300120BDE8FC81B6
:1041D800A5370008893C0008A08E0408968A0408C0
:1041E8001D3C0008953B0008813A0008DB390008AF
:1041F800A739000831350008E5AB050868700408E0
:10420800E3AB0508F8B51646002834D01378002B20
:104218002ED0028B002327E0046A257C042D21D1AF
:1042280065682F888F421DD195F8313053B16F8E54
:1042380001F0B4FE04F1080268866369204606CAE4
:1042480098476F86A81C31462E22FFF7D3F995F8B8
:1042580031307BB104F108026369204606CA9847E9
:104268000120F8BD013304309342D5D30020F8BDB6
:104278001846F8BD0120F8BD70B5B8B1068B0446E4
:10428800002310E0256A287C04280AD16D68288854
:10429800884206D11046A91C2E22FFF7ABF901204F
:1042A80070BD01330434B342ECD3002070BD38B57F
:1042B800044620B3134BC361134BC0F89830134B1B
:1042C800C0F89C30124B00257822C0F8A0308575C4
:1042D800C5750583294600F1200012F0BBFDD4F80E
:1042E80098302046294698470A4A1388312B07D820
:1042F800094941F8234001331380012038BD38BDF6
:10430800284638BDBD350008B535000855350008C4
:104318002B360008FC0C0020441900202DE9F04140
:104328000446002800F0B380078B02460025A8E069
:10433800136A1E7C042E00F08780012E23D1586852
:1043480003888B4240F09B8005F1080712F098FA29
:1043580054F827004FF00008C0F8048012F090FAD3
:10436800228B531E9D4208D00732238354F8221013
:1043780044F8271044F8228002E044F82780258377
:104388003046BDE8F081052E5ED0032E5CD0022EAB
:1043980013D15B68186803888B4270D14388013B4E
:1043A8009BB243800BB912F06BFA05F1080654F87A
:1043B8002630586812F064FA4EE0072E21D15E6864
:1043C800338A8B425BD1002706E0BB1D013756F8C4
:1043D800230012F055FAFFB2B38ABB42F5D8002782
:1043E800B78205F1080654F82630586812F048FAE2
:1043F80054F8260033E044F8267025830120BDE8F0
:10440800F081062E1ED1586803888B4237D105F1FA
:10441800080612F035FA54F826000027476012F013
:104428002FFA228B531E9D4209D00833013A54F8C3
:104438002310228344F8261044F82370DEE744F85A
:1044480026701AE0082E1AD1586803888B4216D1B4
:1044580012F016FA05F1080654F8260000274760FE
:1044680012F00EFA228B531E9D42C4D0073254F824
:10447800221044F8261044F822702383BEE7013541
:104488000432BD42FFF454AF0020BDE8F081BDE81E
:10449800F08170B5044600282AD0068B751E0836B0
:1044A80000EB86061EE056F8043D1A7C042A13D059
:1044B800012A11D0052A0FD0032A0DD0022A02D1D1
:1044C8005B681B6809E0072A02D15B68198A05E066
:1044D800062A01D0082A04D15B6819882046FFF70C
:1044E8001DFF013D681CDED100232383012070BD20
:1044F80070BDF0B528B30023068B1A461EE0046A87
:10450800257C072D18D16468258A8D4214D1A78A85
:10451800002504EB83040DE004EB050C0435DCF8FE
:1045280018C09CF818C0BCF1010F03F1010301D1B8
:10453800D8B2F0BDBB42EFD301320430B242DED371
:104548000020F0BD70B508B3048B00231BE0026A9D
:10455800157C072D15D15268158A8D4211D100237B
:10456800958A11461C46012007E013B996693076F2
:1045780001E08E69347601330431AB42F5D3012072
:1045880070BD01330430A342E1D3002070BD2DE992
:10459800F04128B30023078B1A461EE0046A257CE5
:1045A800072D18D16468258A8D4214D1B4F814C037
:1045B800002504EB83040CE066190435B66996F807
:1045C8001880B8F1010F03D106F10800BDE8F081A9
:1045D80001336345F0D301320430BA42DED3002000
:1045E800BDE8F0812DE9F04700282FD00023B0F86E
:1045F80018C01D4627E0046A267C072E21D164686E
:10460800268A8E421DD1B4F81480002604EB830953
:1046180015E009EB0604A7693C7E012C0DD192F840
:1046280000A0BAF1000F08D007F1080011461022C7
:10463800FEF7E0FF2046BDE8F08701330436434526
:10464800E7D3013504306545D5D30020BDE8F087B0
:10465800F0B5B0B1068B002510E0046A277C062F60
:104668000AD1646827888F4206D123819DF81430C7
:104678006260A3720120F0BD01350430B542ECD36D
:104688000020F0BD10B500210446FEF793FF204638
:104698000121BDE81040FEF78DBF38B598B1048BF5
:1046A800024600230CE0106A058804328D4206D1C8
:1046B80000F10802436906CA9847012038BD013352
:1046C800A342F0D3002038BD10B50C460021FEF7F8
:1046D80071FF20460121BDE81040FEF76BBF13B5FE
:1046E80002AC04E90C00BDF80230834206D8BDF8DC
:1046F8000030834234BF0020012000E00020BDF8D4
:1047080006308B4206D8BDF804308B4234BF0021F6
:10471800012100E00021002818BF0846C0B21CBDD6
:1047280038B5114B114A1988002319E052F8045F73
:10473800A87D012812D100240CE004F1080355F8E3
:104748002300037C082B03D1436800211B69984789
:104758000134A4B22B8BA342EFD838BD01339BB2EE
:104768008B42E3D138BD00BFFC0C0020401900206B
:10477800704770B5094CA5787DB9094B1E78012E94
:104788000BD16368013363606268064B9A4204D9AF
:10479800284601F0A1FCA670656070BDFC0C0020E5
:1047A8009801002040420F00054A9060134602E03D
:1047B80099680139996091680029F9D1704700BF5B
:1047C800FC0C0020F0B585B001F032FF002800F0A5
:1047D8004981002502A80DF10A01ADF80850ADF88D
:1047E8000A5001F027FF03A80DF10E01ADF80C5097
:1047F800ADF80E5001F06AFFBDF80C10BDF80820A6
:104808000091BDF80E10BDF80A3001912C46964D66
:10481800964908200AF0C0FDA878012803D101F0C4
:104828005BFCAC7019E1924B5B78012B40F0158171
:10483800AB78002B40F011816B6029888D4A09E123
:1048480052F8046FB07D012840F002810025FAE09B
:1048580005F10803BDF8080056F82340BDF80A1012
:1048680004F108030CCBFFF73AFF002800F0E980B9
:10487800237C013B062B00F29F80DFE803F004292C
:10488800159D1F9D4C006668012304F108053377C8
:1048980095E8060063692046984700233377204649
:1048A800636995E8060086E0636893F8252012F1AD
:1048B800FF3218BF012283F8252077E0636893F858
:1048C8002C2012F1FF3218BF012283F82C206DE052
:1048D8006268137E1568002B6ED16E882F462946B4
:1048E800184606E051F804EFDEF804E001338EF8CC
:1048F8001800B342F6D301231376002607E057F8D1
:10490800040F00F10802436906CA984701366B880C
:104918009E42F4D350E0656820892E68A37B227BF1
:104928000096A0F1160189B2FFF721F81420FFF7CD
:104938003BFF2B7AC3B9AF8A29461A461E4609E0BF
:10494800886990F818E00676BEF1010F08BF134693
:1049580004310132BA42F3D301220BB9AB6924E026
:10496800053355F8233020E06368DB685A68002374
:10497800908A154619461F4609E0AE6996F818E070
:104988003776BEF1010F08BF0B460435013181426D
:10499800F3D3411E8B4203D1053052F8203003E097
:1049A80004D2073352F8233001221A7604F10802A0
:1049B80006CA636920469847237C013B072B4CD8DD
:1049C800DFE803F00410074B0A0D123A63681B6A0C
:1049D80034E063689B6A2DE063681B6B2AE06368B8
:1049E8001B6927E0636824E063681A7A7AB9988AB1
:1049F8001946013800E00132824204D28C69247ED3
:104A08000431002CF7D0063253F8223011E0DB686D
:104A18005A68908A11460138002300E00133834226
:104A280004D28C69247E0431002CF7D0063352F866
:104A38002330DB69984710E06368DB6820469847B5
:104A48000BE00135ADB2338BAB423FF601AF04E06A
:104A580001339BB28B427FF4F3AE01F02FFE0F209F
:104A6800FFF7A2FE05B0F0BDFC0C00200BAC05085A
:104A78009801002040190020034B9A6812B19A68E7
:104A8800013A9A60704700BFFC0C00202DE9F347FB
:104A98000120DFF8D080DFF8D09001460CF016F83E
:104AA800012400254FF48076022740466946009687
:104AB8008DF804708DF805408DF806508DF8074084
:104AC8000BF05CFC4046082122460BF0D7FC244B37
:104AD800DFF898801A6844F2A243B2FBF3FA0AF1AD
:104AE800FF3A204621461FFA8AFA0CF01FF8C8F848
:104AF80004A048464146A8F80050A8F80250A8F873
:104B0800085088F80A500CF0ADFB7023A8F80C3058
:104B18000423A8F810300AF1FF3A6323642203FB48
:104B28000AF3B3FBF2F39BB2C8F8143008F10C0196
:104B38004846A8F80E40A8F81870A8F81A50A8F81F
:104B48001C60A8F81E500CF0ABFC484621460CF03F
:104B58001EFC484621460CF024FFBDE8FC8700BF38
:104B6800E401002000000240000001400C0D00207C
:104B780083B50E460746154910201C4615460AF00F
:104B88000BFC102012490AF007FC102011490AF00A
:104B980003FC10200E490AF0FFFB002310200E49E9
:104BA80001930AF0F9FB334610200C493A460AF003
:104BB800F3FB10200A492A460AF0EEFB10200949A7
:104BC80022460AF0E9FB019B0133E7E745AC0508FB
:104BD8004AAC05086AAC05087AAC05088AAC050831
:104BE8009FAC0508B0AC050808B5164B1A6A013227
:104BF8001A621A6A012A1A4603D0134840F21E2183
:104C08000FE05862194602E04B6A013B4B62506A5A
:104C18000C4B0028F8D11A6A012A06D00A4840F23B
:104C280029210A4A0A4BFFF7A3FF1A6A013A1A62B6
:104C38001B6A2BB10448054A064B40F22B21F2E7C8
:104C480008BD00BF0C0D0020C1AC050846A804082B
:104C5800EBAC0508FCAC050810B5084C0221002295
:104C680020460BF000FC44F6FF70FFF7BDFF20461E
:104C780002210122BDE810400BF0F5BB0004024000
:104C88000C4B0D491A6844F2A2436428B2FBF3F3B3
:104C9800D4BF20EAE0706420013B9BB24B60013B2B
:104CA80058436422B0FBF2F080B2486103480C31EB
:104CB8000CF079BBE40100200C0D0020000001403D
:104CC80010B5134B93F828202AB11248124A134BF7
:104CD80040F209310EE0012283F8282066234FF0C4
:104CE800C042013BDBB2108033B90A480A4A0C4B78
:104CF80040F21331FFF73CFF1488A4B28442F0D18C
:104D0800084B1980024B002283F8282010BD00BFF1
:104D18000C0D0020C1AC050850A804080DAD05080D
:104D2800E3AB05080000026010B5FFF7AFFE642092
:104D3800FFF7A6FF21210720FFF7C2FF3220FFF768
:104D480053FF01210020FFF7BBFF3220FFF74CFF84
:104D580023210720FFF7B4FF3220FFF745FF00218A
:104D68001020FFF7ADFF41F28830FFF73DFF3321F8
:104D78000720FFF7A5FF3220FFF736FF112046F680
:104D88003001FFF79DFF3220FFF72EFF4FF4C0617F
:104D98000220FFF795FF3220FFF726FF122046F684
:104DA800EB41FFF78DFF3220FFF71EFF03204AF685
:104DB800A401FFF785FF3220FFF716FF00210C2022
:104DC800FFF77EFF3220FFF70FFF0D2040F60C01A2
:104DD800FFF776FF3220FFF707FF0E204FF42C5124
:104DE800FFF76EFF3220FFF7FFFEB0211E20FFF70E
:104DF80067FF3220FFF7F8FE012042F63F31FFF748
:104E08005FFF3220FFF7F0FE05200021FFF758FF73
:104E18003220FFF7E9FE00210620FFF751FF32207C
:104E2800FFF7E2FE16204EF61C71FFF749FF32200D
:104E3800FFF7DAFE172040F20311FFF741FF322097
:104E4800FFF7D2FE00210B20FFF73AFF3220FFF7D1
:104E5800CBFE00210F20FFF733FF3220FFF7C4FEFF
:104E680041200021FFF72CFF3220FFF7BDFE422032
:104E78000021FFF725FF3220FFF7B6FE002148206A
:104E8800FFF71EFF40F23F143220FFF7ADFE214628
:104E98004920FFF715FF3220FFF7A6FE00214A2020
:104EA800FFF70EFF3220FFF79FFE00214B20FFF790
:104EB80007FF3220FFF798FE44204FF46F41FFF7B9
:104EC800FFFE3220FFF790FE00214520FFF7F8FE95
:104ED8003220FFF789FE21464620FFF7F1FE3220F7
:104EE800FFF782FE302040F20771FFF7E9FE32201B
:104EF800FFF77AFE31204FF40171FFF7E1FE32200F
:104F0800FFF772FE32204FF40171FFF7D9FE40F22D
:104F180002543220FFF768FE21463320FFF7D0FE07
:104F28003220FFF761FE342040F20751FFF7C8FE38
:104F38003220FFF759FE35204FF40171FFF7C0FE0C
:104F48003220FFF751FE36204FF40171FFF7B8FE0B
:104F58003220FFF749FE21463720FFF7B1FEA4F5BE
:104F680000743220FFF740FE21463A20FFF7A8FEE2
:104F78003220FFF739FE2F2041F2BE21FFF7A0FEB5
:104F88003220FFF731FE21463B20FFF799FE322001
:104F9800FFF72AFE00212320FFF792FE3220FFF7B9
:104FA80023FE00212420FFF78BFE3220FFF71CFE92
:104FB80025204FF40041FFF783FE3220FFF714FE4F
:104FC80000214F20FFF77CFE3220FFF70DFE4E2018
:104FD8000021FFF775FE3220BDE8104004E608B551
:104FE800124B93F829202AB11148124A124B40F269
:104FF80023310FE0012283F82920222166234FF074
:10500800C042013BDBB2118033B90948094A0B4B56
:105018004FF44F71FFF7ACFD108880B22228F0D111
:10502800024B002283F8292008BD00BF0C0D002088
:10503800C1AC05085DA804080DAD0508E3AB05087B
:1050480010B51B4B032826D8DFE800F0021A080E1B
:105058001C8841F2280246F628000AE01C8841F222
:10506800080246F6080004E01C8841F2300246F6C1
:10507800300049F241318C4214BF014611460BE021
:10508800188846F6200249F24131884214BF114679
:105098004FF4815100E000211A8848F689139A429A
:1050A80002D11120FFF70CFEBDE8104097E700BFC2
:1050B8009A010020014B18800A2095E50000026043
:1050C8004FF0C043188003F500331A881A881888EF
:1050D80080B270474FF0C04322221A8003F5003394
:1050E80082B01A8892B2ADF806201B889BB2ADF840
:1050F8000630BDF8060080B202B07047072040F2C3
:105108007311DDE507200021DAE582B0044BADF824
:105118000600BDF8062092B25A8502B0704700BF5B
:105128000C0D002082B0044BADF80600BDF8062037
:1051380092B25A8002B070479A010020014B80B2A7
:1051480018807047000002604FF0C04380B218809A
:105158007047024B80B21880704700BF00000260A1
:105168004FF0C04380B218807047024B80B218805D
:10517800704700BF0000026082B0044B0190019AA2
:10518800DA62DA6A002AFCD102B070470C0D0020FE
:1051980070B54FF0C0452A242C800A4C060AC0B2CC
:1051A80026802080100AD2B2208022802B222A80DA
:1051B8000A0A2280C9B21A0ADBB22180228023801F
:1051C80070BD00BF0000026010B50B4614460246D1
:1051D800FFF7DEFF4FF0C0432C22A0B21A80BDE8D3
:1051E800104067E70B4B1A8848F689139A4210B5A6
:1051F80004460AD1C1F1EF014E2089B2FFF760FDE4
:105208004F202146BDE810405AE502460B46BDE84E
:105218001040BDE79A01002008B5FFF7E3FF0F4BE8
:105228001B78012B4FF0C0420D4B0FD12E2111805E
:105238001A881A881B8892B202F0FC0002F478429D
:1052480042EAC000C3F3C423184308BD22211180D9
:105258001A881A88188880B208BD00BF141A00205E
:105268000000026070B5074D06460124214630460D
:10527800FFF7D2FF0134A4B2C82C25F8020FF5D1EC
:1052880070BD00BF3638002010B5084B1B78012BC5
:10529800144602D1BDE8104096E7FFF7A3FFFFF7D9
:1052A8009EFE2046BDE8104004E700BF141A002007
:1052B80070B5074D064601242146013435F8022F02
:1052C8003046A4B2FFF7E0FFC82CF5D170BD00BF8F
:1052D8003638002070B505460E46FFF7C3FF012497
:1052E8002146013428463246A4B2FFF7CDFFC82C28
:1052F800F6D170BD2DE9F84F0C4693460546C71800
:10530800DFF82CA00AE0BAF82A20B1B292B24046DF
:10531800FFF7BAFF01364E45F5DB0135BD4205DA28
:10532800264604EB0B091FFA85F8F4E7BDE8F88F69
:105338000C0D00202DE9F04104460D461646BDF837
:105348001880032B39D8DFE803F00B3519273819F3
:1053580080B2294642460137FFF796FFBFB200E008
:105368000027B742F3D1BDE8F081E01B80B229469F
:1053780042460137FFF788FFBFB200E00027B74277
:10538800F3D1BDE8F081E91B89B2204642460137D6
:10539800FFF77AFFBFB200E00027B742F3D1BDE8BC
:1053A800F081791989B2204642460137FFF76CFF30
:1053B800BFB200E00027B742F3D1BDE8F08170B575
:1053C800194B1A4A598E92F9004064180025A4B264
:1053D8008AB0AC4208BF0124C62C28BFC624157069
:1053E8000F264FF6FF721E865C865A8519202B46BB
:1053F800009221460A22FFF79DFF21463046FFF71B
:105408000BFF224603460A4902A811F0A3FD02AA8F
:1054180006A8084911F09EFD3220D22106AA2B4683
:1054280000F0D0FE0AB070BD0C0D0020811A0020DB
:1054380022AD05082AAD05082DE9F341BDF8205035
:105448000C4690461F461A46002306460095FFF76D
:1054580071FF611E414430463A46002389B20095E7
:10546800FFF768FF30462146424601230095013E7A
:10547800FFF760FFBF19B8B22146424601230895DD
:1054880002B0BDE8F04155E770B50D461C49044629
:10549800088848F6891188422CD1C5F1F001661EAA
:1054A8009E198A1AC5F1EF0392B29BB29A422CBF99
:1054B80011461946EF2928BFEF219A4238BF1346F3
:1054C80043EA0121B6B289B24420FFF7F9FBA642AC
:1054D80034BF314621464520FFF7F2FBA64238BFCC
:1054E800264640F23F139E4234BF314619464620B5
:1054F800FFF7E6FB20462946BDE8704072E600BF8C
:105508009A01002000200146F0224FF4A073BBE767
:1055180070B54FF0C0452A242C80094C060A268015
:105528002080080A208021802B212980110A2180CF
:1055380022801A0A228023802C232B8070BD00BF72
:105548000000026070B5114B1B78012B044607D18F
:10555800002040F23F110246EF23FFF7D9FF04E095
:10556800FFF7D0FF0020FFF76BFDF02509E0013EB3
:105578002046B6B2FFF79EFD002EF8D1013DADB230
:1055880015B14FF4A076F2E770BD00BF141A0020E1
:105598002DE9F04F1C463E4B87B01B78039183469C
:1055A8009DF8441010980591012B039B0490924696
:1055B8001FFA8BF09AB208D1411E531E09195344A1
:1055C80089B29BB2FFF7A4FF09E01FFA8AF51146DA
:1055D800A3B22A46FFF758FF0020FFF731FD002746
:1055E800DDF80C803E4640F23F1CA14639E0BBF195
:1055F800000F2EDB65452CDC0398002829DBB8F169
:10560800EF0F26DC220702D1002CC8BF0136214942
:105618002140002903DA013961F00F010131059AAF
:105628000AB1C1F10F01049830F8162003FA01F10C
:105638000A4012B26AB118494A8D029392B2A8B2CE
:105648001FFA88F1CDF804C0FFF71EFEDDF804C08C
:10565800029B013401354C45C9DB0136013708F19D
:105668000108574503DA5D4600240123F3E7084B98
:105678001B78012B08D1002040F23F110246EF238E
:1056880007B0BDE8F04F43E707B0BDE8F04F39E792
:10569800141A00200F0000800C0D00202DE9F74F90
:1056A8001F463B4BDDF830801B7816469DF83420AA
:1056B800012B044601920D4680B28AB208D1411EE0
:1056C800531EC9199B1989B29BB2FFF721FF09E044
:1056D8001FFA86FE1146BBB27246FFF7D5FE0020C0
:1056E800FFF7AEFC4FF0000BDA463DE0002C30DB54
:1056F80009EB040340F23F1293422ADC002D28DB19
:105708000BEB0503EF2B24DC19F00F0F04D1B9F1D3
:10571800000FC8BF0AF1010A1E4B09EA0303002B58
:1057280003DA013B63F00F030133019A0AB1C3F1B5
:105738000F03012202FA03F338F81A2013401BB2B0
:1057480013B1154B588D01E0144A508880B2FFF709
:10575800B1FC09F1010901E04FF00009B945C5DBC9
:105768000AF1010A0BF1010BB345F5DB084B1B7875
:10577800012B08D1002040F23F110246EF2303B06D
:10578800BDE8F04FC4E603B0BDE8F04FBAE600BF8D
:10579800141A00200F0000800C0D00209A01002030
:1057A8002DE9F0411C4F069C3F789DF81C60012FA5
:1057B80002FB03F580B28FB209D1411ECB1899B212
:1057C8007B1E9A1893B23A46FFF7A2FE07E092B200
:1057D8009BB23946FFF758FE0020FFF731FC00273F
:1057E80009E034F8020B1EB1030A43EA002080B234
:1057F800FFF760FC0137AF42F3DB074B1B78012B47
:1058080007D1002040F23F110246EF23BDE8F041E6
:105818007EE6BDE8F04175E6141A00202DE9F04354
:105828001F2093B0FFF78EFE4FF47840FFF78AFEF3
:105838004FF6E0754FF4FC60FFF784FE2846FFF74B
:1058480081FE0020514CFFF77DFE00204FF6FF79C6
:10585800014664220346A4F82A90CDF80090FFF789
:1058680069FD00200A2164220346CDF80090FFF765
:1058780061FD00200146642201234FF478476585C5
:105888000095FFF757FD7720EF21C82200234FF43A
:10589800FC6667850097FFF74DFDBD213222012385
:1058A80040F23F1066850096FFF744FDA0203222A3
:1058B8000023782167850097FFF73CFDA020782119
:1058C800322201234FF01F0866850096FFF732FD4C
:1058D800A020782132220223A4F82A80CDF8008063
:1058E800FFF728FDA0207821322203236585009543
:1058F800FFF720FD264B2749A3F8028002AD3C2282
:10590800284611F065FAEB20C321052230230095C3
:105918000025A4F82A900195FFF7C0FE32210A203D
:1059280096220B4667850097FFF786FD32213C20BB
:1059380096220B4666850096FFF77EFD32210B46C0
:1059480096226E20A4F82A80CDF80080FFF774FD17
:10595800FFF7D8FBFFF7D2FB3220FFF791F9284673
:10596800FFF78EF96420FFF78BF90B4B03F1100258
:105978008DE8240028465A681B682946FFF710FF5F
:105988001195119B01331193FBE700BF0C0D00200B
:105998009A01002072A8040830CD01082DE9F14FC2
:1059A800FFF774F84FF0C0456420FFF769F9012745
:1059B800FFF752F94FF028096D48FFF715F92F80C6
:1059C8000520A5F8009003F04DFACF232B80694BF2
:1059D800002683221E801A8030221A80ED222A8017
:1059E8004FF064080322A3F800801A8012221A805C
:1059F80081221A80E8222A8085221A8079221F8033
:105A08001A80CB222A8039221A804FF0340C0224C3
:105A18002C21F72219801E80A3F800C01C802A8040
:105A280020221A80EA222A80C0221E80C1211E80DC
:105A38002A8026221A80298011211980C5212980CF
:105A4800352119803E211980C7212980BE2119805E
:105A5800362129803A205521A3F800902880198002
:105A6800B12129804FF0100BF2211E80A3F800B05D
:105A78002980082119802A80E0221F804FF01F0901
:105A88002A801A22A3F800904FF0180A1A800F21D2
:105A98000A22A3F800A01A8019800621198045213E
:105AA8001980872119803221198007211A804FF027
:105AB800E10E19801C80052419801C801E80A5F821
:105AC80000E04FF0250E1E80A3F800E04FF0270EEF
:105AD800A3F800E01C80A3F800B04FF0090BA3F86E
:105AE80000B04FF0780B1880A3F800B04FF04D0BC2
:105AF800A3F800B01C800D24A3F800A01C80382453
:105B08001C8018802A20A3F80090EF2428802B20DE
:105B18001E801E801E801C8028803F201E801E80C4
:105B28001F801880B720A5F800C028801980B621EA
:105B380029801A8082221A801122A3F800E04046A8
:105B48001E8029272A8003F08DF940462F8003F014
:105B580089F90948FFF748F82C232F8030462B8015
:105B680040F23F113246234601B0BDE8F04FCFE482
:105B7800400D03000000026040420F002DE9F04193
:105B8800022098B0012100240AF0A0FF0125022676
:105B98008048169616A98DF85D408DF85E408DF800
:105BA8005F408DF85C500AF0E9FB182029460AF09E
:105BB8008DFF284629460AF0A1FF21460C22764887
:105BC8000AF05CFC0C22744829460AF057FC0421B0
:105BD8000C2271480AF052FC05210C226E480AF08A
:105BE8004DFC07210C226C480AF048FC08210C22C5
:105BF80069480AF043FC09210C2267480AF03EFC78
:105C08000A2165480C220AF039FC0B2162480C2253
:105C18000AF034FC0E210C225F480AF02FFC0F21F9
:105C28000C225D480AF02AFC07210C225B480AF086
:105C380025FC08210C2259480AF020FC09210C22D5
:105C480056480AF01BFC0A210C2254480AF016FC9C
:105C58000B210C2251480AF011FC0C210A464F482E
:105C68000AF00CFC0D210C224C480AF007FC0E210E
:105C78000C224A480AF002FC0C2248480F210AF07C
:105C8800FDFB4CF6B3734448169316A98DF85C6077
:105C98008DF85E408DF85F408DF85D500AF06EFB20
:105CA80016A94FF680733D4816938DF85C608DF801
:105CB8005E408DF85F408DF85D500AF05FFB40F65E
:105CC800B830FEF791FFFEF7C7FF40F6B830FEF791
:105CD8008BFF0F2311934FF4805310270DF13C08CD
:105CE800099368464FF40023109412941494159461
:105CF80000940194029403970494069407940894DA
:105D08000A9405940B940C93CDF834800F95139551
:105D18000AF0ADF80523684611930F961094129473
:105D280014941594CDF8388013950AF0A0F82946F4
:105D380020460AF01CF940F6B830FEF755FF204619
:105D4800FFF7BEF904461649164E3846224609F0B2
:105D580023FB41F289239C4248F68918124F01D04F
:105D680044450ED1FEF7E0FF00233B70A6F8008003
:105D780010200E4948F6891241F2892309F00CFBDC
:105D880005E0FFF70BFE49F241333D70338018B050
:105D9800BDE8F08100040240000C024000100240FF
:105DA8002FAD05089A010020141A002046AD0508F9
:105DB8004FF0C04336221A8003F50033012814BF80
:105DC800682048201880704770B5244B01228CB099
:105DD8001A7000240AE0A9B21F2230460135FFF7E5
:105DE80053FA642DF7D10134642C02D00025A6B2F1
:105DF800F1E73220014602460346FFF7C9F94FF0A2
:105E0800C0432E221A8003F5003300201E881C8808
:105E18001D88A4B2B6B200F09BF8ADB22346104973
:105E28000095324603A811F095F800230A20C821EE
:105E380003AA00F0C7F904F0FC0204F4784444EA29
:105E4800C20242EAD522074903A811F083F80A20C2
:105E5800DC2103AA002300F0B5F9FEE7141A00209C
:105E680085AD05089DAD05082DE9F04F40F23F19B5
:105E7800484534BF04464C46EF2B34BF98464FF094
:105E8800EF084A4538BF9146EF2934BF0D46EF2544
:105E9800C4EB090AC5EB080785B0BAF1000FB8BF13
:105EA800CAF1000A002FB8BF7F424FF6FF734C4576
:105EB8002CBF1A4601221FFA8AFA454538BF01232A
:105EC800BFB202930FFA8AF63BB29E42BDF838B0D1
:105ED800019202DDC6F34F0607E0022693FBF6F6B1
:105EE8007642B6B201E01E4603E00FFA8AF35B423F
:105EF8000393144A1378022B204629465A4602D1A6
:105F0800FDF721FD01E0FFF7BFF94C4501D14545FB
:105F180014D0039A33B2934205DD019AF31BA418F7
:105F28009BB2A4B200E0334636B23AB29642DADA0D
:105F3800029A5344AD189BB2ADB2D4E705B0BDE8A0
:105F4800F08F00BF582C0020004870471C1A002012
:105F580082B0064BADF80600BDF8062092B21A8052
:105F6800188880B202B0FFF7D0B800BF181A002016
:105F7800014B188880B27047181A002082B0064B6F
:105F8800ADF80600BDF8062092B21A80188880B2D3
:105F980002B0FFF7C7B800BF1A1A0020014B1888D3
:105FA80080B270471A1A0020FFF7CCBAFFF76CBA14
:105FB80010B5BDF808400294BDE81040FFF7BAB923
:105FC80010B5BDF808400294BDE81040FFF734BA98
:105FD800FFF790B92DE9F04F4FEA420800253D4CF4
:105FE80085B082468B46C8F1030817462E461FFA2D
:105FF80087F909EB0B0C228805EB0A031FFA8CFCC6
:106008009BB26146184692B2CDF804C00293FFF7DE
:106018003BF9C9EB0B0292B20392029B22880399C7
:10602800184692B2FFF730F9DDF804C02288C5EBB4
:106038000A039BB26146184692B20293FFF724F90D
:10604800029B22880399184692B2FFF71DF905EBC7
:106058000B0292B2039209EB0A03228803999BB2BE
:10606800184692B20293FFF70FF9029B2288C5EBFC
:106078000B0C1FFA8CFC1846614692B2CDF804C08E
:10608800C9EB0A09FFF700F9228803991FFA89F971
:1060980092B24846FFF7F8F82288DDF804C092B2B9
:1060A80048466146FFF7F0F8B8F1000F04DA08EB4C
:1060B800860808F1060805E0F31B08F10A0808EB52
:1060C8008308013F01360135BE42ADB28FD905B014
:1060D800BDE8F08F181A002008B9FFF713B8012897
:1060E80001D1FFF70BB87047704700200146F02236
:1060F8004FF4A073FFF7C8B9704708B505280CD846
:10610800DFE800F0121403050709094808BD09482B
:1061180008BD094808BD094808BD0948094A0A4B8D
:1061280040F24111FEF724FD084808BD084808BDA3
:1061380088010020780100207001002068010020FB
:10614800A8AD0508AEA80408E3AB05089001002037
:106158008001002010B50446FFF7CFFF014B1860FF
:106168001C7110BDA0010020014B1879704700BFB9
:10617800A001002008B5FFF7C0FF808808BD08B55A
:10618800FFF7BBFFC08808BDF7B51F460B4B0C4E89
:106198001D681446EA882B68203C5443A4B2AE1B01
:1061A80003EB440418BF0126AB888DE8500017B1F3
:1061B800FFF7EEF901E0FFF771FAFEBDA00100203C
:1061C800900100202DE9F0410F46984615460446F7
:1061D800084E08E0204643463946FFF7D5FF3368A6
:1061E8009B88E418A4B215F8012B002AF2D1BDE867
:1061F800F08100BFA001002010B5044608462146E2
:10620800BDE81040DEE7094B70B5044618790E4624
:106218001546FFF7B4FFC6F1F001091A89B2204606
:106228002A460023BDE87040CCE700BFA00100204B
:10623800704700BF044B1A680AB9044A1A601A6802
:106248001018186010467047400D0020D43C0020FC
:106258004FF0FF30704708B50248034A034B372117
:10626800FEF786FCC7AD0508C4A80408E3AB05081B
:106278000120704710B504460A4802210AF0ACFE16
:106288000028F9D0074821460AF06FFE0548012189
:106298000AF0A2FE0028F9D00248BDE810400AF032
:1062A80061BE00BF0038004010B5194802210AF04D
:1062B80093FE0028F9D0164800210AF056FE14482B
:1062C80001210AF089FE0028F9D011480AF04AFE97
:1062D8000402A4B2002301E001339BB2002BFBD0DF
:1062E8000B4802210AF078FE0028F9D0084800215E
:1062F8000AF03BFE064801210AF06EFE0028F9D09C
:1063080003480AF02FFE2043C0F3CB0010BD00BFA6
:10631800003800402DE9F0478AB00AAF0A20012171
:106328000AF0D4FB4FF4604347F8143D474EDFF8BA
:1063380024A1012400254FF00208304639468DF883
:106348001A508DF818808DF819808DF81B400AF0C6
:1063580015F830460D2105220AF090F830460E2136
:1063680005220AF08BF8052230460F210AF086F83C
:1063780021464FF480400AF0CDFB50460AF0A8FCB5
:106388004FF48273ADF802304FF40073ADF80A3061
:106398003823ADF80C30504607236946ADF8103065
:1063A800ADF80050ADF80450ADF80650ADF80850FF
:1063B800ADF80E500AF0BEFC504621460AF055FDD5
:1063C800A9468DF81A5030464FF480553946059540
:1063D8008DF818408DF819808DF81B4009F0CEFF14
:1063E800304629460AF03BF84025394618488DF8CA
:1063F80018908DF819808DF81A908DF81B40059526
:1064080009F0BCFF21464FF480400AF08FFB0621BB
:1064180003200AF019FE0C2307A88DF821300795F0
:106428008DF820908DF8224009F09CFC17238DF8F8
:10643800243009A80F238DF825308DF826308DF8E3
:10644800274002F02DFF0AB0BDE8F08700040240A3
:10645800000C024000380040014B1878704700BF1C
:10646800440D0020024B5A889B8802800B8070479D
:10647800440D0020014B00221A707047440D002083
:10648800F0B593B068460021482210F0E3FC6D4651
:10649800002464484FF4805109F0E3FF002301E031
:1064A80001339BB2002BFBD09020FFF7E3FE0023C3
:1064B80001E001339BB2002BFBD0FFF7F5FE4FF450
:1064C80080510746574809F0CAFF002301E001330D
:1064D8009BB2002BFBD053484FF4805109F0C1FF09
:1064E800002301E001339BB2002BFBD0D020FFF743
:1064F800C1FE002301E001339BB2002BFBD0FFF764
:10650800D3FE4FF480510646464809F0A8FF45F8E7
:10651800047B01342E6244484021E4B209F08DFF27
:1065280010B9092CB5D101E0092C78D19DE80C00EF
:10653800D218029B03980699D218049BC018059B91
:10654800C018079BCB180899032490FBF4F092FB22
:10655800F4F25B1893FBF4F3151AC11A9C1A002D78
:10656800B8BF6D420029B8BF4942002CB8BF644289
:10657800502D03DD502909DD502C50DC8D4205DA01
:10658800AC424FF0020405DB111806E08C424FF0D4
:10659800020401DAD11800E0C1180A9B099A0C9884
:1065A8000F9DD2180B9BD2180D9BC0180E9BC018BC
:1065B800109BEB18119D91FBF4F1032492FBF4F26C
:1065C80090FBF4F05B1993FBF4F3161AC41A9D1AA6
:1065D800002EB8BF7642002CB8BF6442002DB8BF69
:1065E8006D42502E89B203DD502C09DD502D16DC8A
:1065F800A64205DAB5424FF0020405DB131806E09F
:10660800A5424FF0020401DAD31800E0C318074A84
:1066180093FBF4F39BB2938001235180137013B062
:10662800F0BD00BF00040240000C0240440D0020F1
:10663800FFF712BFF7B505460C4601A80DF1060194
:10664800FFF710FF1B4BBDF80660BDF8040093E888
:106658000600724301FB002299685218164992FB02
:10666800F1F207EE102AF8EEC77A40F23F17FCEE77
:10667800E77A17EE902A92B2B2F5207F28BF3A4601
:106688002A801D69DA685B696E4302FB0060C018E6
:1066980090FBF1F107EE101AF8EEC77AFCEEE77AF4
:1066A80017EE903A9BB2B3F5F07F28BFEF23238013
:1066B800FEBD00BF4C0D002040420F00FFF7DABEC0
:1066C800014B187E704700BF4C0D0020FFF7CABE73
:1066D800042808B505D90748074A084B7D21FEF765
:1066E80047FA054B03EB8000038B0B80438B138029
:1066F80008BD00BFE8AD0508CAA8040806AE05082D
:1067080008B5082001F0BAF942F69643C31A584270
:1067180040EB030008BD10B50A2001F0D7F90C4C76
:1067280020600E2001F0D2F96060122001F0CEF94D
:10673800A060162001F0CAF9E0601A2001F0C6F93D
:1067480020611E2001F0C2F901236061237610BD8B
:106758004C0D002010B5FFF7DDFD01F06DFA044681
:1067680001F076FA074903462246202008F014FE75
:10677800FFF7C6FF28B101F079FA10B9BDE810405B
:10678800C9E710BD42AE050810B5104C0A202168B3
:1067980001F083F961680E2001F07FF9A1681220E9
:1067A80001F07BF9E168162001F077F921691A20D8
:1067B80001F073F961691E2001F06FF9082042F6B3
:1067C8009641BDE8104001F04BB900BF4C0D0020C8
:1067D8002DE9F04F0346A7B0B0F800C01C898688A1
:1067E800DF885D89CDF810C0B249B0F802C0B3F8AF
:1067F8000C90B3F80E80CDF824C00FFA84FB30B2A9
:1068080001220FFA87FE0BEB000C0A7629B20FFA69
:1068180089FACDF888C001EB0E0C0FFA88F2CDF892
:1068280090C00AEB0B0CCDF830C002EB010CCDF890
:1068380058C0B3F810C05B8ACDF800C00FFA8CFCC2
:1068480006910CEB00010A9102930CEB0A011BB2B2
:10685800239103EB0E010E9199182591049900FAE2
:1068680081F0584450446044DDF824C006990EFA7B
:106878008CFEDDF810C01FFA80FB1CFB0CF08E4468
:1068880016FB0600964414FB0400009A19FB090045
:106898009E4412FB02001FFA8EFA0BF0A7FCDDF8EB
:1068A80024C0029ACDE912011CFB0CF017FB07006B
:1068B80015FB050018FB080012FB02000BF096FC04
:1068C800DDF824C0029ACDE9140104991CFB01F3F8
:1068D80017FB063615FB0466009B18FB096612FBBE
:1068E80003600BF083FCDDE91423CDE90001DDE949
:1068F80012010BF0F1FC04460D46DDE900010246E9
:106908000B460BF0E9FC02460B46204629460BF0E5
:106918002FFBCDE9180158460BF078FCCDE91001A2
:10692800DDE91023DDE900010BF0D6FCCDE9060115
:1069380050460BF06BFC804689464246DDE9120161
:106948004B460BF0C9FCDDE91023CDE91C01DDE95C
:1069580014010BF0C1FC002206460F46564BDDE938
:1069680018010BF0B9FC424604460D464B46DDE9DA
:1069780006010BF0B1FC02460B460BF0FBFA02468F
:106988000B46204629460BF0F5FA424604460D46CA
:106998004B46DDE91C010BF09FFC02460B462046E6
:1069A80029460BF0E5FADDE9102304460D4630468A
:1069B80039460BF091FC02460B46204629460BF05F
:1069C800D7FADDF828C0CDE902014FEA8C10DDF8CE
:1069D80030C000EB0C20DDF810C0A0241CFB040024
:1069E8000BF004FCDDF838C0CDE90A014FEA8C1041
:1069F800DDF858C000EB0C20DDF824C01CFB0400B7
:106A08000BF0F4FBCDE90C0150460BF0EFFBDDE990
:106A18001023CDE91601DDE90C010BF05DFC4246BF
:106A2800CDE91E014B46DDE90A010BF055FC424653
:106A3800CDE920014B46DDE900010BF04DFC324663
:106A48003B460BF095FACDE90E0158460BF0CEFB0C
:106A5800DDE91C23CDE91A01DDE906010BF088FA0E
:106A6800DDF88CC0C024CDE9060104FB0CF0DDF88C
:106A780088C0302505FB0C00DDF810C078261CFB0B
:106A880006000BF0B3FBDDF894C0824604FB0CF063
:106A9800DDF890C005FB0C00DDF824C01CFB0600E7
:106AA8008B460BF0A3FBDDE9102306460F460BF0DF
:106AB80013FC03E04C0D0020000014404246CDE9D1
:106AC80004014B46504659460BF006FCDDE91423F9
:106AD80080468946DDE90A010BF0FEFBDDE900236B
:106AE80004460D46DDE90C010BF0F6FB02460B46A9
:106AF800204629460BF03CFA0022A14B0BF0ECFB98
:106B0800DDE9202304460D46DDE91E010BF030FACD
:106B180002460B46DDE916010BF0DEFB02460B468A
:106B2800204629460BF026FA002204460D46954BCE
:106B3800DDE90E010BF0D0FB02460B462046294644
:106B48000BF018FADDE902230BF0F0FC88A3D3E977
:106B580000230BF0C1FB0BF059FE8B490860DDE9FF
:106B68001223DDE90C010BF0B7FBDDE90023044635
:106B78000D46DDE90A010BF0AFFB02460B46204645
:106B880029460BF0F5F900227D4B0BF0A5FBDDE95A
:106B98001E2304460D46DDE920010BF0E9F9024603
:106BA8000B46DDE91A010BF097FB02460B4620461F
:106BB80029460BF0DFF9002204460D46714BDDE94A
:106BC80006010BF089FB02460B46204629460BF0CE
:106BD800D1F9DDE902230BF0A9FC65A3D3E9002371
:106BE8000BF07AFB0BF012FE674A5060DDE90E23CA
:106BF800DDE90A010BF070FBDDE9062304460D46CA
:106C0800DDE90C010BF068FB02460B4620462946DD
:106C18000BF0B0F9002204460D465A4BDDE9180185
:106C28000BF05AFB02460B46204629460BF0A2F908
:106C3800DDE902230BF07AFC4DA3D3E900230BF026
:106C48004BFB0BF0E3FD504B59469860DDE91423EC
:106C580050460BF041FBDDE9002304460D46304663
:106C680039460BF039FB02460B46204629460BF005
:106C78007FF90022424B0BF02FFB424604460D469B
:106C88004B46DDE904010BF073F902460B46DDE9DA
:106C980016010BF021FB02460B46204629460BF055
:106CA80069F935A3D3E9002304460D46DDE90E0151
:106CB8000BF012FB02460B46204629460BF05AF908
:106CC800DDE902230BF032FC29A3D3E900230BF002
:106CD80003FB0BF09BFDDFF8B0C0DDE91223CCF815
:106CE8000C00394630460BF0F7FADDE9002304467C
:106CF8000D46504659460BF0EFFA02460B46204621
:106D080029460BF035F900221D4B0BF0E5FADDE9B9
:106D1800042304460D46404649460BF029F902462D
:106D28000B46DDE91A010BF0D7FA02460B4620465E
:106D380029460BF01FF910A3D3E9002304460D469A
:106D4800DDE906010BF0C8FA02460B462046294643
:106D58000BF010F9DDE902230BF0E8FB04A3D3E9FB
:106D680000230BF0B9FA0BF051FD074908610DE05B
:106D78000000000080842E410000000000C0824016
:106D880000001440000089404C0D0020DDE90E236E
:106D9800504659460BF0A0FADDE9062304460D4695
:106DA800304639460BF098FA02460B4620462946EB
:106DB8000BF0E0F811A3D3E9002304460D46DDE902
:106DC80018010BF089FA02460B46204629460BF0BB
:106DD800D1F8DDE902230BF0A9FB0AA3D3E90023CC
:106DE8000BF07AFA0BF012FD034A506127B0BDE8A8
:106DF800F04FC9E4AFF300804C0D00200000000004
:106E080000C082400000000080842E41AFF3008063
:106E1800064A074B1A60074A074B1A60074B42F2AB
:106E280010721A60064B64221A60704740420F00C5
:106E38004C26002080C3C901642C0020402C00206F
:106E4800F8250020012808B503D05AD3022851D1CB
:106E58003CE02C4B1B78012B03D013D3022B49D1D8
:106E680021E0294BC820196800F017FE274BCC20D9
:106E7800196800F012FE264BD020196800F00DFEAC
:106E8800D42033E0204BD820196800F006FE1F4BB1
:106E9800DC20196800F001FE1D4BE020196800F0A5
:106EA800FCFDE42022E0184BF820196800F0F5FDFD
:106EB800164BFC20196800F0F0FD154B4FF480705C
:106EC800196800F0EAFD4FF482700FE00E4BE820DD
:106ED800196800F0E2FD0D4BEC20196800F0DDFDAB
:106EE8000B4BF020196800F0D8FDF420094B196805
:106EF80000F0D3FD04F0C0FE18B9BDE8084004F066
:106F0800CCBE08BD1C0E00204C260020642C00209E
:106F1800402C0020F825002008B52E4B1B78012BAB
:106F280002D0022B55D140E02B4B1B78012B03D00C
:106F380013D3022B4DD121E0C82000F0C7FD274B09
:106F48001860CC2000F0C2FD254B1860D02000F05E
:106F5800BDFD244B1860D42022E0D82000F0B6FDF7
:106F68001E4B1860DC2000F0B1FD1D4B1860E020BE
:106F780000F0ACFD1B4B1860E42011E0F82000F095
:106F8800A5FD164B1860FC2000F0A0FD144B1860FE
:106F98004FF4807000F09AFD124B18604FF4827025
:106FA80000F094FD104B186008BDE82000F08EFD3D
:106FB8000A4B1860EC2000F089FD094B1860F0209E
:106FC80000F084FD074B1860F42000F07FFD064BAD
:106FD800186008BDC90100201C0E00204C260020A6
:106FE800642C0020402C0020F825002008B504F06F
:106FF80043FE10B1BDE808408EE7BDE8084007E74A
:10700800064B07495960C021002219721E211A70C7
:10701800D9601A745A611A76DA617047481A0020E2
:1070280040787D0110B50321FF22C02001F020FC2B
:107038001F4C102180222060C02001F019FC112172
:1070480080222060C02001F013FC122180222060E1
:10705800C02001F00DFC132180222060C02001F027
:1070680007FC142180222060C02001F001FC1521BA
:1070780080222060C02001F0FBFB802220601621C6
:10708800C02001F0F5FB2060C0201721802201F00C
:10709800EFFB80222060B721C02001F0E9FB054BFF
:1070A80000221A745A611A76DA6101221A7010BD28
:1070B80020260020481A002038B5C0200321FF22CE
:1070C80001F0D6FB0B4D00242B19615D5A78C020C6
:1070D800023401F0CDFBC82CF6D1B121AC22C0207E
:1070E80001F0C6FBC0200321002201F0C1FB0020F3
:1070F80038BD00BFF6A804082DE9F34706460F4639
:1071080092461D461AB90C1FE401914635E005EE7A
:10711800902A06EE903AB8EE657AF8EE667AFC01A7
:10712800C7EE277AA4F500749FED5C7A67EE877A3C
:1071380017EE900A0BF07CF841EC100B0DF0A8F953
:1071480059EC108B494640460BF088FB24184FEA4F
:10715800CA100BF04BF8CDE9000128460BF046F8B1
:107168004B4642460BF0B8F802460B46DDE90001F3
:107178000AF0FEFE0BF072FB8146002E14BF4FF0A2
:1071880022084FF01A08C5F307224146C02001F033
:107198006FFB08F10101EAB2C02001F069FBC4F3FA
:1071A800014208F10201C02001F062FBC4F307228A
:1071B80008F10301C02001F05BFBE2B208F1040111
:1071C800C02001F055FBC9F3034305F4702243EADC
:1071D800123208F10501C02001F04AFB08F106014E
:1071E800C9F30722C02001F043FB08F107015FFA49
:1071F80089F2C02001F03CFBC020B121A02201F09F
:1072080037FB07EE107A264CF8EEC77A0EBBD4EDA2
:10721800015A06EE90AAB8EE657A05EE905AB8EED5
:10722800666AF8EE656A0123C6EE266A237477EE6D
:10723800A67A67EE277A17EE900A0AF0F9FF41EC72
:10724800100B0DF025F951EC100B0BF007FB6061EA
:1072580020E005EE90AAD4ED016AB8EE656A05EE65
:10726800905AB8EE667AF8EE656A0123C6EE266A89
:10727800237677EEA67A67EE277A17EE900A0AF059
:10728800D7FF41EC100B0DF003F951EC100B0BF08C
:10729800E5FAE0610020BDE8FC8700BF000000437C
:1072A800481A00200022012326E7012838B50D4698
:1072B80004D002280CBF3C242C2400E034242146AE
:1072C800C02001F04FFB05F0070200F00F0040EA74
:1072D80002122146C020BDE8384001F0C9BA2DE9A4
:1072E800F3470A9C1D4607468A461646524B01E05C
:1072F8006D0864089C42FBD82DB906F10076043E5F
:10730800F601A94634E006EE905AB8EE667A06EE23
:10731800904AF8EE667AF601C7EE277AA6F5007667
:107328009FED467A67EE877A17EE900A0AF080FF9B
:1073380041EC100B0DF0ACF859EC108B4946404667
:107348000BF08CFA3618E8010AF050FFCDE900017D
:1073580020460AF04BFF4B4642460AF0BDFF024664
:107368000B46DDE900010AF003FE0BF077FA8146CF
:10737800022F9BBF324BDB194FF0000893F8C880EF
:10738800C4F307224146C02001F072FA08F1010156
:10739800E2B2C9B2C02001F06BFA08F10201C9B229
:1073A800C6F30142C02001F063FA08F10301C9B233
:1073B800C6F30722C02001F05BFA08F10401C9B244
:1073C800F2B2C02001F054FA04F47024C9F3034364
:1073D80008F1050143EA1432C9B2C02001F048FAA5
:1073E80008F10601C9B2C9F30722C02008F107084D
:1073F80001F03EFA5FFA89F25FFA88F1C02001F0E5
:1074080037FABAF1010F0CBF2F220F220DB942F043
:107418004002012F06D002D3022F0AD105E0C02076
:10742800102104E0C020112101E0C020122101F048
:107438001FFA0020BDE8FC87FFFF0F000000004393
:10744800F6A8040807B5012300930023FFF747FFB8
:107458000EBD00280CBFFF22002208B5C020032162
:1074680001F006FA002008BD08B5C020B121AC2201
:1074780001F0FEF9002008BD08B50420012109F03B
:1074880025FB4FF480700121BDE8084009F04EBB90
:1074980007B50223009303238DF804300348002323
:1074A80069468DF8073008F069FF0EBD00080240F4
:1074B80030B5124D8BB0002406A8069407940894A2
:1074C800099408F029F900948DF804408DF80540D6
:1074D8000294039404942846012469468DF81440C4
:1074E80008F0EBF828460B212246062308F060F93D
:1074F8002846214608F02AF90BB030BD002001408B
:1075080010B5002104460122302001F0B1F9C0B9BC
:10751800012001F0A7FC002CB8BF4034E4B21021D0
:107528002246302001F0A4F9012001F09BFC302014
:107538001121224601F09CF90120BDE8104001F01C
:1075480091BC10BD10B5002104460122302001F085
:107558008FF9C0B9012001F085FC002CB8BF403478
:10756800E4B212212246302001F082F9012001F014
:1075780079FC30201321224601F07AF90120BDE878
:10758800104001F06FBC10BD38B5012205460C460D
:107598003020002101F06CF9F0B9012001F062FC03
:1075A80025EAE5725F2AA8BF5F223B21D2B23020CC
:1075B80001F05EF9012001F055FC24EAE4725F2A2B
:1075C800A8BF5F22D2B230203C2101F051F901203E
:1075D800BDE8384001F046BC38BD302810B5044637
:1075E8000ADC10F17F0F02DB002802DB05E06FF0F8
:1075F8007E0404F5807400E03024002130200A461F
:1076080001F036F9A8B90120E4B201F02BFC4121C0
:107618002246302001F02CF9012001F023FC302013
:107628004221224601F024F90120BDE8104001F072
:1076380019BC10BD282810B5044609DC10F1180F34
:1076480002DB002802DB04E06FF017047F3400E05F
:107658002824002130200A4601F00AF9A8B901209F
:10766800E4B201F0FFFB53212246302001F000F97B
:10767800012001F0F7FB30205421224601F0F8F8F0
:107688000120BDE8104001F0EDBB10BD08B5302069
:107698000021012201F0ECF860B9012001F0E2FBC1
:1076A80030203321402201F0E3F80120BDE80840F2
:1076B80001F0D8BB08BD10B530200021012201F02F
:1076C800D7F8044660B9012001F0CCFB3020332103
:1076D800224601F0CDF80120BDE8104001F0C2BB00
:1076E80010BD10B530200021012201F0C1F8044678
:1076F800A0B9012001F0B6FB34212246302001F068
:10770800B7F8012001F0AEFB30203721224601F006
:10771800AFF80120BDE8104001F0A4BB10BD402027
:10772800EEE640200EE708B500210122302001F0E6
:107738009FF8012001F096FB30203421024601F029
:1077480097F8012001F08EFB30203721024601F026
:107758008FF80120BDE8084001F084BB08B500217E
:107768000122302001F084F8012001F07BFB302059
:1077780034210C2201F07CF80120BDE8084001F01A
:1077880071BB0000000000002DE9F04F984B994AAA
:107798001968994B002914BF91469946974B2DEDCE
:1077A800048BC3F80090964B0025002287B01A80FE
:1077B800AA46AB46A8465AE0A2004046CDF804C007
:1077C80002920AF035FD0746584601F100460AF0D4
:1077D8002FFD02460B46384631460AF0C9FB39F9F7
:1077E800243007EE103AF8EEC77A064617EE900AEC
:1077F8000F460AF01DFD02460B46304639460AF090
:10780800B9FB0BF04BF8074650460AF011FD044649
:10781800284601F100460AF00BFDCDE90401DDE937
:107828000423204631460AF0A3FB029A09EB02031F
:107838000446B3F9023007EE103AF8EEC77A0D465F
:1078480017EE900A0AF0F4FC02460B462046294639
:107858000AF090FB0BF022F8DDF804C0684A0CF13E
:10786800010CC3465546A2F800C08246B846644B90
:10787800B3F800C00FFA8CF4B32C9DDD58460AF01B
:10788800D7FCCDE9020140460AF0D2FC00220646A8
:107898000F465C4BDDE902010AF01EFD02460B466D
:1078A800304639460AF066FB0022574B0AF03EFE86
:1078B8000AF0F4FF4CA3D3E9002309EE900ADDE9AE
:1078C80002010AF009FD00224F4B0AF02FFE0AF0D0
:1078D800E5FF09EE100A28460AF0AAFC04465046BD
:1078E8000D460AF0A5FC002206460F46204629460A
:1078F800444B0AF0F1FC02460B46304639460AF082
:1079080039FB0022404B0AF011FE0AF0C7FF36A3EC
:10791800D3E9002308EE900A294620460AF0DCFC49
:107928000022394B0AF002FE0AF0B8FF08EE100AEE
:1079380069EE287A58EE297A17EE900A0AF078FC50
:1079480068EE097A48EEA97A044617EE900A0D46C1
:107958000AF06EFC45EC104B41EC110B0CF09CFE50
:1079680051EC100B0AF09AFF28EE088A08EEA88A54
:1079780007EE100A254B264CF1EE477AC3ED007A44
:1079880018EE100A0AF054FC41EC100B0CF092FFB0
:1079980029EE099A51EC100B09EEA99A0AF07EFF1C
:1079A800206019EE100A0AF043FC41EC100B0CF0B1
:1079B80081FF51EC100B0AF071FFD4ED007A07EE4D
:1079C800100A87EE877A134B1860134BFDEEE77A9F
:1079D80083ED007A114BC3ED007A07B0BDEC048B40
:1079E800BDE8F08FAFF30080912B50E67AB6EB3FFD
:1079F800701A0020F2220020521D00206C1A00206C
:107A0800781A00200000E03F00005940682C002050
:107A1800802C0020742C0020702C0020741A002068
:107A280010B5084C204608F0F6F8074B1860FFF729
:107A3800ABFE064B0649012220461A80BDE81040DD
:107A480008F06AB910600240701A0020680D002022
:107A580020800010014B1868704700BF741A00207E
:107A680038B505460C460135C1F3072101F008FA7F
:107A7800A8B2E1B201F004FA00B238BD38B5044644
:107A880001F038F801340546A0B201F033F8EDB240
:107A9800C0B240EA052000B238BD37B50B0E8DF8EC
:107AA80004300B0C8DF805300B0A8DF806308DF874
:107AB8000710002400E0284601AB451CE15C0134B6
:107AC80001F0DEF9042CADB2F5D13EBD37B5002486
:107AD80000E02846451C01F00DF801ABADB2E054BA
:107AE8000134042CF5D19DF805009DF804300004FC
:107AF80040EA03609DF8073018439DF8063040EAD5
:107B080003203EBD37B500230193002400E028463A
:107B1800451C00F0EFFF01ABADB2E0540134042C7A
:107B2800F5D19DED010A3EBD7047000038B5044609
:107B3800642001F097F925786068AD00EDB22570F2
:107B480008F081FC237A40FA03F000F003000543B3
:107B5800104B257005F00F055A5D6378D218D2B224
:107B6800D3B20132D2B2022A637001D80022A270C5
:107B78005BB2012B03DD0123A3700023637094F92A
:107B88000130013303DAFF23A3700023637094F9F3
:107B9800020038BDC2A90408F7B504200121234F0B
:107BA80008F094FF02AD01214FF48040012408F051
:107BB800BDFF00264FF4B0733846694645F8083DC6
:107BC8008DF804608DF8074008F0D8FB1020214696
:107BD80008F07CFF78236946154800938DF8046007
:107BE8008DF8074008F0CAFB0420214608F06EFF14
:107BF80021464FF4804008F099FF1C233846694617
:107C080000938DF804608DF8074008F0B7FB022058
:107C1800214608F05BFFB02306488DF804606946EA
:107C28008DF80740009308F0A9FBFEBD000802404C
:107C38000010024000040240802108B5034808F003
:107C4800FCFBD0F1010038BF002008BD0004024051
:107C580008B54FF48071044808F0EFFBD0F101003B
:107C680038BF002008BD00BF0008024008B5FFF774
:107C7800E3FF08B1FFF7ECFFC0B208BD70B50028FC
:107C88003AD01E4B1A7880181D4AC0B292F90020CB
:107C9800187040B282421B4A02DD1178013919700E
:107CA80093F9001092F9002091FBF2F402FB1414EE
:107CB8001549E4B21C700A88144B1A80144B154AF3
:107CC80018881080144A92F9000064B2013094FBBD
:107CD800F0F200FB1240114C2688114C258800FB5D
:107CE800065008800F4908880F49098802FB0012CE
:107CF8001A800E4B01221A7070BD00BF0E3A002088
:107D08003936002015360020443A00205A36002023
:107D18000C3A00200C380020463A00206837002032
:107D2800A83A0020D43A0020EA3700201436002070
:107D3800F0B5264A264C00231370264A2568167883
:107D4800254A12680FE0D45C2F197F7817F0040FCA
:107D580007D0302C02D12023135431E01B4A137072
:107D680003E00133DBB29E42EDDA184B1B78834205
:107D7800194B16D9A9B11A68164C31211154302162
:107D88000BE01A681518125C2E2A19D0303AD2B2B4
:107D9800092A88BF29700130C0B222788242F0DAFD
:107DA8000EE01B681A5C79B12E2A0DD05118C9B2A1
:107DB800392903D82F2998BF302100E039211954D7
:107DC800BDE8F040FCF7ACBCF0BD00BF6C0D002076
:107DD80048030020C83B0020303A002010B564203A
:107DE80001F040F88248FFF7A1FE824B1B78044659
:107DF8000C2B00F25F81DFE813F00D000D005D0130
:107E08007500750037008C008C00B700BA00D400EC
:107E18008C003901FFF71CFF18B10120F9F786FD26
:107E280048E1754B1888754B1B88C01A744B1B8822
:107E380090FBF3F0734B1A88734B1B88D31A734A61
:107E4800128893FBF2F3DBB2C0B2032B00F2CC80B2
:107E5800DFE803F0020406086D4A40E06D4A3EE0A0
:107E68006D4A3CE06D4A3AE0FFF7F2FED8B10021D6
:107E78000A226B4810F0BEF96A4B002118600A22EA
:107E8800694810F0B7F9694B18600420FEF762F9E9
:107E980096200521664A0023FEF794F90020FEF794
:107EA80059F906F0EBFF544B1888544B1B88C01A3D
:107EB800534B1B8890FBF3F0524B1A88524B1B888C
:107EC800D31A524A128893FBF2F3DBB2C0B21BB149
:107ED800012B40F0898001E0514A00E0524A554B9D
:107EE8001A6081E0002800F0E580534B1A7806DD1F
:107EF8000132D2B2102A1A7008D9112205E0013ACB
:107F0800D2B2112A1A7001D900221A70F9F7EEFEBE
:107F1800D0E0002800F0CE80484B1A788418E4B2EC
:107F28000322B4FBF2F102FB1144E4B21C70444B8F
:107F3800444A1B5D022B137009D0052B0CD0012B72
:107F480040F0B8804FF4917069213F4A08E04FF43F
:107F5800917069213D4A03E03D4A4FF491706921CF
:107F68000023FEF72FF9A5E03A4B1870A2E0FFF7BF
:107F78006FFEA0B10021384810F088F8374B042074
:107F880083ED000AFEF7E6F8B4200521344A002301
:107F9800FEF718F9FAF7B6FA0020FEF7DBF82E4AD2
:107FA80016E0FFF755FE90B100212E4810F06EF84C
:107FB8002D4B042083ED000AFEF7CCF8962005210E
:107FC800274A0023FEF7FEF80020FEF7C3F8254AEB
:107FD800184B1A60084B1888084B1B88C01A084BA6
:107FE8001B8890FBF3F0C0B22146FFF7A1FE61E0C9
:107FF800A8010020CD250020443A0020A83A0020FE
:10800800683700200C3A0020EA370020D43A0020D4
:1080180010260020342600204A2C0020FC250020B1
:10802800B03A0020C4010020203A0020C0010020FE
:108038007DAE0508303A002046260020D50D0020E8
:10804800300300201C0300208DAE050890AE050803
:1080580093AE05083C3A00202C360020240300206B
:1080680096AE05085036002020030020FFF7F0FDEB
:1080780008B107F0DBF814B1254B01221A70254B23
:108088001A68A41814F5967FB8BF234A1C60B8BFB5
:108098001A601B68B3F5967F03DD1E4B4FF496728A
:1080A8001A601B4C23782BB11C4B186801F0DAFAC4
:1080B800002323701A48FFF739FD1A4B1B78013B40
:1080C8000A2B24D8DFE803F00623232320151523E1
:1080D80011111500FFF7D2FDFFF7AEFD002816D0ED
:1080E8000220BDE81040F9F721BC0F4B1B78022B8A
:1080F8000AD100280D4B01D1187010BD01DD0122F5
:1081080000E0FF221A7010BDBDE81040B6E510BDB2
:1081180048260020403A0020D4FEFFFFEC2500202E
:10812800B4010020CD25002034380020811A002019
:1081380010B58CB01E490F2268460EF049FE1D4945
:108148000F2204A80EF044FE1B490F2208A80EF0C7
:108158003FFE00210822302000F08AFB012000F0B9
:1081680081FE002404AB1DF80420E15C302000F0FF
:108178007FFB0134012000F075FE0F2CF2D10021A5
:108188000922302000F074FB012000F06BFE00246F
:1081980008AB1DF80420E15C302000F069FB0134D5
:1081A800012000F05FFE0F2CF2D10CB010BD00BF13
:1081B800D4A90408E3A90408F2A9040810B58CB0EE
:1081C8001E490F2268460EF003FE1D490F2204A81F
:1081D8000EF0FEFD1B490F2208A80EF0F9FD002144
:1081E8000822302000F044FB012000F03BFE002470
:1081F80004AB1DF80420E15C302000F039FB0134A9
:10820800012000F02FFE0F2CF2D10021092230208E
:1082180000F02EFB012000F025FE002408AB1DF81D
:108228000420E15C302000F023FB0134012000F041
:1082380019FE0F2CF2D10CB010BD00BF01AA040822
:1082480010AA04081FAA040810B58CB01E490F22F2
:1082580068460EF0BDFD1D490F2204A80EF0B8FDBA
:108268001B490F2208A80EF0B3FD00210822302078
:1082780000F0FEFA012000F0F5FD002404AB1DF823
:108288000420E15C302000F0F3FA0134012000F012
:10829800E9FD0F2CF2D100210922302000F0E8FA84
:1082A800012000F0DFFD002408AB1DF80420E15C8C
:1082B800302000F0DDFA0134012000F0D3FD0F2C4E
:1082C800F2D10CB010BD00BF2EAA04083DAA0408C4
:1082D8004CAA040807B50220012108F0F7FB012386
:1082E80000938DF8043002238DF8053004480023EC
:1082F80069468DF806308DF8073008F03FF80EBD56
:108308000004024010B5084C01210022204608F064
:10831800AAF840F2FF4000F0A5FD012120460A46D8
:10832800BDE8104008F09FB80004024008B5FFF708
:10833800E9FF00210A46302000F09AFA012000F0F7
:1083480091FD01210A46302000F092FA012000F048
:1083580089FD00210122302000F08AFA012000F076
:1083680081FD01210822302000F082FA012000F06E
:1083780079FD02210122302000F07AFA012000F074
:1083880071FD00210A46302000F072FA012000F049
:1083980069FD1B21CD22302000F06AFA012000F08F
:1083A80061FD04210322302000F062FA012000F070
:1083B80059FD06210922302000F05AFA012000F068
:1083C80051FD07210822302000F052FA012000F068
:1083D80049FD08217022302000F04AFA012000F0FF
:1083E80041FD1E213020B02200F042FA012000F0A9
:1083F80039FD05219122302000F03AFA012000F0E1
:1084080031FD0D210322302000F032FA012000F066
:1084180029FD0E210022302000F02AFA012000F068
:1084280021FD14218022302000F022FA012000F0E2
:1084380019FD0B218822302000F01AFA012000F0E3
:1084480011FD0C218222302000F012FA012000F0E8
:1084580009FD12218822302000F00AFA012000F0DC
:1084680001FD13218C22302000F002FA012000F0D7
:10847800F9FC00210A46302000F0FAF9012000F04A
:10848800F1FC3D210222302000F0F2F9012000F039
:10849800E9FCFFF74DFEFFF791FEFFF7D5FE302010
:1084A8000021012200F0E4F9012000F0DBFC3D216D
:1084B8006422302000F0DCF9012000F0D3FC032115
:1084C8000022302000F0D4F9012000F0CBFC042178
:1084D8000022302000F0CCF9012000F0C3FC00217C
:1084E8000122302000F0C4F9012000F0BBFC0C216F
:1084F8000822302000F0BCF9012000F0B3FC0D2167
:108508000822302000F0B4F9012000F0ABFC0E2165
:108518000822302000F0ACF9012000F0A3FC0F2164
:108528000822302000F0A4F9012000F09BFC002173
:108538000A46302000F09CF9012000F093FC02224A
:108548004021302000F094F9012000F08BFC30200D
:108558004121002200F08CF9012000F083FC3F212A
:10856800D422302000F084F9012000F07BFC0021A7
:108578000122302000F07CF9012000F073FC10216A
:108588000F22302000F074F9012000F06BFC11215B
:108598000F22302000F06CF9012000F063FC12215A
:1085A8000022302000F064F9012000F05BFC132168
:1085B8000022302000F05CF9012000F053FC092172
:1085C8003C22302000F054F9012000F04BFC00213F
:1085D8000122302000F04CF9012000F043FC30204B
:1085E8003421024600F044F9012000F03BFC302021
:1085F8003721024600F03CF9012000F033FC362117
:108608000322302000F034F9012000F02BFC39213E
:108618000322302000F02CF9012000F023FC3B213C
:108628003C22302000F024F9012000F01BFC3C2102
:108638000A46302000F01CF9012000F013FC00214C
:108648000A46302000F014F9012000F00BFC5121FB
:10865800C022302000F00CF9012000F003FC522168
:108668003020002200F004F90120BDE8084000F0A5
:10867800F9BB00BF2DE9F04F454E464D93B001219F
:108688004FF4001008F022FA304607F0C5F94FF011
:10869800C0630293404B0393404B002404934FF470
:1086A800B4794FF400334FF480684FF400674FF407
:1086B800005A4FF4807B304602A90C930193099726
:1086C800CDF8189005940794CDF82080CDF828A00F
:1086D800CDF82CB00D9407F02BFA224630463049DD
:1086E80007F081FA3046012107F087FA01210A468E
:1086F8004FF0402008F058FC284607F08DF9294A29
:10870800019B0392284A0C9304922846402202A90E
:10871800059209970294CDF818900794CDF8208017
:10872800CDF828A0CDF82CB00D9407F001FA224618
:1087380028461E4907F057FA2846012107F05DFA36
:1087480042F2107701220221194808F02DFC384620
:1087580000F088FB3046012107F025FA0121284660
:1087680007F021FA384600F07DFB0B238DF84430E2
:1087780011A801238DF845408DF846408DF8473003
:1087880000F08EFD384600F06DFB13B0BDE8F08FA9
:1087980010600240886002400C400040F222002035
:1087A800521D00200C3C004022200020821A00208C
:1087B800003C004002481021012207F06BBA00BFBC
:1087C8001060024013B50220012108F07FF94FF430
:1087D80010730E4C009302238DF804308DF8053089
:1087E80001238DF806302046002369468DF80730AE
:1087F80007F0C4FD20460621042207F03FFE20466C
:108808000921042207F03AFE1CBD00BF0004024003
:1088180030B5154D85B001214FF4001008F07AF9F4
:10882800284607F041FE0023ADF804304BF6FF73ED
:10883800ADF806303323ADF808304FF48063ADF857
:108848000A304FF48043ADF80C3004AC074B28468F
:10885800012144F8103D07F0C9FE2846694607F093
:1088680051FE05B030BD00BF00540040801A06001C
:1088780073B54FF4961306460D461446019304E06B
:10888800019B5A1E0192002B57D031484FF40031FA
:1088980007F0C4FF0028F3D12D48012107F0B2FEEC
:1088A8004FF48053019304E0019B5A1E0192002B60
:1088B80045D02748274907F09CFF0028F4D02448D2
:1088C8003146002207F0B6FE4FF48053019304E0CE
:1088D800019B5A1E0192002B33D01D481E4907F0F8
:1088E80088FF0028F4D01A48294607F026FF4FF4DD
:1088F8008053019303E0019B5A1E01921BB3144855
:10890800164907F076FF0028F5D01148214607F0F0
:1089180014FF4FF49613019303E0019B5A1E019232
:108928009BB10B480E4907F079FF0028F5D008489D
:10893800012107F073FE002008E0012006E0022074
:1089480004E0032002E0042000E005207CBD00BF15
:108958000054004001000300820007008000070067
:108968000400001037B54FF4961304460D460193E2
:1089780005E0019B5A1E0192002B00F09B8056488F
:108988004FF4003107F04AFF0028F2D15248012184
:1089980007F038FE4FF48053019305E0019B5A1EFF
:1089A8000192002B00F088804B484C4907F021FFCA
:1089B8000028F3D048482146002207F03BFE4FF438
:1089C8008053019304E0019B5A1E0192002B75D03D
:1089D8004148434907F00DFF0028F4D03E48294696
:1089E80007F0ABFE4FF48053019304E0019B5A1E3D
:1089F8000192002B64D038483A4907F00FFF00284D
:108A0800F4D03548012107F0FDFD4FF48053019360
:108A180004E0019B5A1E0192002B53D02E482F4987
:108A280007F0E7FE0028F4D02B482146012207F082
:108A380001FE4FF48053019304E0019B5A1E0192FA
:108A4800002B41D0244C2849204607F0E7FE002897
:108A5800F3D02046002107F0F5FD20460121238BA5
:108A680007F0DCFD4FF48053019304E0019B5A1E8C
:108A78000192002B2AD018481C4907F0CFFE002885
:108A8800F4D0154807F05BFE4FF480530193124A67
:108A980003E0019B591E0191D3B113889B05F8D4BB
:108AA800012104460C4807F0CDFD0B48104907F09A
:108AB800CFFE0EE001240CE002240AE0032408E0C3
:108AC800042406E0052404E0062402E0072400E06C
:108AD800082420463EBD00BF0054004001000300AA
:108AE800820007000400001002000010400000107F
:108AF8000004001013B54FF496130446019305E0E3
:108B0800019B5A1E0192002B00F0AF8060484FF481
:108B1800003107F083FE0028F2D15D48012107F0FB
:108B280071FD4FF48053019305E0019B5A1E019299
:108B3800002B00F09C805648564907F05AFE002842
:108B4800F3D05348A021002207F074FD4FF480535E
:108B5800019305E0019B5A1E0192002B00F08980C9
:108B68004B484D4907F045FE0028F3D0210A4848F4
:108B780007F0E3FD4FF48053019304E0019B5A1E74
:108B88000192002B77D04248444907F047FE00285D
:108B9800F4D0E1B23E4807F0D0FD4FF48053019382
:108BA80004E0019B5A1E0192002B66D038483B49CD
:108BB80007F034FE0028F4D03548012107F022FDE3
:108BC8004FF48053019304E0019B5A1E0192002B3D
:108BD80055D02F482F4907F00CFE0028F4D02C4818
:108BE800A121012207F026FD4FF48053019304E0F0
:108BF800019B5A1E0192002B43D0254C2849204640
:108C080007F00CFE0028F3D02046002107F01AFDDB
:108C180020460121238B07F001FD4FF48053019377
:108C280004E0019B5A1E0192002B2CD018481D49C4
:108C380007F0F4FD0028F4D0154807F080FD4FF444
:108C480080530193124A03E0019B591E0191E3B13D
:108C580013889905F8D4012104460D4807F0F2FC61
:108C68000B48114907F0F4FD10E001240EE002243E
:108C78000CE003240AE0042408E0052406E00624A6
:108C880004E0072402E0082400E0092420461CBD73
:108C98000054004001000300820007000400001097
:108CA80002000010400000100004001013B54FF43B
:108CB80096130446019305E0019B5A1E0192002B6E
:108CC80000F0AF8060484FF4003107F0A7FD00289E
:108CD800F2D15D48012107F095FC4FF480530193D0
:108CE80005E0019B5A1E0192002B00F09C8056481B
:108CF800564907F07EFD0028F3D05348A0210022F2
:108D080007F098FC4FF48053019305E0019B5A1E2D
:108D18000192002B00F089804B484D4907F069FD0E
:108D28000028F3D0210A484807F007FD4FF4805384
:108D3800019304E0019B5A1E0192002B77D0424810
:108D4800444907F06BFD0028F4D0E1B23E4807F033
:108D5800F4FC4FF48053019304E0019B5A1E0192E6
:108D6800002B66D038483B4907F058FD0028F4D05E
:108D78003548012107F046FC4FF48053019304E085
:108D8800019B5A1E0192002B55D02F482F4907F0FE
:108D980030FD0028F4D02C48A121012207F04AFC1C
:108DA8004FF48053019304E0019B5A1E0192002B5B
:108DB80043D0254C2849204607F030FD0028F3D041
:108DC8002046002107F03EFC20460121238B07F0B6
:108DD80025FC4FF48053019304E0019B5A1E019235
:108DE800002B2CD018481D4907F018FD0028F4D096
:108DF800154807F0A4FC4FF480530193124A03E08E
:108E0800019B591E0191E3B113889C05F8D40121F7
:108E180004460D4807F016FC0B48114907F018FDE9
:108E280010E001240EE002240CE003240AE00424EC
:108E380008E0052406E0062404E0072402E00824EC
:108E480000E0092420461CBD005400400100030036
:108E5800820007000400001002000010400000100B
:108E68000004001082B0002304E0019B0133019349
:108E7800009B01330093009B8342F6D302B07047F6
:108E880037B54FF4805304460D46019304E0019B27
:108E98005A1E0192002B6DD03C484FF4003107F068
:108EA800BDFC0028F3D13948012107F0ABFB4FF492
:108EB8008053019304E0019B5A1E0192002B5BD062
:108EC8003248334907F095FC0028F4D02F48A021F8
:108ED800002207F0AFFB4FF48053019304E0019B9D
:108EE8005A1E0192002B49D028482A4907F081FCD4
:108EF8000028F4D0210A254807F01FFC4FF48053BE
:108F0800019304E0019B5A1E0192002B38D01F48A0
:108F1800214907F06EFC0028F4D0E1B21B4807F0A5
:108F28000CFC4FF48053019303E0019B5A1E0192FD
:108F380043B31648184907F05CFC0028F5D01348DD
:108F4800294607F0FAFB4FF49613019303E0019BBF
:108F58005A1E0192C3B10D48104907F05FFC002862
:108F6800F5D00A48012107F059FB0D48FFF77AFFB1
:108F780000200AE0012008E0022006E0032004E0C7
:108F8800042002E0052000E006203EBD0054004019
:108F980001000300820007008000070004000010A1
:108FA800A0860100F7B54FF4805304460D461646D7
:108FB800019304E0019B5A1E0192002B74D0404893
:108FC8004FF4003107F02AFC0028F3D13C48012176
:108FD80007F018FB4FF48053019304E0019B5A1EDD
:108FE8000192002B62D03648364907F002FC00286F
:108FF800F4D03348A021002207F01CFB4FF4805323
:10900800019304E0019B5A1E0192002B50D02C487A
:109018002D4907F0EEFB0028F4D0210A284807F074
:109028008CFB4FF48053019304E0019B5A1E01927C
:10903800002B3FD02248254907F0DBFB0028F4D05D
:10904800E1B21F4807F079FB4FF48053019304E025
:10905800019B5A1E0192002B2ED019481B4907F07C
:10906800C8FB0028F4D000244FF4961710E0295DBF
:10907800134807F062FB019703E0019B5A1E019217
:10908800E3B10F48124907F0C9FB0028F5D00134B5
:10909800E3B2B342EBD30A48012107F0BFFA0D4807
:1090A800FFF7E0FE00200AE0012008E0022006E0C9
:1090B800032004E0042002E0052000E00620FEBDB5
:1090C80000540040010003008200070080000700F0
:1090D80004000010A086010013B50520012107F047
:1090E800F5FC184C4FF4E053009302238DF804303C
:1090F8008DF805302046002369468DF806308DF836
:10910800073007F03BF920460A21062207F0B6F996
:1091180020460C21062207F0B1F9062220460B2131
:10912800A4F5006407F0AAF94FF400432046694605
:10913800009307F023F920460F21062207F09EF935
:109148001CBD00BF000802401FB50446FFF7C2F867
:10915800FFF75EFBFFF7EAF8FFF7BEFF01214FF4C8
:10916800004007F0D7FC02940F4C1023ADF80230F2
:10917800204600236946ADF80430ADF80C30ADF850
:109188000030ADF8063007F0F4FD69464FF0402096
:1091980007F0C3FE2046012107F073FE4FF0402080
:1091A800012107F06EFE1FBD003C004082B0002385
:1091B80004E0019B01330193009B01330093009B62
:1091C8008342F6D302B0704707B50420012107F0A7
:1091D8007DFC01214FF4804007F0A8FC4FF4007398
:1091E800009300238DF804300348012369468DF865
:1091F800073007F0C3F80EBD000802400D4B07B555
:109208001A680D484FF47A73B2FBF3F20B4B013A2C
:109218005A600B4AF02182F8231000229A60072234
:109228001A60084B084A00930121084B01F0F8FF27
:109238000EBD00BFE40100205026002010E000E031
:1092480000ED00E000030020E40200204C020020B2
:10925800054B1A6812B11A68013A1A60034B1A686A
:1092680001321A60704700BF0C2600202426002017
:1092780082B0044B0190019A1A601A68002AFCD146
:1092880002B070470C260020704700BF40F0BE6057
:10929800024B40F42020D860704700BF00ED00E08A
:1092A800C37810B503B3164B4278DB688478DB4388
:1092B800C3F30223C3F10401C9B202FA01F10F2278
:1092C80042FA03F2C9B222400A430E4B0178120156
:1092D800CB18D2B283F8002303780122590903F08E
:1092E8001F0302FA03F307E003780122590903F088
:1092F8001F0302FA03F32031024A42F8213010BD5D
:1093080000ED00E000E100E021F0604121F07F0184
:10931800014B08439860704700ED00E0044B1A6960
:1093280009B1104301E022EA00001861704700BF4C
:1093380000ED00E0044B1A6804280CBF42F0040258
:1093480022F004021A60704710E000E0014B93ED30
:10935800000A7047702C0020014B93ED000A7047FB
:10936800682C0020014B93ED000A70477C2C0020EC
:10937800014B93ED000A70476C2C0020014B93EDD4
:10938800000A7047802C0020014B93ED000A7047BB
:10939800742C00200000000008B5FDF743FE0020F3
:1093A800012324210246FDF7A7FE124B1B78013B3F
:1093B800DBB20020012B05D80146FDF776FF01201E
:1093C800002104E00721FDF770FF01200721FDF7C8
:1093D8006CFF63221221C020FFF74AFA0220012104
:1093E800FDF763FFFEF740F80120BDE80840FEF7EF
:1093F80030B800BF1C0E00200E4B1B78062B05D181
:109408000D4B0E4A196812688A181A600C4B1B78A3
:10941800013BDBB2012B084B196805D8094A914278
:1094280007DD01321A607047074A914201DD0132B7
:109438001A607047CD250020442C0020C425002048
:109448001C0E00207FD1F008FF27ED080F4B1B787A
:10945800062B05D10E4B0F4A196812688A1A1A6032
:109468000D4B1B78013BDBB2012B094B05D80B4A8E
:109478001968914208DC1A6070471A68B2F57A2FA9
:10948800DCBF4FF47A221A60704700BFCD25002058
:10949800442C0020C42500201C0E002020A1070019
:1094A8002DE9F04F6A4B6B4C1B688DB019220A905E
:1094B80069485343B0FBF1F01C190D4608F096FEBD
:1094C80041EC100B0AF0E4FF51EC100B09F0C6F95F
:1094D80010F0010F804618BF00F1FF3805FB08F0B7
:1094E80008F084FE064620460F4608F07FFE024636
:1094F8000B463046394609F019F804460D4645EC46
:10950800104B0AF0C5FF57EC106B204632463B461D
:10951800294608F02DFDCDE902013946304609F00B
:109528009DF947A3D3E900230B90DDE9020109F077
:109538004FF9002858D1012000264FF0150931466F
:1095480007464FF0000A4FF0000B03E0304639465B
:10955800069E049FA7FB0A23541807FB0B333F4AB8
:1095680043F100050023A242AB41CDE904453ED3B7
:10957800A6FB0A23141806FB0B33384843F10005F1
:109588000021A042A941CDE9064530D3DDE9020119
:109598002DA3D3E90023049C069D09F019F940BBCB
:1095A800DDE9022300202E4908F0C0FF82468B46E1
:1095B8004BEC10AB0AF06CFF5046594653EC102B9D
:1095C8008DED080B08F0D4FCCDE90201DDE90801B6
:1095D80009F012FC09F1FF395FFA89F982468B46D6
:1095E800B9F1000FB2D104E00125002401E03546AD
:1095F8003C460B9A0A9BD1B25BB9184622462B46C9
:10960800FDF77AFD0A980123009301464246034676
:1096180009E022462B460120FDF76EFD012000904F
:10962800014642460023FDF75AFEFDF71DFF0120C3
:109638000DB0BDE8F04FFDF70CBF00BFAFF30080E1
:10964800956479E17FFDA53DBBBDD7D9DF7CDB3DC6
:10965800403A002040787D0100E9A435FFFF0F0063
:109668000000F03F244A254B1278013AD2B2012A71
:1096780010B5186009D8224A904201DD01321A60FB
:10968800204A1B6893420DDC0AE01F4A904201DD24
:1096980001321A601B68B3F57A2F03DC4FF47A2283
:1096A800164B1A60154B194A1968194B194C1B6847
:1096B800CB18934223601ADC0020FFF7F1FE01204B
:1096C8002168FFF7EDFE0C4B1B78013BDBB2002055
:1096D800012B05D80146FDF7E8FD0120002104E033
:1096E8000721FDF7E2FD01200721FDF7DEFD034B11
:1096F8001A68094B1A6010BD1C0E0020442C00206B
:109708007FD1F00820A10700FF27ED0880D1F008DD
:109718005C2C0020602C002028360020014B1868A3
:10972800A0E700BF402600207047FEE7FEE7FEE7FF
:10973800FEE770477047704702F02EB910B5094C24
:10974800A37A4BB1084B1A6822F006021A6000F09F
:1097580013F8204600F041FE4FF48020BDE8104089
:1097680006F068BB5026002010ED00E0014801F02B
:1097780003B800BF50260020364BD3F8882042F4A7
:109788007002C3F88820344B1A6842F001021A604C
:1097980000229A60196821F0847121F480311960DF
:1097A8002E495960196882B021F480211960DA6065
:1097B800009201921A6842F480321A601A6802F420
:1097C80000320192009A01320092019A1AB9009A65
:1097D800B2F5A06FF2D1204B1B6813F4003318BF09
:1097E80001230193019B012B2ED11B4B1A6C42F0D4
:1097F80080521A641A4A116841F4804111609A68CB
:109808009A609A6842F400429A609A6842F4A052B8
:109818009A60144A5A601A6842F080721A6019688D
:109828000D4A8901FBD5104B40F205611960936818
:1098380023F003039360936843F0020393609368F3
:1098480003F00C03082BFAD1024B4FF000629A6028
:1098580002B0704700ED00E00038024010300024EC
:109868000070004008544007003C0240184B194A59
:10987800996801F00C01042903D0082903D0164B7C
:1098880019E0164B17E059685A6811F4800F5968A7
:1098980014BF124B104B02F03F02B3FBF2F30C4A19
:1098A8005268C2F30142C1F38811013252004B439E
:1098B800B3FBF2F3074A1360054B9A68054BC2F3F2
:1098C80003129A181968127921FA02F21A6070477D
:1098D80000380240E40100200024F40000127A005D
:1098E80037B51C230124002501A88DF804308DF814
:1098F80005508DF806408DF80740FFF7D1FC20464B
:10990800214607F007F90A4940F2E1434B6040F26B
:109918004F130B800D814D804FF0804007F0A2FC63
:109928004FF080402146224608F061F83EBD00BF56
:10993800842C002008B54FF08040012108F06CF815
:1099480060B101214FF0804008F071F8FEF746FA47
:10995800034B044A11781A788A181A7008BD00BF98
:10996800F02500203C3A002008B5402006F054FAC3
:1099780030B1FCF785FD4020BDE8084006F05ABA32
:1099880008BD0000014608B5044808F00FFA03486E
:10999800402108F0B8FA0028F9D008BD004400407A
:1099A800F0B589B04FF4E1330120019300232B4C2B
:1099B800ADF808301E460146ADF80A30ADF80C3057
:1099C800ADF810300C23ADF80E3007F07FF84FF4E7
:1099D8000030012107F09EF820680221072206F0D6
:1099E8004DFD07226068032106F048FD0125022786
:1099F80004232068059305A98DF81A608DF81B507B
:109A08008DF818708DF8197006F0B8FC0823606896
:109A1800059305A98DF8187006F0B0FCA06801A997
:109A280008F01AF92A4640F225510D4808F052FA72
:109A3800262307A88DF81C308DF81D608DF81E6050
:109A48008DF81F50FFF72CFCA068294608F081F913
:109A5800044A054B1A6009B0F0BD00BFF8010020A8
:109A6800004400408D990008CC3B0020024B9868C8
:109A7800002108F06EB900BFF801002010B5094CAC
:109A880040F22551204608F048FA50B1A288D2B2D7
:109A9800112A02D1044B01211970044B19884A403C
:109AA8001A8010BD004400407D0D0020880D002064
:109AB8007047704773B50120014607F007F8264C38
:109AC8004FF4D8530093022303268DF80430204620
:109AD800002369468DF806308DF807308DF805604B
:109AE80006F04CFC204608210A2206F0C7FC204656
:109AF80009210A2206F0C2FC20460B210A2206F0A0
:109B0800BDFC0A2220460C2106F0B8FC01254FF4C2
:109B180080632046694600938DF806508DF80750FB
:109B28008DF8056006F02AFC0A210A46204606F050
:109B3800A5FC29464FF4804006F0F8FF802029460E
:109B480006F0D0FF4FF08050294607F01FF828464E
:109B580006F070F97CBD00BF0000024007B54FF465
:109B6800C060FFF793FB43238DF8043003220123E1
:109B780001A88DF805308DF806208DF80730FFF71D
:109B88008FFB0EBD782358430723B0FBF3F0002367
:109B980001338342FCD970474FF47A735843F1E795
:109BA80037B50023104C019305460320FFF7EAFF61
:109BB800EB681A69013C019213D0019A002AF4DA81
:109BC800019A42F001020192019A1A61064A196942
:109BD800013A019102D00199C907F8D40320FFF78F
:109BE800D1FF00203EBD00BF410D030010B5C47871
:109BF80074B900EB820003339B10D0F8D0002246E2
:109C080003E051F8044C0132046004319A42F8D15F
:109C1800002010BD033230B59210D0F8D0400B466A
:109C2800002003E02568013043F8045C04339042C7
:109C3800F8D101EB800030BD0122F0B5002382701D
:109C480040220129C37082800CD1082303700423A9
:109C580043704FF4A073C38002230372C1724FF0A4
:109C6800A04309E041B90C230370062343704FF465
:109C7800A063C3801F4BC17203F500620261C36019
:109C88004678044601461A46002508E002F5106C9D
:109C980002F530620A65C1F814C001353A4604314C
:109CA800B54202F12007F1D303F58062426103F562
:109CB8008862C0F8CC20067803F5A065014600222A
:109CC80003E0C1F88C50013220350431B242F8D398
:109CD8001946002202E0C4F8CC1001320434B24222
:109CE80001F58051F7D303F56063C0F80C3100200B
:109CF800F0BD00BF0000044038B5037AC2680025F3
:109D0800012B044625D1936B417A65F3104309B1C1
:109D180043F480139363D36823F4800323F0500340
:109D280043F010036FF3C3036FF3C7136FF351438B
:109D38006FF3D343D3602046FFF732FFE378012B5C
:109D48003ED1052363F34405E36845F020059D6093
:109D580036E0D36843F04003D360FFF721FF237A4E
:109D6800627A032B14BF4FF434134FF43C130AB137
:109D780043F48013E26814209363FFF70DFFE26851
:109D8800217AD368032908BF43F48033D360237A48
:109D9800032B15D1156B012363F39B656FF3D7551F
:109DA8002D2345F0805563F316451563C820FFF74A
:109DB800F3FEE36845F400051D63C820FFF7ECFED9
:109DC800E378012B07D1E3689D68052262F3440517
:109DD80045F020059D60002038BDC3689A6842F0B0
:109DE80001029A6000207047C3689A6822F0010255
:109DF8009A600020704707B500230193019B43F048
:109E080020030193019B61F38A130193019BC268AC
:109E18001361064B1169013B019102D00199880633
:109E2800F8D40320FFF7AEFE00200EBD410D03005D
:109E380007B500230193019B43F010030193019B95
:109E4800C2681361064B1169013B019102D0019967
:109E5800C906F8D40320FFF795FE00200EBD00BF09
:109E6800410D030008B5C268D36801296FF35D731B
:109E78006FF39E7302D143F0005302E009B943F037
:109E880080433220D360FFF787FE002008BDC368F7
:109E9800586900F001007047C3685B6913F0010F4F
:109EA80014BF002001207047C368586900F0010002
:109EB8007047C3685A69986910407047C368586802
:109EC800704703691A6861F301021A607047C26833
:109ED800002393614FF0FF335361536053610B4B81
:109EE8009361C3789169002B14BF4FF400634FF45A
:109EF800016343F4701343F4405343F0080321EA29
:109F080003010B4393610020704700BF00080080E5
:109F1800F8B5D0F80C3100221A60036915461A68A2
:109F280065F3CC221A60C37A012B04461BD10321A6
:109F3800FFF7C7FFE36880214FF4800261F30F0247
:109F480059629A62C02262F30F0561F31F454FF40C
:109F5800A072C3F8045162F30F056FF31F45C3F8ED
:109F68000851C3F80C5110212046FFF744FF204642
:109F7800FFF75EFF226900234FF0FF31136120468F
:109F880053611E469161FF25D361214610E0826925
:109F98001768C7F3076707F08007FFB2002F14BFE1
:109FA8004FF0904700271760013316610430956021
:109FB80062789342EBD300231D46FF2010E04A6DE0
:109FC8001668C6F3076606F08006F6B2002E14BFC0
:109FD8004FF09046002616600133156104319060F9
:109FE80062789342EBD323691A6942F480721A614A
:109FF800E278012A04D1054A402161F359421A63E3
:10A008002046FFF764FF0020F8BD00BF03010100F0
:10A0180003699B68C3F34103013B022B9ABF024AC1
:10A02800D05C0320704700BF90AA040810B50369EC
:10A0380081699C680A68C4F34100022802D06FF362
:10A048000A0202E0032060F30A020A605A6842F436
:10A0580080725A60002010BD30B54D780B78002210
:10A06800012D00EB830405D105FA03F3A46963F31A
:10A078000F0205E0012505FA03F3646D63F31F423F
:10A088002368C3F3072505F08005EDB26DB98D6827
:10A0980065F30A03CD78C98865F3934361F399534F
:10A0A80043F0805343F4004323600369D9690A43AA
:10A0B800DA61002030BD30B54D780B780024012DD1
:10A0C800224600EB830105D105FA03F3896963F39E
:10A0D8000F0205E0012505FA03F3496D63F31F42FA
:10A0E80003696FF3CF340C60D96921EA0202DA619F
:10A0F800002030BDF8B54F780B78012F00EB8303B3
:10A1080049D19E694C69356833692A4664F312035C
:10A1180014B967F3DC430BE08F68E419013CB4FB26
:10A12800F7F7CC7867F3DC43012C08BF64F35E7360
:10A138003361C378012B06D10B780C6900EB8303DC
:10A148009B695C610CE0CB78012B09D04B693BB172
:10A1580003690C785E6B012707FA04F434435C63E7
:10A16800CB78012B07D103699B68DB0554BF45F009
:10A17800005245F080520B7800EB830342F0044212
:10A188009B691A60CB78012B38D10A788B8AC96809
:10A19800FFF72CFD32E05E6D4F6935688C683369D6
:10A1A8002A462FB964F31203012464F3DC430AE05E
:10A1B8003F19013FB7FBF4F7BF05BF0D67F3DC4359
:10A1C8007C4364F312033361C378012B05D10B7808
:10A1D8000C6900EB83035B6D5C61CB78012B06D1C6
:10A1E8004B7913B145F0005201E045F080520B78ED
:10A1F80000EB830042F00442436D1A600020F8BD72
:10A2080073B54D78012D3DD183694A691E681C6973
:10A218000094E4B242B962F306048DF800409DF858
:10A22800024065F3C4040EE08D68AA4286BF4D6102
:10A2380065F3060462F306048DF800409DF80240B9
:10A24800012262F3C4048DF80240009A1A61C278B0
:10A25800012A05D10A780C6900EB820292695461DF
:10A2680046F004421A60C378002B34D14B69002BA6
:10A2780031D003690A78586B012101FA02F20243CE
:10A288005A6328E00B784E698C6800EB83035B6D9A
:10A298001A681D690095EDB206B14C6164F30605B4
:10A2A8009DF802408DF80050012565F3C4048DF82F
:10A2B8000240009C1C61C378012B05D10B780C6906
:10A2C80000EB83035B6D5C610B7800EB830042F06D
:10A2D8000442436D1A6000207CBD4B78012B0B783B
:10A2E80000EB83000AD182691368C3F3076101F0A8
:10A2F8008001C9B221B143F0804301E0426D136887
:10A3080043F400131360002070474B78012B0B783F
:10A31800C97800EB83000CBF8269426D023913686B
:10A32800C9B26FF35553012998BF43F080531360A6
:10A338000020704703699A69D8691040000C70477B
:10A3480000EB810102694B6D9B68506918407047AA
:10A3580003699869DB69184080B2704782B00023AE
:10A368000093C0238DF803300122002362F3C40355
:10A378008DF8023018238DF80030009A436D1A6169
:10A38800C278012A06D100F5B96058611A684FF001
:10A3980080221A6002B07047D0F8143110B5044614
:10A3A800D3B103699A68D20716D5827A42B1D0F838
:10A3B8000C21D0F80C116FF341026FF300020A6010
:10A3C8005A6842F001025A600520FFF7E5FB23694D
:10A3D8005A6822F001025A6010BD837A63B103699A
:10A3E8009B68D90708D5D0F80C31D0F80C216FF349
:10A3F80041036FF3000313607047012310B5002277
:10A4080080F8123104460346FF2104E05869816050
:10A41800186D01328160607804338242F6D3236973
:10A4280000221A615A61DA614FF0FF329A612046C0
:10A43800FFF7FEFC20461021BDE81040DBE44B7816
:10A44800012B0B7800EB83000FD183691868C0F3E8
:10A45800074000F02003DBB2CBB900F00200C0B225
:10A4680000280CBF302020207047436D1868C0F3C7
:10A47800074000F02003DBB25BB900F00200C0B275
:10A4880000280CBF4FF440504FF400507047102084
:10A4980070474FF4805070474B78012B0B7810B5FC
:10A4A80000EB83030AD19C69102A236802D1BDE816
:10A4B800104012E7202A0CD0302A0FE05C6DB2F56C
:10A4C800805F236802D143F400131BE0B2F5005FFC
:10A4D80002D143F0006315E0B2F5405F0FD1C3F33A
:10A4E800074202F02002D2B222B100234B71BDE82C
:10A4F80010400AE743F0806343F0802302E00AB982
:10A5080062F3CF33236010BDF8B50446FFF794FB20
:10A518000122002384F8122184F8133128271646D3
:10A52800194640250CE007FB03F000F58C70221853
:10A538002354D3805670D1709560D1605161013336
:10A5480062789342EFD300232826194640250CE071
:10A5580006FB03F000F55C7022182354D380517079
:10A56800D1709560D1605161013362789342EFD325
:10A578002046FFF739FC2046FFF7BEFB00212046A6
:10A58800FFF770FC2046FFF7C3FC2046BDE8F84003
:10A59800FFF723BC70B5CDB20C464FF0280601F08A
:10A5A8007F0106FB010115F0800F14BF01F58C71C6
:10A5B80001F55C7104F07F04ED090C704D708A6040
:10A5C800CB7005B1CC80022B01D100230B71FFF7B2
:10A5D80043FD002070BD10B5CAB201F07F034FF0F3
:10A5E800280404FB030312F0800F14BF03F58C73D7
:10A5F80003F55C7301F07F01D20919705A7019468E
:10A60800FFF759FD002010BD38B501F07F0528245B
:10A618006C4304F55C7401194B6100238B614B702A
:10A62800EBB20355CA60C478012C08BF0A6113B99C
:10A63800FFF7E6FD01E0FFF75DFD002038BD70B5CE
:10A6480001F07F042825654305F58C75411901261D
:10A65800E4B2CA600A6100224E7044558A614B61B7
:10A6680014B9FFF7CDFD01E0FFF744FD002070BDF0
:10A67800CAB212F0800F10B54FF0280306D001F0CF
:10A688007F0403FB040303F58C7303E003FB01035E
:10A6980003F55C73D209012401F07F0119709C70E5
:10A6A8005A701946FFF719FE002010BDCAB212F001
:10A6B800800F10B54FF0280306D001F07F0403FB8C
:10A6C800040303F58C7303E003FB010303F55C73D8
:10A6D8000024D20901F07F0119709C705A70194644
:10A6E800FFF713FE204610BD08B50B0604D501F090
:10A6F8007F01FFF780FB01E0FFF79AFB002008BD10
:10A708000369002261F30A1219680A431A60704744
:10A7180003695A6803206FF341025A60FFF73CBA95
:10A7280003695A68032042F002025A60FFF734BAFC
:10A7380011F0800F4FF0280306D001F07F0103FBD2
:10A74800010101F58C7103E003FB010101F55C7166
:10A75800FFF775BE11F0800F4FF0280306D001F007
:10A768007F0103FB010101F58C7103E003FB01018B
:10A7780001F55C71FFF790BE2DE9F74F0446FFF72E
:10A788008BFB002800F03F822046FFF792FB05462E
:10A79800002800F03882C0F3074000F00800C0B27B
:10A7A800002861D02046FFF7C5FDA146824627460E
:10A7B8004FF00008DFF86CB32E4650E01AF0010F96
:10A7C80046D05FFA88F2114620460092FFF7B8FD9E
:10A7D80010F0010F0546009A20D07B6D01259D6081
:10A7E800E178A94207D11B69D9F87813C3F312039A
:10A7F800CB1AC9F88833DBF8003020461B681146AD
:10A808009847E378012B09D1B8F1000F06D194F8E5
:10A818001131052B02D12046FFF7A0FD05F00203F8
:10A82800DBB213B17B6D02259D6005F00403DBB23A
:10A8380013B17B6D04259D6005F00805EDB23DB1AF
:10A84800DBF8003020469B6898477B6D08209860AD
:10A8580008F101084FEA5A0A043709F12809BAF140
:10A86800000FABD135460120C5F3074303F00403BD
:10A87800DBB2002B00F0AF802046FFF769FD2646CB
:10A8880083464FF0000801959FE01BF0010F00F090
:10A89800978023695FFA88F919695D6B04EB89026F
:10A8A80025FA09F59269ED019268EDB20D4315405C
:10A8B800EA071CD55A6B012000FA08F122EA0102C6
:10A8C8005A63B369974A9860136805465B682046DF
:10A8D80049469847E378AB4209D1B8F1000F06D151
:10A8E80094F81131042B02D12046FFF737FD05F00B
:10A8F8000403DBB213B1B36904259D6005F00803B6
:10A90800DBB213B1B36908259D6005F01003DBB213
:10A9180013B1B36910259D6005F02003DBB213B1B4
:10A92800B36920259D6005F04003DBB213B1B3691C
:10A9380040259D6005F00203DBB213B1B36902251F
:10A948009D6025F07F0515F0FF0F39D0282505FB00
:10A95800084505F58C75C246AB696A69C3EB020CFC
:10A96800AB689C4528BF9C460CF1030CB3694FEAC1
:10A978009C0C9B696746A04614E0AA68E9681C1B02
:10A98800944228BF1446A3B240464A46FFF72EF920
:10A99800EB681B19EB60AB69E71C1C19AC61B36968
:10A9A8009B69BF089BB2BB4205D9AC696B699C42E5
:10A9B80001D2002BE1D1B369802544469D60D04681
:10A9C80008F101084FEA5B0B0436BBF1000F7FF476
:10A9D8005CAF019D012005F00203DBB213B1E3680F
:10A9E80002225A61C5F3076303F08003DBB2CBB1DF
:10A9F800A37A43B1D4F80C31D4F80C216FF3410396
:10AA08006FF30003136023695A6822F001025A6049
:10AA1800444B1B6820469B699847E3684FF0004207
:10AA28005A610120C5F3072303F00803DBB2F3B131
:10AA38003C4B1B6820465B6998472369E2689B6822
:10AA48004FF400615161A27A82B1DB070ED5D4F8C8
:10AA58000C311A6842F001021A601A6842F00302C7
:10AA68001A60314B1A6942F006021A61012005F09A
:10AA78000803DBB243B12B4B1B682046DB689847C1
:10AA8800E36808225A61012005F01003DBB2002BAD
:10AA980033D0E3689A6922F010029A611F6A282667
:10AAA80007F00F0306FB0346C7F34343022B06F5E3
:10AAB8005C7602D0062B1AD10EE047F6F0733B40C5
:10AAC800ABB1C7F30A172046F1683A46FFF7A2F878
:10AAD800F368DB19F36007E004F5B9612046082242
:10AAE800FFF798F8C7F30A17B369DF19B761E36886
:10AAF8009A6942F010029A610120C5F3072303F016
:10AB08001003DBB2002B39D023695A68002622F0E3
:10AB180001025A6031462046FFF76DF92346324656
:10AB2800FF2108E09402002000ED00E058698160F0
:10AB3800186D01328160607804338242F6D323694C
:10AB480001274FF0FF3267F30F069A6167F31F463C
:10AB58000F22DE615A612F221A611A686FF30A12F6
:10AB68001A602046FFF7FAFBE3684FF480525A61F7
:10AB7800264B1B6820461B6998473846C5F30723B0
:10AB880003F02003DBB2EBB12046FFF74FFAE3688E
:10AB98002046DE68FFF73CFA032806D10023A3709D
:10ABA8004FF40073A380092304E00123A37040231A
:10ABB800A380052363F38D26E3684FF40052DE601B
:10ABC80001205A61C5F3074303F01003DBB24BB110
:10ABD8000E4B1B682046DB699847E3684FF48012E8
:10ABE8005A610120C5F3074505F02005EDB255B1BE
:10ABF800064B1B6820461B6A9847E3684FF400120F
:10AC08005A610120FFE7BDE8FE8F00BF94020020D3
:10AC180043230B80004870470402002038B51F4BBF
:10AC28001A68511C052A196035D1197900220129A1
:10AC38001A6030D09968B1F5006F08BF9A60174B59
:10AC48009968DC68A1421A4602D100221A7122E0F2
:10AC580086BFC1F500631361C1EB0404D0F8EC357D
:10AC680098BF14611569B3F839300C4C9D428AB20B
:10AC780004D95918ED1AA160256104E06918A1608A
:10AC88000021ABB22161054901240C7104498A18DD
:10AC98008121FFF7D4FC002038BD00BF8C0D0020B7
:10ACA800232D002038B528230A4D03FB01010A4B48
:10ACB800B1F888131B69044628469847D4F8EC3540
:10ACC8002046B3F8403001212A46FFF79DFC0020BA
:10ACD80038BD00BFDB2C00208002002070B50B7847
:10ACE80013F0600506460C4625D0202D1FD1CD88CF
:10ACF800B5B113F0800F487808D0214B21499B68E3
:10AD08002A469847E2881F49304625E01E4B1D49D0
:10AD180058641E4B30465D612A4600F022FB1DE058
:10AD2800174B48789B6829462A46984725E000F043
:10AD380077FB022521E04B780A2B11D00B2B14D07E
:10AD4800062B1AD14B881B0A212B03D1CA883A2A11
:10AD580028BF3A220E49304600F0EAFA00250CE0F6
:10AD68000C49012200F0E4FA07E08B781BB9074A86
:10AD78001D46936101E000F053FB284670BD00BFFB
:10AD8800800200201B2D0020040200208C0D0020D2
:10AD980016020020A40D002010B581210446FFF7FB
:10ADA8001AFC01212046FFF716FC82212046FFF7F6
:10ADB80012FC024B5B689847002010BD80020020FF
:10ADC80038B5D0F8EC350446B3F839208121022390
:10ADD800FFF7E0FBD4F8EC350121B3F8402020461A
:10ADE8000223FFF7D7FB8221082203232046FFF71F
:10ADF800D1FB094B022200251A715D71074B1B68B4
:10AE08009847D4F8EC35064AB3F84030204601217B
:10AE1800FFF7FAFB284638BDC40200208002002054
:10AE2800DB2C002010B5074C606CFF2807D0064BC0
:10AE3800064A9B68064952699847FF2363640020C5
:10AE480010BD00BF04020020800200208C0D0020ED
:10AE58001B2D002038B510490B79012B19D10C692D
:10AE68000CB90C7115E0D0F8EC358D68B3F83930B1
:10AE78009C42AAB203D95D198D60E41A03E0A3B21B
:10AE88002C198C6000240C61044952188121FFF7A9
:10AE9800D6FB002038BD00BF8C0D0020232D0020DC
:10AEA80000207047002070470023F0B5084A094E7B
:10AEB8001D4609E01468C75C375501340133B4F501
:10AEC800006F146008BF15608B42F3D10020F0BDFD
:10AED800980D0020232D0020104B114AD3F800C0F4
:10AEE80000232DE9F0410F4F16461D460DE014686A
:10AEF80010F8038007F804800134802C08BF2C4622
:10AF080014603468644505D001338B42EFD10020CA
:10AF1800BDE8F0810220BDE8F08100BFA435002023
:10AF2800B83500202435002021280FD1084B1A6895
:10AF38000A701A68120A4A705A888A70DA78CA70CF
:10AF48001A790A715A794A719B798B710020704776
:10AF58007802002007B502AB012103F8010D18465D
:10AF6800FFF7A2FF0EBD002100E00131435C002B7A
:10AF7800FBD199E798E70B4B0B491A68096891428E
:10AF88000BD00A498A5C02701A680132802A1A605A
:10AF980005D100221A600120704700207047012067
:10AFA800704700BFA4350020B835002024350020A4
:10AFB800204B1A68204B1B689A42F0B509D135E03E
:10AFC8000133802B08BF00239A4203D11A4B1A6021
:10AFD8002CE01A4CE15C0029F2D00A29F0D00D29A6
:10AFE800EED0154C1549134D23600E460023CF189B
:10AFF8002268BA5CC254226801339F18802F08BFA8
:10B0080053422F689A18974210D0B25C1AB10A2A94
:10B0180001D00D2AEBD10022C254074A11685918F1
:10B028007F29116003D98039116000E00023184698
:10B03800F0BD00BFB8350020A4350020243500201D
:10B04800704700BFD0F8E43510B51B69044698472F
:10B05800032384F81231002010BD08B5042380F8BA
:10B068001231D0F8E435DB689847002008BD08B5F0
:10B07800D0F8E035DB6903B19847002008BD08B572
:10B08800D0F8E0351B6A9847002008BD08B5D0F80D
:10B09800E0355B6A9847002008BD002110B54022C2
:10B0A80004460B46FFF776FA80214022002320460B
:10B0B800FFF770FA012384F81231D4F8E435A07848
:10B0C8005B689847002010BD13B56946044600F038
:10B0D80085F99DF8001001F01F03012B07D0022B02
:10B0E8000AD073B92046694600F026FA0FE02046D8
:10B0F800694600F007FA0AE02046694600F0A2F91E
:10B1080005E021F07F01C9B22046FFF7B1FA00201F
:10B118001CBD38B5044600293DD190F81131022BE9
:10B1280042D1D0F83421D0F820319A4211D9C178CF
:10B13800D21A0129C0F8342104D1D0F82411CB182F
:10B14800C0F8243192B22046D4F8241100F000F956
:10B158002AE0D0F83821B2FBF3F503FB152565B9D1
:10B168009A420AD3D0F83C319A4206D229462A4656
:10B1780000F0EEF8C4F83C5116E0D4F8E035DB688E
:10B188002BB194F81221032A01D120469847204672
:10B1980000F00FF908E0D0F8E0355B6923B190F8CA
:10B1A8001221032A00D19847002038BD10B5044663
:10B1B80059BB90F81131032B30D1D0F88C23D0F83B
:10B1C80078339A4214D9C178D21A0129C0F88C234D
:10B1D80004D1D0F87C13C918C0F87C139A4228BF50
:10B1E8001A4692B22046D4F87C1300F0CAF815E04B
:10B1F800D0F8E0351B6923B190F81221032A00D159
:10B208009847204600F0C6F808E0D0F8E0359B697A
:10B2180023B190F81221032A00D19847002010BDCD
:10B228002DE9F041069F0446164698460D46FEF75E
:10B2380041FC20462946C4F8E085C4F8E475C4F802
:10B24800E865FFF761F9D4F8E4351B6898472046AC
:10B25800BDE8F041FEF782BC00207047D0F8E03529
:10B2680010B504461B689847D4F8E4359B6898479E
:10B27800002010BD08B5D0F8E0355B68984700207D
:10B2880008BD000012230B8000487047C40200204C
:10B2980004230B8000487047D602002010B5044CE8
:10B2A80004480A46214600F075FA204610BD00BF42
:10B2B800BC3500205EAF05080A4608B502480349B8
:10B2C80000F068FA014808BD71AF0508BC350020D8
:10B2D8000A4608B50248034900F05CFA014808BD6F
:10B2E8007FAF0508BC35002008B50A4608B90448F0
:10B2F80000E00448044900F04DFA034808BD00BFC7
:10B308008AAF050897AF0508BC35002008B50A467E
:10B3180008B9044800E00448044900F03BFA03482F
:10B3280008BD00BFA4AF0508C5AF0508BC3500209F
:10B3380010B513460C46C0F83821C0F83421022253
:10B3480080F8112100212246FFF779F9002010BD6D
:10B3580010B50C46134600212246FFF770F900206D
:10B3680010BD10B513460C46C0F89023C0F88C23C6
:10B37800032280F8112100212246FFF745F9002019
:10B3880010BD10B50C46134600212246FFF73CF9C4
:10B39800002010BD0021042310B50A46044680F899
:10B3A80011310B46FFF74BF92046FEF7D7FF002077
:10B3B80010BD0021052310B50A46044680F8113156
:10B3C8000B46FFF721F92046FEF7C8FF002010BD05
:10B3D800282303FB0100B0F88803704790F8C835AC
:10B3E8000B7090F8C9354B7090F8CB2590F8CA359A
:10B3F80003EB02234B8090F8CD2590F8CC3503EB76
:10B4080002238B8090F8CF2590F8CE3503EB0223EA
:10B418009BB2CB80C0F83C31012380F811317047D2
:10B4280010B591F90030002B044601DBCB880BB92D
:10B43800802100E00021FFF71BF92046BDE81040FD
:10B44800FEF78CBF38B50D4604466B780979012B99
:10B4580010D027D3032B51D190F81231022B28D0CA
:10B46800032B47D16B889BB991B1802910D0FFF786
:10B47800FFF80DE090F81231022B1AD0032B39D1C6
:10B488006B88002B3AD149B1802907D0FFF70EF914
:10B49800D4F8E03520469B68294698472046FFF7B0
:10B4A80079FF2BE090F81231022B02D0032B21D127
:10B4B80006E019B3802921D02046FFF7D9F81DE00E
:10B4C80011F0800F4FF0280306D001F07F0103FB35
:10B4D800010393F81A2103E003FB010191F8722399
:10B4E800074B02B101221A60204605490222FFF7E4
:10B4F8001FFF03E020462946FFF792FF002038BDD2
:10B50800A80D002038B590F81231032B04460D46DB
:10B518000CD10B79012B09D8D0F8E0359B689847F6
:10B52800EB883BB92046FFF735FF03E02046294664
:10B53800FFF776FF002038BD73B54B7804460D46FB
:10B54800092B00F21C81DFE813F0D10008011A0171
:10B55800E4001A0172000A001A01C00092004B8828
:10B568001A0A013A062A00F20A81DFE812F00700F7
:10B578001A0027000801080108010801D4F8E83575
:10B58800A0781B680DF106019847EB88402B01460F
:10B5980003D094F81231012B3AD10823ADF80630C4
:10B5A80036E0D4F8E035A0789B6A0DF1060198479B
:10B5B800022343700146C4F8EC0529E0DBB2052BF1
:10B5C80000F2DD80DFE803F003080D12171CD4F841
:10B5D800E835A0785B6817E0D4F8E835A0789B6870
:10B5E80012E0D4F8E835A078DB680DE0D4F8E83547
:10B5F800A0781B6908E0D4F8E835A0785B6903E017
:10B60800D4F8E835A0789B690DF106019847014602
:10B61800BDF80630002B00F0B680EA88002A00F05A
:10B62800B2809A4228BF1A46ADF806205CE08B88A3
:10B63800002B40F0A480CB88002B40F0A08094F829
:10B6480012214B88032A00F09A8003F07F052046D8
:10B6580084F813512946FFF753F82046FFF79AFE5E
:10B668000DB1022300E0012384F812318BE08978C0
:10B67800464E0129317100F2828094F81231022B72
:10B6880002D0032B7BD108E0002962D001210323DB
:10B6980084F8101184F8123113E041B9022384F8B8
:10B6A800123184F810112046FFF7E4FD51E094F8B8
:10B6B8001011012920464DD0FFF7DCFD317984F8BF
:10B6C80010112046FFF7CAFD43E0CA88012A56D167
:10B6D80094F81231022B02D0032B50D102E02046FD
:10B6E8002B4913E004F5887120460FE094F81231D5
:10B6F800023B012B43D8D4F814312449002B0CBF4A
:10B708000123032341F80C3F20460122FFF710FED6
:10B7180039E04B88012B29D0022B34D18B8813F0C8
:10B72800FF0F30D121691B0A013B4A68042B0FD84F
:10B73800DFE803F0030507090B00012306E00223F5
:10B7480004E0032302E0042300E0052363F3061268
:10B758004A602046FFF71EFE15E094F81231023BBE
:10B76800012B0CD84B88012B0DD10023C4F81431C0
:10B77800D4F8E03520469B6829469847E9E72046F3
:10B788002946FFF74DFE00207CBD00BFA80D002014
:10B79800B00D002030B5C8B10023DDB20133C418A4
:10B7A80014F8014C002CF8D16B1C5B0013800B7053
:10B7B80003234B70022305E0CA545A1CD2B2023349
:10B7C8008C54DBB210F8012B002AF5D130BD00BF34
:10B7D8007047704770477047704770477047000060
:10B7E80008B5FCF729FA094B5A78187002435A70C1
:10B7F8001AB19A7801329A7030B99B78034A012BB2
:10B8080002D900235370937008BD00BFB80D002003
:10B818002DE9F84F3F4B1B78012B2DED028B09D0FA
:10B8280002D3022B0FD108E03B4B1A68802392FB0E
:10B83800F3F206E0384B1A6803E0374B1B68032223
:10B848005A43364B5A61364B1A8892B2002AFBD0BB
:10B85800334B00221A80FDF779FD10EE105AFDF7E0
:10B868007BFD284610EE104A06F0E2FC8046204692
:10B87800894606F0DDFC41EC100B41EC180B08F092
:10B88800AFFD57EC106BB0EE480AF0EE680A08F00E
:10B89800A7FE32463B46404649465BEC10AB06F0F5
:10B8A8001BFD06F0FBFF9FED1F8A07EE100ADFED78
:10B8B8001E7A57EE087A194C52465B46C4ED007A58
:10B8C8004046494606F008FD06F0E8FF07EE900AF4
:10B8D80027EE888A84ED018AFDF750FD84ED020A7F
:10B8E800FDF752FD84ED030AFCF7B4F80F4B6269CB
:10B8F8001B68D31A0E4A07EE100A1268F8EEC77AC8
:10B9080093FBF2F3C4ED047A2383BDEC028BBDE80C
:10B91800F88F00BF1C0E0020442C0020EC370020BC
:10B92800680D00200000F04200008C4240260020F4
:10B93800C425002007B50420012105F0C7F84FF4FD
:10B948006043009301238DF8043002238DF80530FD
:10B958000448002369468DF806308DF8073004F056
:10B968000DFD0EBD00080240084B1A684FF47A73AB
:10B97800B2FBF3F2064B013A5A60064AF02182F80C
:10B98800231000229A6007221A607047E401002001
:10B9980010E000E000ED00E0034B5A6812B15A686D
:10B9A800013A5A60704700BFB80D0020024B58603A
:10B9B8005A68002AFCD17047B80D002030B585B010
:10B9C80004460D4601A862490A220BF001FA614BB0
:10B9D8001B78032B10D8DFE803F00205080B01A839
:10B9E8005D4907E001A85D4904E001A85C4901E060
:10B9F8005C4901A80BF0D6FA04AA131913F80C3CF9
:10BA08005D19EDB22F2D01D80A3502E0392D01D983
:10BA18000A3DEDB204AB1C194FF6FF7004F80C5C3C
:10BA2800FAF796FA0020FAF795FB0DF103050F24B3
:10BA3800204623345A21002315F8012FA4B2FAF71F
:10BA4800A3FBB4F5A57FF3D164205A212C2200234F
:10BA5800FAF79AFB0023CD205A212C22FAF794FBFF
:10BA68000020FAF775FA3B4B1B78032B6ED8DFE8FA
:10BA780003F0022E576201A937480BF093FA0A2205
:10BA8800002135480CF0B6FB374A384B127818605D
:10BA9800012A0BD002D3022A15D109E0B0F5FA5FCA
:10BAA800BCBF4FF4FA521A60314A07E0314A00E04D
:10BAB800314A904201DC01321A60304A1B689342D5
:10BAC800C4BF2A4B1A602E4B1A682E4B26E001A9D8
:10BAD80022480BF067FA0A22002120480CF08AFB62
:10BAE800214A294B12781860012A0BD002D3022A66
:10BAF8002CD109E0B0F5FA5FBCBF4FF4FA521A60D6
:10BB08001B4A07E01B4A00E01B4A904201DC013255
:10BB18001A601A4A1B68934218DD1B4B1A6015E01D
:10BB280001A90F480BF03EFA0D4800210A220CF03B
:10BB380061FB164B09E001A90A480BF033FA0948E2
:10BB480000210A220CF056FB114B186005B030BDDD
:10BB5800E6AF05083F2600201026002034260020E6
:10BB68004A2C0020FC2500201C0E00204C2600201A
:10BB780050DA11001FA10700FFE0F50580D1F00899
:10BB880040260020442C0020642C0020402C00205B
:10BB9800F825002010B50D4B0D4C1A680D482146AC
:10BBA8000BF0D8F90C4B0D481A6821460BF0D2F966
:10BBB8000B4B0C481A6821460BF0CCF90A4B0B4882
:10BBC8001A682146BDE810400BF0C4B94C26002085
:10BBD800C6A5050810260020642C00203426002065
:10BBE800402C00204A2C0020F8250020FC250020AD
:10BBF8009FED010A704700BF000000009FED010A99
:10BC0800704700BF000000009FED010A704700BFA9
:10BC18000000000018B1012801D1034B00E0034BDC
:10BC28001868FDF71FBD00BF302600204026002001
:10BC380010B9034B18687047024B1868704700BF6B
:10BC48004C2600204026002010B9034B1868704786
:10BC5800024B1868704700BF642C00203026002073
:10BC680008B54FF49570FBF709FF40F26523C31A36
:10BC7800584240EB030008BD08B5C620FBF7FEFE9E
:10BC880040F28D13C21A504240EB020008BD4FF437
:10BC9800957040F26521FBF7E3BEC62040F28D1196
:10BCA800FBF7DEBEDCE760EEA00AB7EE007AF0EE46
:10BCB800606A70EE077A40EE006A47EEA70A36EE31
:10BCC800C77A08B5C7EE200A10EE900A06F0B0FA57
:10BCD8000022084B06F000FB0022074B06F04AF949
:10BCE80006F0DCFD07EE900AFDEEE77A17EE900A03
:10BCF8009F3008BD000059400000E03F38B52DEDE9
:10BD0800028BF7EE008AB0EE608A70EE288A10EE99
:10BD1800900A28EE088A06F08BFA08EEA88A002214
:10BD28000F4B06F0D9FA044618EE100A0D4606F035
:10BD38007FFA02460B462046294606F0F7FB00220A
:10BD4800084B06F017F906F0A9FD07EE900AFDEE7C
:10BD5800E77A17EE900A7730BDEC028B38BD00BF4A
:10BD6800000069400000E03F2DE9F04F884F2DEDBD
:10BD7800068B97E80F0091B00CAC103784E80F00E1
:10BD88000FCF05AE0FC697E807004FF6FF7386E89A
:10BD980007009F2077216422F7F7A3FDA0207721D1
:10BDA80064224FF6FF73F7F79CFD9E2077216422EB
:10BDB8004FF6FF73F7F795FD9F20762164224FF623
:10BDC800FF73F7F78EFD4FF6FF73782164229F20EB
:10BDD800F7F787FD0020F9F798F99F20772165226A
:10BDE800FAF7F8F80C349F2077216422FAF7F2F872
:10BDF8000DF12C0A0394F7EE009A4FF00F0B00E0B8
:10BE08004D460AF1040AF7EE008A9AED009A0024DA
:10BE1800B0EE68AA01E0B846354618EE900A06F07A
:10BE280007FA59A3D3E9002306F056FA06F036FDBF
:10BE380008EE900A38EEE98AB0EE490AF0EE480AB0
:10BE4800FFF731FFB0EE490AF0EE480A0646FFF761
:10BE580055FFB2B2074683B22CB9104619460F22D5
:10BE6800F9F712FA06E0A8B21FFA88F1CDF800B087
:10BE7800F9F7FAFF0134B4F5967FCCD13D46F7EED9
:10BE8800008A002401E045464E4618EE900A06F066
:10BE9800CFF93DA3D3E9002306F01EFA06F0FEFC15
:10BEA80008EE900A39EEE88AB0EE490AF0EE480A40
:10BEB800FFF7F9FEB0EE490AF0EE480A8146FFF7AF
:10BEC8001DFF1FFA89F2804683B22CB91046194625
:10BED8000F22F9F7D9F905E0B0B2A9B2CDF800B050
:10BEE800F9F7C2FF0134B4F5967FCCD1039B9A458C
:10BEF80086D104AD0DF12C0B4FF0000A01E0B846D5
:10BF0800B146043595ED009AF7EE008A002401E069
:10BF1800B846B14618EE900A06F08AF91AA3D3E992
:10BF2800002306F0D9F906F0B9FC08EE900A38EEBD
:10BF3800CA8AF0EE490AB0EE480AFFF7B4FEB0EE3E
:10BF4800480AF0EE490A0646FFF7D8FEB2B207469D
:10BF580083B22CB9104619462246F9F795F907E03D
:10BF68001FFA89F01FFA88F1CDF800A0F9F77CFFD5
:10BF78000134B4F5C87FCBD15D45C0D111B0BDEC5B
:10BF8800068BBDE8F08F00BF295C8FC2F528F03F13
:10BF980094AA0408121A06EE902A081AB8EEE67A4D
:10BFA80006EE900AF8EEE67A08B5C7EE277A17EE9D
:10BFB800900A06F03DF90022044B06F08DF90022A4
:10BFC800034B05F0D7FF06F021FC08BD00007440C4
:10BFD8000000E03F8A1A06EE902A081AB8EEE67AC0
:10BFE80006EE900AF8EEE67A08B5C7EE277A17EE5D
:10BFF800900A06F01DF90022044B06F06DF90022A4
:10C00800034B05F0B7FF06F001FC08BD00006940CE
:10C018000000E03F70B506460D460024610704D5D0
:10C02800A0B231462A46F9F72FF90134B4F5A07FBA
:10C03800F4D170BD70B506460D460024600704D5DE
:10C04800A1B230462A46F9F71FF90134C82CF5D1B8
:10C0580070BD234B1B78012B03D011D3022B3DD18C
:10C0680023E0204B1A68204B1A60204B1A68204B9B
:10C078001A60204B1A68204B1A60204B1A6811E08E
:10C08800184B1A68184BD2011A60184B1A68184BCB
:10C09800D2011A60174B1A68174BD2011A60174B56
:10C0A8001A68D201164B1A6070470E4B0E4A19686F
:10C0B800032391FBF3F111600C4A11680C4A91FBC0
:10C0C800F3F111600B4A11680B4A91FBF3F111600F
:10C0D8000A4A126892FBF3F3094A1360704700BFDB
:10C0E8001C0E00204C26002040260020642C002036
:10C0F80030260020402C0020C42500201C260020CB
:10C108005C2C0020014B1868FDF7ACBA40260020D3
:10C1180008B5FFF79EFFBDE80840F3E770B50021BA
:10C128000A222748274D284E284C0CF063F8002196
:10C138000A22286026480CF05DF800210A223060A7
:10C1480024480CF057F800210A22206022480CF0FD
:10C1580051F8224B326818602B682149D31A06EE31
:10C16800903A2368B8EEE67A06EE903AF8EEE67A68
:10C17800C7EE277AFCEEE77A17EE903A9AB20B8070
:10C18800531C07EE903AB8EEE77ADFED167A67EEC1
:10C19800277A154BFCEEE76A16EE901A8AB206EE7D
:10C1A800902AB8EEE67A198077EEC77AF5EEC07A6B
:10C1B800F1EE10FA01DD01321A80BDE87040A7E700
:10C1C800102600204C260020642C0020402C002043
:10C1D800342600204A2C0020FC250020F8250020C9
:10C1E8002C3A00200000803DC03A00200022F0B523
:10C1F8001346202603254FF02C0C00E02646303E3F
:10C20800F6B217460132092E10F8014B0AD897FBEF
:10C21800F5F605FB16772FB9CE1801F803C0747030
:10C22800023301E0CC540133092AE7D12022CA5451
:10C23800CB1848225A707A229A700022DA70F0BD20
:10C24800F0B51F46144B1E78012E8DB005460C46DE
:10C2580020D0A6F1030CDCF1000646EB0C06CEB9A3
:10C268000E4908A80AF076FE08A86946FFF7BEFF3F
:10C278000B496A4604A80AF06DFEBDF84800F9F7B4
:10C2880067FE3846F9F77AFE2846214604AA33465F
:10C29800F9F798FF0DB0F0BDCD250020C6A505081B
:10C2A8002AAD050810B501210446F9F713F8014B2A
:10C2B8001C8110BDB80D002008B50021C620FBF771
:10C2C800CFFB4FF495700021BDE80840FBF7C8BBD1
:10C2D800014B9F221A817047B80D002000200146AB
:10C2E800C82240F23F13F9F705B807B50DF107006A
:10C2F800FEF741FE9DF807000EBD08B5FFF7F5FFF4
:10C308000028FBD108BD30B5044687B010EE100AEE
:10C318000D4605F08DFF02460B4601A805490AF0B7
:10C3280019FE2046294601AA0023F9F74BFF07B05A
:10C3380030BD00BFF0AF050808B5084803F080FA23
:10C348000648022103F04DFB0028F9D0034803F00A
:10C35800A3FA07EE900AB8EE670A08BD002001406C
:10C3680010B52DED028B9FED098A1924FFF7E4FF24
:10C37800013CE4B238EE008A002CF7D19FED040AA4
:10C3880028EE000ABDEC028B10BD00BF00000000C3
:10C39800ACC868392DE9F04F994B9A4C5D695F68D4
:10C3A8002DED068B93ED00AAC7B006461AEE100ACB
:10C3B80093ED038AD3ED04AAD3ED028A93ED069A8E
:10C3C80005F036FF41EC100BCDE9040108F0ECF95B
:10C3D80032468D493BA88DED0C0B0AF0BBFDA068D9
:10C3E80005F026FF02460B462BA888490AF0B2FD45
:10C3F800E06805F01DFF02460B462FA884490AF0A5
:10C40800A9FD1AEE900A05F013FFCDE90A01DDE94E
:10C418000A23804933A80AF09DFD284605F008FF45
:10C42800CDE90601DDE906237B4937A80AF092FD2C
:10C4380018EE900A05F0FCFE8046894642464B46B7
:10C44800764913A80AF086FD18EE100A05F0F0FEEA
:10C4580082468B46524672495B4617A80AF07AFD17
:10C46800DDE904236F491BA80AF074FD384605F07E
:10C47800DFFE5BA3D3E90023CDE9080105F02CFF1B
:10C4880002460B461FA868490AF064FD49EC118B67
:10C498004BEC10AB08F000F951A3D3E9002351ECA1
:10C4A800100B05F019FF02460B4627A85F490AF052
:10C4B80051FD19EE100A05F0BBFE0B4602465C4919
:10C4C80023A80AF047FDD4ED047AFDEEE77A59492E
:10C4D80017EE902A0FA80AF03DFD0022564BDDE921
:10C4E8000C0105F0F9FE06F0D9F905F0A1FE0246A7
:10C4F8000B4643A851490AF02DFDB5EEC08AF1EE6E
:10C5080010FADFED4F9A37D5304605F07FFE36A397
:10C51800D3E9002305F0E0FEF1EE487A044617EE71
:10C52800900A0D4605F084FE02460B462046294631
:10C5380005F0D2FE02460B462DA1D1E9000105F017
:10C54800F5FF06F0ABF99FED3F7A07EE900AF4EE9F
:10C55800C77AF1EE10FAC6BFC7EEA97A3A4C3B4C3F
:10C56800F4EEE97AF1EE10FA38DD9FED357A384DC0
:10C57800384CC7EE877A78E01FA3D3E900235046EA
:10C58800594605F0A9FE044630460D4605F03EFE24
:10C5980015A3D3E9002305F09FFE02460B4620466B
:10C5A800294605F0C3FF06F079F907EE900AB7EEC1
:10C5B800007AF4EEC77AF1EE10FA46BF67EEA97A70
:10C5C800254C264CF4EEE97AF1EE10FA4CDD9FED9D
:10C5D8001C7A234D234CC7EE877A46E01C4D44E075
:10C5E8006666666666A64C401F85EB51B81E194004
:10C5F800000000A2941A6D420000000080842E41C1
:10C60800DC390020EC37002012B005081CB0050802
:10C6180027B0050832B005083CB0050846B0050843
:10C6280051B005085CB0050867B0050872B0050888
:10C638007DB0050889B00508000034C096B005082B
:10C6480000007A440024744901B00508FEAF0508CB
:10C65800A2AF05080AB0050807B0050804B0050828
:10C668000DB005080FB005089D4D17EE900A05F0AE
:10C67800DFFD2A46CDE900013FA89A4902940AF055
:10C6880069FC994B1A68994B1B689642CCBF0022EB
:10C6980001229E42964BD8BF0022DA60954B1B7848
:10C6A800082B40F0AE800220F9F754FD4FF6FF70DA
:10C6B800F9F764FC1F20F9F74BFC192100238E4A77
:10C6C8002D20F9F77FFD4FF6FF70F9F757FC002092
:10C6D8000024F9F73DFC0F20B42132464FF6FF73D2
:10C6E8000094FFF7ADFD0F206E2123462BAAF9F722
:10C6F80069FDB0206E2123462FAAF9F763FD0F20AC
:10C70800382123461BAAF9F75DFDB02038212346BE
:10C718001FAAF9F757FD0F205C21234633AAF9F722
:10C7280051FD2346B0205C2137AAF9F74BFD0F20B5
:10C738004A21234613AAF9F745FDB0204A2123468A
:10C7480017AAF9F73FFD0F209B21234623AAF9F7E3
:10C7580039FD0F20842123463FAAF9F733FDB02085
:10C768008421234627AAF9F72DFDB0209B2143AA4F
:10C778002346F9F727FD614B1B68B3F57A7FCCBFD9
:10C788004FF4FC604FF47840F9F7F8FB0023A02041
:10C79800B4210FAAF9F716FD594B1C78012C0CD0BF
:10C7A80002D3022C1DD111E04FF6E070F9F7E6FB39
:10C7B8004FF48C700221534A10E04FF4FC60F9F7F3
:10C7C800DDFB4FF48C7002214F4A07E04FF6E07012
:10C7D800F9F7D4FB4D4A4FF48C7021460023F9F742
:10C7E800F1FC0020F9F7CAFB4FF4FC60F9F7B0FB45
:10C7F800FFF7B6FD0F20DC21FFF785FD1F20F9F7B5
:10C80800BDFB3C4B1B789A1FD2B2012A02D90B2BD5
:10C8180040F053823E4B1B78023B052B00F24D82C1
:10C82800DFE813F006007E00EF004801E60165012D
:10C83800DFED387A2AEE27AA1AEE100A05F0F8FC7E
:10C848009DED080B8046894607F0CAFD404653EC2B
:10C85800102B494605F040FD1DA3D3E9002305F040
:10C8680089FB05F0D3FF9DED080B044607F0B8FEE1
:10C87800404653EC102B494605F02EFD02460B4668
:10C8880015A1D1E9000105F073FB05F0BFFF4FF6D4
:10C89800E0730093054600230520DC213246FFF7AC
:10C8A800CFFC134BDB6853B11B4B18881B4B4FF461
:10C8B800784719880097A2B2ABB2F9F7D5FA164BA8
:10C8C8001C60164B4FF6E0701D60F9F741FBF4E170
:10C8D8000000000000E063400000000000C05D4070
:10C8E8000DB00508A4B00508642C00204C260020D3
:10C8F800B80D0020CD250020B1B00508741A00201D
:10C908001C0E00200CAF050810AF050814AF050871
:10C91800582C00200000C84228380020CC3A0020BB
:10C92800A74B1868A74B32461968FFF733FBA64B8D
:10C938001B784FF4FA7292FBF3F307EE903AB8EED5
:10C94800E79ADFEDA27AF4EE498AF1EE10FAC8BF51
:10C95800F0EE498AF5EE408AF1EE10FA48BFF0EEA3
:10C96800678AF4EEC98AF1EE10FA044620D8F4EE8C
:10C97800E78AF1EE10FA1BDBFDEEC97AFDEEE88AD4
:10C9880017EE901A18EE902A0020FFF723FB904B21
:10C99800DB68054653B18F4B18888F4B4FF6FF77EE
:10C9A80019880097A2B2ABB2F9F75EFA8A4B1D60FC
:10C9B800B4EE498AF1EE10FAC8BFB0EE498AF1EE3A
:10C9C800497AB4EE678AF1EE10FA48BFB0EE678A8A
:10C9D800B4EEC98AF1EE10FA00F26F81B4EEE78A7C
:10C9E800F1EE10FAC0F26981FDEEE77ABDEEC99A60
:10C9F800BDEEC88A17EE900A19EE101A18EE102A22
:10CA0800AEE06F4B18686F4B32461968FFF7C2FAF1
:10CA1800F5EEC0AAF1EE10FA044627DDDDE90A01B9
:10CA280059A3D3E9002305F0C9FEF8B158A3D3E907
:10CA38000023DDE90A0105F04FFC0B460246674971
:10CA4800002005F095FA05F0E1FE614BDB6805462C
:10CA580053B1604B1888604B4FF6FF7719880097E1
:10CA6800A2B2ABB2F9F700FA5B4B1D60DDE9060133
:10CA780049A3D3E9002305F0BFFE002800F01D817B
:10CA8800DDE9060140A3D3E9002305F097FE00285D
:10CA980000F0138142A3D3E90023DDE9060105F084
:10CAA8001BFC02460B4600204D4905F061FA05F0D3
:10CAB800ADFE57E0424B1868424B32461968FFF703
:10CAC80069FA39A3D3E900230446DDE9040105F036
:10CAD80093FE50B19DED040B07F066FE002251EC69
:10CAE800100B404B05F0F8FBD2E0C825D3E030A38B
:10CAF800D3E90023DDE9080105F0EEFB2EA3D3E915
:10CB0800002305F013FD05F0C9FE2D4B08EE100AB1
:10CB180018682C4B32461968FFF73CFADFED327A79
:10CB28004AEE677A2A4BFDEEE77ADB6817EE905AF1
:10CB3800044625EAE57553B1264B1888264B4FF66F
:10CB4800FF7719880097A2B2ABB2F9F78DF9BDEE5D
:10CB5800C88A214B18EE102A1D606FF0B300B4216B
:10CB6800FFF738FA1A4BDB68054653B1194B18889A
:10CB78001E4B4FF4FC6719880097A2B2ABB2F9F7C5
:10CB880073F91A4B96E000BF9A9999999999B93F08
:10CB98000000000000409F409A9999999999B9BF5F
:10CBA8000000000000408F4089B5F81400E3693F99
:10CBB80000000000008076401F85EB51B81E194028
:10CBC8004C260020642C00201C03002000000000DC
:10CBD800B80D002028380020CC3A00200000694019
:10CBE80000005940000054C0000048431836002097
:10CBF8003B4B187805F00AFB02460B4600203949E2
:10CC080005F094FC05F04AFE08EE100A05F010FB4A
:10CC180041EC100B07F0C8FDB4EE489AF1EE10FA9B
:10CC2800C8BFB0EE489AB4EEC89AF1EE10FA5BECC1
:10CC380010AB42D82C4B18682C4B32461968FFF7BA
:10CC4800A9F9044619EE100A05F0F2FA41EC100BA6
:10CC580007F0AAFD5946504659EC108B05F01EFE08
:10CC68009FED237A07EE900AC7EE277A17EE900A0F
:10CC780005F0DEFA42464B4605F02EFB02460B460F
:10CC880000201C4905F074F900221B4B05F072F9CD
:10CC980005F0BCFD0546194BDB6853B1184B1888E5
:10CCA800184B4FF6FF7719880097A2B2ABB2F9F785
:10CCB800DBF8144B1D60124B1C60134B1B78022BC6
:10CCC80009D043B14FF6FF7300930520DC213246AB
:10CCD8000023FFF7B5FA47B0BDEC068BBDE8F08F2F
:10CCE8001C030020000059404C260020642C002022
:10CCF80000004843000069400000E03FB80D0020F4
:10CD080028380020CC3A0020582C002010B54FF4C9
:10CD1800C770FAF7B3FEDB2805D14FF4C870FAF7ED
:10CD2800ADFE84B219E041F2E104214644F201006B
:10CD3800FAF796FE44F20100FAF7A0FEA04214BFEB
:10CD480080244FF4007421B24FF4C870FAF788FEBB
:10CD58004FF4C770DB21FAF783FE204610BD024B63
:10CD680000221A60704700BF3436002070EEA10A16
:10CD780088B030EE010A08B0704770EEE10A88B05A
:10CD880030EE410A08B07047F0EE407A20EEA10A72
:10CD980060EE810A47EEA10A88B017EE810A08B052
:10CDA8007047D0B561EEA17A41EE017A2DED048B82
:10CDB80017EE900A88B0B0EE409AF0EE609AF0EE66
:10CDC800418AB0EE618A05F033FA00220023064654
:10CDD8000F4605F0E9FCE8B969EE887A49EE287A49
:10CDE80029EE088A17EE900A05F022FA32463B46E9
:10CDF80005F09CFB19EEA88A05F050FD044618EED4
:10CE0800100A05F015FA32463B4605F08FFB05F08F
:10CE180045FD01E00448044600EE900A00EE104A81
:10CE280008B0BDEC048BD0BD0050C347F0B58E4BA5
:10CE38002DED068B93ED001AD3ED011A8FB0F0EEAD
:10CE4800408AB0EE608A8DED060ACDED070A30EE15
:10CE5800410A70EEE10A38EE811A78EE211A8DED5A
:10CE68000C1ACDED0D1A8DED0A0ACDED0B0AFFF760
:10CE780098FF8DED040ACDED050A04AA92E8030097
:10CE880008AB83E80300DDED099A9DED08AA69EE79
:10CE9800A97A4AEE0A7A17EE900A05F0C9F941EC28
:10CEA800100B07F007FD51EC100B05F0F7FC09EE2D
:10CEB800100A19EE900A05F0BBF904461AEE100A9A
:10CEC8000D4605F0B5F945EC104B41EC110B07F098
:10CED800E3FB51EC100B05F0E1FC68EE087A48EE34
:10CEE800A87AB1EE48AAC8EEA79A604B604D5A6975
:10CEF8001B8B6860EA612B8404468AEE27AA85EDBD
:10CF0800009A19EE100AC5ED028A85ED038AC5ED6F
:10CF1800049A85ED05AA05F08BF94DA3D3E9002302
:10CF280005F06AFCDFED537A002818BFB0EE679A67
:10CF3800B7EE007A79EE077A37EE497A4E4BC7EEAC
:10CF4800877A1B78033BC5ED067A042B71D8DFE896
:10CF580003F0032738664F0018EE100A05F068F949
:10CF6800044618EE900A0D4605F062F906460F468B
:10CF780047EC116B45EC104B07F08EFB36A3D3E959
:10CF8800002351EC100BCDE9004505F0A5F9324618
:10CF9800CDE902013B463949394809F0DBFF48E051
:10CFA80019EE900A05F044F904461AEE100A0D46E7
:10CFB80005F03EF92246CDE900012B4630483149BB
:10CFC8002AE019EE100A05F033F941EC100B07F0CE
:10CFD800EBFB00222C4B51EC100B05F07DF905F012
:10CFE8005DFC05F025F902460B46254827491EE059
:10CFF80019EE100A05F01CF9064620460F4605F002
:10D0080017F917A3D3E9002305F066F9CDE9000164
:10D018001B481F4932463B4609F09CFF09E017EEC2
:10D02800900A05F005F902460B461548194909F01A
:10D0380091FF134C00230220CA212246F9F7C2F8B7
:10D04800002323700FB0BDEC068BF0BDAFF300805A
:10D05800AE47E17A14AEEF3F6666666666A64C4058
:10D06800F6285C8FC2A54C405C360020EC370020C7
:10D07800DC390020A4707D3F582C0020D0B0050872
:10D08800F8350020EAB00508000034C0FAB00508F9
:10D098000CB1050828B1050800B560EEA07A40EE8D
:10D0A800007A2DED028B17EE900A87B0B0EE408A19
:10D0B800F0EE608A8DED020ACDED030A05F0B8F8AE
:10D0C80041EC100B07F0F6FB51EC100B05F0E6FBFA
:10D0D800DFED117A07EE100A78EEA78A38EE078A94
:10D0E80068EEA87A48EE087AC7EE277A17EE900A13
:10D0F80005F09EF841EC100B07F0DCFB51EC100B2F
:10D1080005F0CCFB00EE900A20EE880A60EEA80A33
:10D1180007B0BDEC028B00BD00000000F0B52DED9E
:10D12800028BDFED3A1A3A4B8DB030EEA17AF0EE71
:10D13800407AB7EE001A8DED020A83ED001A30EE40
:10D14800010AC3ED011A31EE671A71EEE01ACDED4E
:10D15800030AF0EE470A8DED077A8DED081ACDED3A
:10D16800091A8DED060AFFF71CFE8DED000ACDEDBC
:10D17800010A9DE8030004AB83E803009DED058ADE
:10D18800DDED048A68EE087A48EEA87A17EE900A70
:10D1980005F04EF841EC100B07F08CFB18EE100A66
:10D1A80057EC106B05F044F8044618EE900A0D464B
:10D1B80005F03EF845EC104B41EC110B07F06CFA0A
:10D1C8003946304655EC104B05F068FB05F030F851
:10D1D80041EC100B07F062FA002251EC100B0D4BDA
:10D1E80005F07AF805F05AFB29460646204605F070
:10D1F80055FB00EE900AF6EE007A60EEA70A00EE04
:10D20800106A0DB0BDEC028BF0BD00BF000000003D
:10D21800343A00200000E03FF0EE407A86B020EE7D
:10D22800200A67EE810A06B070472DE9F04F2DED10
:10D23800028B85B0FCF78AF810EE105AFCF78CF8D0
:10D24800284610EE104A04F0F3FF8046204689462F
:10D2580004F0EEFF41EC100B41EC180B07F0C0F89E
:10D2680057EC106BB0EE480AF0EE680A07F0B8F910
:10D2780032463B46404649465BEC10AB05F02CF87D
:10D2880005F00CFB9FED138A07EE100ADFED127A0A
:10D2980057EE087A114C5B46C4ED007A5246404678
:10D2A800494605F019F805F0F9FA07EE900A27EE55
:10D2B800888A04AB84ED018A94E8030003E903003B
:10D2C800DDED030A9DED020A05B0BDEC028BBDE859
:10D2D800F08F00BF0000F04200008C42C43A0020EA
:10D2E80030B53F4B2DED088BD3ED008AD3ED019A75
:10D2F8003C4BD3ED00AAD3ED01BA3B4B93ED008A2A
:10D3080093ED019A394B93ED00AA93ED01BA38EEEB
:10D31800EA0A79EEEB0A38EE4A1A79EE4B1A93B01C
:10D328008DED0A0ACDED0B0A8DED0C1ACDED0D1A17
:10D33800FFF72AFD8DED000ACDED010A9DE80300F7
:10D348003AEE6A0A7BEE6B0A04AB38EE681A79EE9D
:10D35800691A83E803008DED081ACDED091A8DEDE1
:10D368000E0ACDED0F0AFFF70FFD8DED000ACDED8A
:10D37800010A9DE8030006AB83E803009DED040A5B
:10D38800DDED050A9DED061ADDED071AFFF709FD2B
:10D398008DED000ACDED010A9DE8030002AD85E898
:10D3A8000300134B9DED021A93ED000AD3ED010A19
:10D3B800DDED031AFFF7E8FC8DED000ACDED010A5B
:10D3C8009DE8030012AB03E903006C46DDED110A8A
:10D3D80085E803009DED100A13B0BDEC088B30BD45
:10D3E800F035002048360020B83A0020483A00209E
:10D3F80010380020F7EE007A77EEC07A20EE022A85
:10D4080020EE210A07EEA00AF0EE420A47EE810A52
:10D4180088B008B070472DE9F0432DED028B924B90
:10D428001B78012B89B08146884646D14FEAC0094E
:10D4380001291FFA89F92BD809F58065A8B2FAF7EE
:10D4480061FB8A4C0435A8B284ED000AFAF75AFB4E
:10D4580009F58645A8B284ED010AFAF753FB844C16
:10D46800043584ED000AA8B2FAF74CFBA9F5FC4094
:10D4780084ED010A80B2FAF745FB7E4CA9F5FA4023
:10D48800FC3884ED000A80B2FAF73CFB84ED010A0F
:10D4980008F1FF385FFA88F8B8F1010F00F2DF8071
:10D4A800A9F57C5080B2FAF72DFB734CA9F57A598F
:10D4B80084ED000AA9F17C09CBE0022B40F0CF8073
:10D4C8006E4B6F4A1B68012992ED007A00F2AC801E
:10D4D80007EE900AF8EE676A07EE903A46EE877A0A
:10D4E800BDEEE77A17EE104AA4B207EE104A04F12F
:10D4F8008005ED00B8EE478AADB2284637EEC88AF7
:10D50800FAF700FB0435A8B204F50665EE008DEDC8
:10D51800020AFAF7F7FAB6B230468DED030AFAF7BF
:10D52800F1FA043604F58257B0B28DED040AFE0014
:10D53800FAF7E8FAB6B230468DED050AFAF7E2FADC
:10D548000436B0B281348DED060AE400FAF7DAFA4F
:10D55800A4B220468DED070AFAF7D4FA434E0434F4
:10D56800A0B286ED000AFAF7CDFA6C1CE400A4B26A
:10D57800204686ED010AFAF7C5FA3D4D0434A0B2FB
:10D5880085ED000AFAF7BEFA7C1CE400A4B2204636
:10D5980085ED010AFAF7B6FA364F0434A0B287EDE2
:10D5A800000AFAF7AFFAD6ED001A96ED012ADDED7A
:10D5B800020AF0EE408A87ED010A9DED031AB0EEEB
:10D5C800480AFFF717FF8DED000ACDED010A9DE827
:10D5D8000300D5ED001A95ED012AB0EE480ADDEDFD
:10D5E800040A86E803009DED051AFFF703FF8DED99
:10D5F800000ACDED010A9DE80300D7ED001A85E881
:10D608000300B0EE480ADDED060A9DED071AB0EEFC
:10D61800682AFFF7EFFE8DED000ACDED010A9DE8BF
:10D62800030087E803006C4608F1FF385FFA88F8C2
:10D63800B8F1010F13D809F5C1594FEAC9091FFA02
:10D6480089F94846FAF75EFA0B4C84ED000A09F1AD
:10D6580004091FFA89F0FAF755FA84ED010A09B0AE
:10D66800BDEC028BBDE8F083C9010020B83A002068
:10D6780048360020483A0020F0350020C825002010
:10D68800082600202DE9F04F6E4B2DED048B1C78F9
:10D69800012CC7B0054605D006D3022C0CBF302498
:10D6A800002402E0002400E010244FF47670FAF71A
:10D6B800E5F907464FF47570FAF7E0F980464FF43C
:10D6C8007470FAF703FA032DC0B21D9040F09480ED
:10D6D8005D4A5E4924A809F03DFCC1B224A8FDF7C3
:10D6E80049FC3B4642465A4924A809F033FCC1B2DA
:10D6F80024A8FDF73FFC574A544924A809F02AFCFE
:10D70800C1B224A8FDF736FC04F1C800FAF7DEF927
:10D71800064604F1CC00FAF7D9F9054604F1D00021
:10D72800FAF7D4F9074604F1D400FAF7CFF9AB1B9E
:10D7380006EE903AB8EEE67A06EE907AF8EEE67AD9
:10D748002B46C7EE277A324601904349009724A812
:10D75800FDEEE77ACDED027A09F0FCFBC1B224A810
:10D76800FDF708FC3D4A394924A809F0F3FBC1B28A
:10D7780024A8FDF7FFFBE820FAF7A8F90546EC20F6
:10D78800FAF7A4F90446F020FAF7A0F90646F420BF
:10D79800FAF79CF9631B07EE903A06EE906AB8EE2A
:10D7A800E77AF8EEE67A2A46C7EE277A01902A4900
:10D7B8000096234624A8FDEEE77ACDED027A09F01B
:10D7C800C9FBC1B224A8FDF7D5FB1D9A022A06D1D0
:10D7D800234924A809F0E6FB24A8142109E01D9B8D
:10D7E800012B40F089821F4924A809F0DBFB24A8FB
:10D7F8001021FDF7BFFB7FE21D9A012A40F00E8140
:10D8080004F1C800FAF762F91B9004F1CC00FAF7AA
:10D818005DF9074604F1D000FAF758F91B9B1C90F4
:10D82800FF1A06EE907AB8EEE67A06EE900AF8EE5F
:10D83800E67A0024C7EE277AFDEEE77ACDED1F7A67
:10D84800E7E000BF1C0E002038B1050833B1050819
:10D8580042B105084FB1050855B105089FB1050843
:10D86800A5B10508BAB105081C9B1B9A20460121E1
:10D8780003FB042AFFF7CFFD914B924A18681768FB
:10D88800D3ED018A92ED019A8F4B904AD3F800901C
:10D89800D3ED019A1368012D209392ED018A7ED170
:10D8A800F5EEC08AF1EE10FA54BF4FF0000C4FF0BD
:10D8B800010CB5EEC09ABCF1000F0CBF4FF02B085D
:10D8C8004FF02D08F1EE10FA54BF4FF0000E4FF054
:10D8D800010EF5EEC09ABEF1000F0CBF2B262D26C7
:10D8E800F1EE10FA54BF00210121B5EEC08A0029DB
:10D8F8000CBF4FF02B0B4FF02D0BF1EE10FA54BF6D
:10D9080000220122002A0CBF2B232D231E93BCF1D9
:10D91800000F01D0F1EE688ABEF1000F01D0B1EE20
:10D92800499A09B1F1EE699A0AB1B1EE488A04F050
:10D938007FFCCDE9000118EE900ACDF8088004F0CC
:10D9480077FCCDE90401384604F072FCCDE9060104
:10D9580019EE100A089604F06BFCCDE90A01484656
:10D9680004F066FCCDE90C0119EE900ACDF838B048
:10D9780004F05EFCCDE91001209804F059FC1E9AD1
:10D98800CDE9120118EE100A149204F051FC524627
:10D99800CDE9160124A84E4909F0DCFA2FE0022D42
:10D9A8002ED1FFF79DFC8DED220ACDED230A22AB87
:10D9B80093E8030046AB03E90300DDED457AF5EE95
:10D9C800C07AF1EE10FA449805D5F1EE677A17EEB1
:10D9D800906A2D2702E017EE906A2B2704F028FCA6
:10D9E80002460B463046CDE90023029704F020FC9E
:10D9F8005246CDE9040124A8364909F0ABFAC6B26B
:10DA080024A83146FDF7B6FA0120FDF7CFFF01340F
:10DA1800A4B21F9BA342BFF627AF6AE11D9A022A50
:10DA280040F06781E820FAF751F81B90EC20FAF7EC
:10DA38004DF80646F020FAF749F81B9B1C9006EEB5
:10DA4800900AF61AB8EEE68A06EE906AF8EEE67ADA
:10DA580004F1C800C7EE887AFDEEE77ACDED1E7AAC
:10DA6800FAF734F8064604F1CC00FAF72FF807461F
:10DA780004F1D000FAF72AF8BF1B07EE100A06EEE9
:10DA8800907AF8EEC77AB8EEE67A1B9A1F9087EE7E
:10DA9800277A931B012D06EE903ABDEEC77A88EEE1
:10DAA800278A0D4B8DED207AB8EEE67A87EE277A35
:10DAB80083ED007A094B83ED008A40F0D0808FE037
:10DAC800B83A002048360020483A0020F0350020B7
:10DAD800CBB1050806B20508C82500200826002095
:10DAE8001F9A002102FB046220462192FFF793FC53
:10DAF80095ED018AD8ED018AB5EEC08AF1EE10FAEB
:10DB080054BF4FF0000C4FF0010CF5EEC08A9AEDAF
:10DB1800019ABCF1000F0CBF2B272D27F1EE10FA4C
:10DB280054BF4FF0000E4FF0010EB5EEC09ABEF193
:10DB3800000F0CBF4FF02B0B4FF02D0BF1EE10FA2E
:10DB480054BF002101212868D8F80090DAF8003085
:10DB580000290CBF2B222D22BCF1000F01D0B1EE01
:10DB6800488ABEF1000F01D0F1EE688A09B1B1EE22
:10DB7800499A19921A9304F05BFBCDE9000118EE5B
:10DB8800100A029704F054FBCDE90401484604F05A
:10DB98004FFBCDE9060118EE900ACDF820B004F04D
:10DBA80047FB1A9BCDE90A01184604F041FB199A74
:10DBB800CDE90C0119EE100A0E9204F039FB219AF6
:10DBC800CDE910014F4924A809F0C4F9C1B224A82D
:10DBD800FDF7D0F901340120FDF7E8FEA4B205E015
:10DBE800494DDFF83481DFF834A10024209BA3429B
:10DBF800BFF676AF0024454D2DE01C9B1B9A2046AE
:10DC0800022103FB0426FFF706FC95ED018AB5EE19
:10DC1800C08AF1EE10FA286803D5B1EE488A2D279C
:10DC280000E02B2704F004FBCDE9000118EE100AF0
:10DC3800029704F0FDFA3246CDE90401344924A8DC
:10DC480009F088F9C1B224A8FDF794F90120FDF77D
:10DC5800ADFE0134A4B21E9BA342CEDA49E0022DE8
:10DC680047D142E01C9B1B9A0121204603FB042557
:10DC7800FFF7D1FBFFF734FB8DED220ACDED230A28
:10DC880022AB93E8030046AB03E90300DDED457AD8
:10DC9800F5EEC07AF1EE10FA449806D5F1EE677AFF
:10DCA80017EE908A4FF02D0903E017EE908A4FF097
:10DCB8002B0904F0BDFA06460F464046CDE9006739
:10DCC800CDF8089004F0B4FA2A46CDE904011049C9
:10DCD80024A809F03FF9C1B224A8FDF74BF9013493
:10DCE8000120FDF763FEA4B200E000241E9BA342BE
:10DCF800B8DA084B1D9A1A7047B0BDEC048BBDE822
:10DD0800F08F00BF1AB20508B83A0020F03500209D
:10DD180048B20508C901002048360020483A0020CA
:10DD2800F0B52DED028B04468DB0002800F0D480AC
:10DD3800714B18890419A4B222B2002A05DB40F2FB
:10DD48003F139A42C8BF1C4600E00024F7F7B0FA18
:10DD5800A0B24EF29C71F7F7BDFA674B1C81674B76
:10DD6800586804F065FA5EA3D3E9002304F0B4FA16
:10DD780004F094FD624B1860624B1B780A2B054631
:10DD880024B23DD107EE104AF8EEC77A17EE900A92
:10DD980004F04EFA5C4B064618680F4604F036FA53
:10DDA80002460B4650A1D1E9000104F0BFFB024630
:10DDB8000B463046394604F08FFA064628460F4689
:10DDC80004F036FA02460B463046394604F084FA27
:10DDD80000224E4B04F0AAFB04F060FD04F028FA80
:10DDE80002460B4604A84A4909F0B4F80020F8F79F
:10DDF800B1F90520D72104AA0023F8F7E3F96BE06D
:10DE0800444B1888604304F001FA39A3D3E900238E
:10DE180004F08CFB04F042FD3F4B08EE100A1B682F
:10DE2800FCEEC87A07EE103A17EE905AF8EEC77A69
:10DE38003A4B68EE277A1B68FDEEE77AADB217EE2B
:10DE4800906A28460121F618FFF7E5FAFFF748FA25
:10DE58008DED020ACDED030A02AC94E8030008AB8D
:10DE680083E80300681C80B20121FFF7D4FAFFF7AA
:10DE780037FA8DED020ACDED030A94E803000CABE6
:10DE880007EE105A03E90300B8EEC70ADDED080AE9
:10DE980038EE400A9DED091ADDED0A1A9DED0B2AB0
:10DEA800FFF7A8FA8DED020ACDED030A94E8030006
:10DEB80006AB83E803004FF6FF73009305200023A9
:10DEC800DC213246FEF7BCF9154B9DED060A1878A1
:10DED800DDED070AFEF7AAFF0DB0BDEC028BF0BD21
:10DEE8007B14AE47E17A843F000000A0D954BD41BD
:10DEF8000000000000F07340B80D00201C03002053
:10DF0800AC3A0020CD250020642C00200000F43F0E
:10DF18005BB205082C3A0020402C00204C2600203B
:10DF2800582C00202DE9F843461F8846B6B2002534
:10DF38000D4F12E008EB040189B23046F7F76CF98F
:10DF480029F814000A200134FAF78CFF062CF1D1C5
:10DF580016350136F22DB6B204D06FF0040407EB83
:10DF68000509E7E7BDE8F883683A00202DE9F04F96
:10DF780085B00B1A0193431E9BB20293431C441FA6
:10DF880000F1060901F1FF3A01F1010B9BB20F46BE
:10DF98001646A4B21FFA89F91FFA8AFA1FFA8BFBF0
:10DFA80003938046204651463246F7F76DF92046DE
:10DFB80039463246F7F768F9204659463246F7F7A8
:10DFC80063F9019B0298E518ADB229463246F7F786
:10DFD8005BF9404629463246F7F756F9013403986B
:10DFE80029463246F7F750F9A4B20A20FAF73AFF61
:10DFF8004C45D7D105B0BDE8F08F2DE9F843461F51
:10E008008846B6B200250E4F12E008EB040139F835
:10E01800142089B23046F7F737F901340A20FAF7A5
:10E0280021FF062CF1D116350136F22DB6B204D0F7
:10E038006FF0040407EB0509E7E7BDE8F88300BFC4
:10E04800683A00202DE9F0432DED068B70EE007A3A
:10E058008DB017EE900AB0EE408A10EE904A20EE8E
:10E06800009A04F0E5F8064620460F4604F0E0F86A
:10E07800F7EE008A41EC100B41EC1A0B06F0B0F9F0
:10E0880079EE287A55EC104B17EE900A04F0D0F888
:10E098002246804689462B463046394604F01CF90C
:10E0A80002460B464046494603F062FF04F0F6FB81
:10E0B800B0EE4A0AF0EE6A0A09EE900A38EEC99AFA
:10E0C800DFED377A89EE299A29EE279A06F088FA41
:10E0D800304653EC102B394604F0FEF8044619EE8E
:10E0E800900A0D4604F0A4F802460B46204629463D
:10E0F80004F01CFA00222B4B04F0EEF804F0CEFBDF
:10E10800B4EE688ADFED287A284BF1EE10FA04465F
:10E1180019EE100A08BFB0EE678A1D6804F088F887
:10E1280002460B4603A8224908F014FF204604F0D3
:10E138007FF802460B4606A81E4908F00BFF78EE4A
:10E14800287A38EEC88A87EE888A18EE100A04F012
:10E158006FF802460B4609A8174908F0FBFE052090
:10E16800014603AA0023F8F72DF80520142106AA72
:10E178000023F8F727F8C820052109AA0023F8F793
:10E1880021F84FF6E07300930520DC212A4600238E
:10E19800FEF756F80DB0BDEC068BBDE8F08300BF66
:10E1A8000000484200004940A4707D3F0838002024
:10E1B80064B205086CB2050874B205082DE9F04F81
:10E1C800494B2DED048B1D78022D85B080467BD1FF
:10E1D800464E348A01212046FFF71DF9FFF780F8E3
:10E1E8008DED000ACDED010A9DE8030004AB03E9BB
:10E1F800030028469DED020ADDED030AFEF716FE30
:10E208003B4B1A683B4B1B6802FB04343A4B1C60BF
:10E218003A4BDFED3B7A93ED008A68EE277A5F6828
:10E2280017EE900A04F004F8824638468B4603F04D
:10E23800FFFF41EC100B41EC190B06F0D1F85046EA
:10E2480053EC102B594604F047F823A3D3E90023D5
:10E2580003F090FE04F002FBB0EE490AF0EE690A02
:10E26800054684B206F0BCF9504653EC102B5946CB
:10E2780004F032F80B46024619A1D1E9000103F077
:10E2880077FE04F0EBFAB37C81461FFA80FA1BB9DB
:10E29800B08AF18AFFF7B1FE002320465146B374D5
:10E2A800FFF740FE204651461F22FFF75FFEB0EE03
:10E2B800480A00EE907AFFF7C5FE338AB582984483
:10E2C800A6F81080A6F8169005B0BDEC048BBDE842
:10E2D800F08F00BFAFF300800000000000E0634053
:10E2E8000000000000C05D40582C0020B80D002040
:10E2F800402C00204C26002008380020DC39002063
:10E308000000C842124B1B78022B10B50CD1114BE0
:10E318001B78022B08D1104C2078C0B140B2FFF70F
:10E328004DFF0023237010BD0C4C237E23B99F2082
:10E33800F6F798FF01232376064B1B78022B06D1AC
:10E34800054C94F90000FFF7EBFC0023237010BD87
:10E35800582C002034380020811A0020B80D0020E5
:10E36800034B00201860034B1870FDF753BC00BF27
:10E378003436002034380020034B00201860034B4B
:10E3880002221A70FDF746BC3436002034380020CB
:10E3980037B500242546A0B228213223024601348D
:10E3A8000095F7F761FDB4F5A07FF4D13EBD2DE9E6
:10E3B800F04F2DED088B022897B080468DED070AA7
:10E3C800B34B05D0032805D0012805D10C2202E063
:10E3D800092200E00B221A701878F2F77DFB04215D
:10E3E80003914FF00009F3EE0EAA9FEDAABADFEDF4
:10E3F800AABA7DE1A94B1A68A94B1B6802FB09332D
:10E4080007EE103A01211FFA89F0B8EEC78AFFF724
:10E4180002F8FEF765FF8DED080ACDED090A08AD93
:10E4280095E803000AAB83E803009E4B1A6802EBE9
:10E43800C9030EAF19689C4B1960039952181268EA
:10E448005A60FEF74DFF8DED080ACDED090A95E8F3
:10E4580003000CAB83E80300DDED0A9A9DED0BAADF
:10E46800DDED0C8A9DED0D9AB0EE690AF0EE4A0AD0
:10E47800B0EE681AF0EE491AFEF786FC8DED080A30
:10E48800CDED090A95E80300B0EE691AF0EE4A1AD4
:10E4980087E80300B0EE680AF0EE490AFEF781FC4F
:10E4A8008DED080ACDED090A95E8030010AB83E865
:10E4B80003009DED0E0ADDED0F0AFEF7EDFD8DED73
:10E4C800080ACDED090A95E8030016AA02E9030037
:10E4D8009DED100ADDED110A149EFEF7DDFD8DEDB0
:10E4E800080ACDED090A95E8030087E80300DDED89
:10E4F8000F0AF5EEC00AF1EE10FA48BFF1EE600A15
:10E508009DED0E0ACDED0F0AFEF708FE8DED080A07
:10E51800CDED090A08AA92E8030012AB83E80300CC
:10E528000798129D03F084FE5D4B139FD3F800B04B
:10E538005E4BBDEEC87AD3F800A0CDE9040117EE12
:10E54800102A58465146FDF725FD07EE10AAF8EEA9
:10E55800C77A07EE10BAB4EEE78AF8EEC77AF1EE9A
:10E5680010FAB4EEE78A8CBF00220122504B0690C5
:10E57800F1EE10FAD4BF002202F00102B8F1020F46
:10E58800DA6012D0B8F1030F3ED0B8F1010F68D1AC
:10E59800304603F04DFE36A3D3E9002303F09CFE7A
:10E5A8000022444B03F0E6FC2AE0284603F040FE34
:10E5B800DDE9042304460D462FA1D1E9000103F04B
:10E5C800B5FF02460B462046294603F085FE2CA3DC
:10E5D800D3E9002303F080FE04F060F907EE900A07
:10E5E800C7EEAA7A17EE900A03F022FE41EC100B50
:10E5F80006F0DAF8002251EC100B2F4B03F06CFEFA
:10E6080004F004F904462CE018EE100A03F010FE9A
:10E61800044638460D4603F00BFE17A3D3E9002342
:10E6280003F05AFEDDE9042303F080FF04F036F915
:10E6380003F0FEFD14A3D3E9002303F04DFE0246C8
:10E648000B462046294603F071FF04F027F907EE30
:10E65800900AB0EE6B7A07EE8B7AFDEEC77A17EE6A
:10E66800904A002C2ADBC72CA8BFC72427E000BF8C
:10E678008716D9CEF753F5BF8FC2F5285CAF434054
:10E68800000000000090704000000080DBC486415C
:10E69800582C00200000C8C30000C843402C0020AC
:10E6A8004C26002020360020F0350020642C002065
:10E6B800B80D002000006940000049C00024114B3B
:10E6C800DB685BB1104B1888104B1988069B4FF616
:10E6D800FF759AB2A3B20095F7F7C6FB0B4B039AE6
:10E6E8001C600699084B0832196009F10109039268
:10E6F800074B1B884B45BFF67DAE17B0BDEC088BAA
:10E70800BDE8F08FB80D002028380020CC3A002052
:10E718002C3A00202DE9F0432E4B85B01878F2F7FB
:10E72800DBF92D4B0B221A702C4B1C78012C05D0D1
:10E7380006D3022C0CBF3024002402E0002400E0A1
:10E748001024274B1B78012B07D104F1C800F9F7D7
:10E75800BDF9064604F1D00004E0E820F9F7B6F95F
:10E768000646F020F9F7B2F900240746DFF8809052
:10E778001C4DDFF8808020E007FB04632046012160
:10E788006B61A8F82040FEF746FEFEF7A9FD8DED67
:10E79800000ACDED010A9DE8030004AB03E903007C
:10E7A8000C4B9DED020A1878DDED030AFEF73EFBDF
:10E7B8006869FDF7EFFD0134A4B2B9F80030A3424F
:10E7C800DADA094B02221A70084B00221A7605B0D1
:10E7D800BDE8F083582C0020CD2500201C0E002019
:10E7E800C9010020EC37002034380020B80D002083
:10E7F8002C3A0020DC3900207FB5FDF709F8274ABC
:10E80800274B1168526819605A60264C264B2268BB
:10E818001B68264DD31A06EE903AB8EEE67AD5ED87
:10E82800006AF8EEE67A0021C7EE277AFCEEE77A6E
:10E8380017EE906AB0B2FEF7EEFDFEF751FD8DEDD2
:10E84800000ACDED010A9DE8030004AB03E90300CB
:10E85800174B9DED020A1878DDED030AFEF7E6FA7C
:10E86800144B1868144B1B6836B200FB0630FDF7D2
:10E8780091FD124B226893F90010286800FB0120D3
:10E888000F4A126890421C4605DCFAF7EBFE0D4B66
:10E898001868FDF78BF8002323707FBDEC37002044
:10E8A800F03500202836002040260020C42500200E
:10E8B800582C0020402C00204C260020F025002059
:10E8C80030260020F825002008B5FFF795FF0C4BEF
:10E8D8001A680C4B1B689A4210DB4FF080400021ED
:10E8E80002F055FD084B1868FAF7BCFE074B0222E8
:10E8F8001A70074A00231370064A137608BD00BF32
:10E9080028360020302600204026002034380020F9
:10E91800F0250020B80D002010B500214FF08040F0
:10E9280002F035FD0A4B00241C700A4B20461C706F
:10E93800F7F73AFB084B1868FAF794FE074B0848B4
:10E9480001221A70074B1C70BDE81040F3F7F9B8A4
:10E95800F02500203836002040260020582C0020C2
:10E96800FC170020CD25002007EE100A034BF8EE17
:10E97800477A0022C3ED007A5A6070475C3600205F
:10E9880007EE100A034BF8EE477A0022C3ED007A2F
:10E998005A607047103800200F4B10491A68104B06
:10E9A8001B68D31A06EE903A0E4B1B68B8EEE67A4F
:10E9B80006EE903AF8EEE67AC7EE277AFCEEE77AAA
:10E9C80017EE903A9AB20B80074B188890422CBFEA
:10E9D80000200120704700BF642C00202C3A002042
:10E9E8004C260020402C00204426002013B502AB02
:10E9F800011D23ED010A054A89B213F8014B14548D
:10EA0800013080B28842F8D11CBD00BF6A370020AF
:10EA18002DE9F8431F4F0740002F04460D4603DA3F
:10EA2800013F67F00F070137BFB2DFF874804FEA84
:10EA3800C7091FFA89F9484698ED000A09F104093F
:10EA4800FFF7D4FF1FFA89F098ED010AFFF7CEFF10
:10EA5800114B10261B8894FBF6F6F6019C42B6B2C1
:10EA68000CD1701980B20D498022FAF79BFA00B1D7
:10EA7800FEE721B24FF47F70F8F7F2FF0F2F07D1AE
:10EA88007519A8B205498022FAF78CFA00B1FEE799
:10EA9800BDE8F8830F0000802C3A00206A37002078
:10EAA800EC3700202DE9F043744B2DED028B1888CC
:10EAB800FF2898BF4FF4807093B0C00007F0D8FECD
:10EAC8006F4B0546186028B90520B4216D4A2B46BE
:10EAD800F7F778FB0024694F6B4E4FF000086AE0A7
:10EAE800FCF796FE20464FF44141FFF791FF674B34
:10EAF8001A685B683260002173602046FEF78BFC61
:10EB0800FEF7EEFB8DED020ACDED030A0DF10809C3
:10EB180099E803000AAB83E803005D4B9DED0A1AF0
:10EB280093ED007AD3ED017ADDED0B1A31EE470A49
:10EB380071EEE70A31EE071A71EEA71A8DED0E0A8B
:10EB4800CDED0F0A8DED101ACDED111AFEF729F94A
:10EB58008DED020ACDED030A99E803000CAB83E8BA
:10EB68000300FF2C4FEAC4032B4404D9C3F80080E8
:10EB7800C3F8048003E00C9A1A600D9A5A603B8827
:10EB880040F23F10604390FBF3F080B24FF4FC6317
:10EB98000246282100933223F7F766F93D4B18689F
:10EBA8003D4B1B68C018FAF75DFD3C4B1868FCF735
:10EBB800FDFE0134A4B23B88A34291DA0122134638
:10EBC8004FF4807105A804F0FDFE354EDFF8F8809B
:10EBD800294605A805F0D8F908233370314B0124DC
:10EBE8001C700020F6F7AEFC2F48F2F7AAFF307829
:10EBF800F1F772FF2D4B9FED2E8ADFED2E8A1C70E8
:10EC08000024D5ED007AB0EE687A07EEC87A20467F
:10EC1800FCEEC77A17EE906A03F0F8FA264B00224A
:10EC280003F05AFB03F01AFEB6B2A3B2C72E28BFF0
:10EC3800C72687B253B1214BB8F8000019884FF6A0
:10EC4800FF7300933A463346F7F70EF91B4BC8F8A3
:10EC5800007001340835B4F5807F1E60D1D1184B9F
:10EC68001868FAF7FFFC114B02221A70154B0022A4
:10EC78001A7613B0BDEC028BBDE8F0832C3A002065
:10EC88002036002035AA0508F0350020EC37002092
:10EC98005C36002028360020C4250020F8250020F6
:10ECA800582C0020790D00205817002034380020F7
:10ECB800000016430000C8420000F43FCC3A002090
:10ECC80040260020B80D002028380020F0B5294B38
:10ECD800294F2A4D2A4E012285B01A7000243AE0A5
:10ECE800284B1A68336802FB04336B61264B1C847B
:10ECF800FCF78EFD20464FF44141FFF789FE234B78
:10ED08002A681A606A6820465A600021FEF783FB69
:10ED1800FEF7E6FA8DED000ACDED010A9DE8030045
:10ED280004AB03E903001A4B9DED020A1878DDEDE8
:10ED3800030AFEF77BF86869FDF72CFB154B18688A
:10ED4800154B1B68C018FAF78DFC144B1868FCF7B4
:10ED58002DFE0134A4B23B88A342C1DA104B1868D7
:10ED6800FAF780FC034B02221A700E4B00221A7627
:10ED780005B0F0BD343800202C3A0020EC370020D4
:10ED88004C260020402C0020DC390020F0350020E3
:10ED9800582C002028360020C4250020F825002003
:10EDA80040260020B80D002038B5FDF7ABF9124B0E
:10EDB800124D9F221A81124B012418782C70F1F7FA
:10EDC8008BFE104B00221A600F4B1B78072B04D0C8
:10EDD8000B2B0DD0062B0ED102E0BDE8384075E7AD
:10EDE8004FF0804021462C70BDE8384002F0CFBA81
:10EDF800BDE838408EE438BDB80D00203438002016
:10EE0800582C002034360020CD2500202DE9F7436A
:10EE1800002581462C46154E154FDFF85C801FE013
:10EE2800FCF7F6FC49462046FFF7F2FDD8F800301B
:10EE38003868C018FAF716FC0E4B1868FCF7B6FDD0
:10EE4800308895FBF0F080B24FF4FC6300932821E2
:10EE580002463223F7F708F805F59E7501340335A5
:10EE68003388A342DCDABDE8FE8300BF2C3A0020D9
:10EE780028360020F8250020C425002010B5104CA5
:10EE88004FF47570B4F90010F8F7EAFD0D4B4FF424
:10EE98007670B3F90010F8F7E3FD40F2D230F8F7D6
:10EEA800EDFDB02804D040F2D230B021F8F7D8FDFB
:10EEB8002088FFF759FD034B1888BDE810405FE52F
:10EEC800C4010020C001002000210A2208B509F071
:10EED80091F9D0F1010038BF002008BD73B5041DB9
:10EEE8000E46A4B20C2200234FF6E07520460136E8
:10EEF8000095F7F75DF800230C22B1B22046009583
:10EF0800F7F756F80D4B1B78012B16D10C4E0D4D0B
:10EF1800308829880024043080B20C2223460094CB
:10EF2800F7F746F83088298800940430013180B218
:10EF380089B20C222346F7F73BF87CBD1436002033
:10EF48005A3600200C38002008B54FF6FF70F6F747
:10EF5800FFFF0020F7F7FEF8E12023212C4A0023C9
:10EF6800F7F730F9E1204621294A0023F7F72AF973
:10EF7800E1206921264A0023F7F724F9E1208C21B2
:10EF8800244A0023F7F71EF92348FFF79DFF20B115
:10EF980021482249012207F0DDFF4B2023211E4A88
:10EFA8000023F7F70FF91E48FFF78EFF20B11C4822
:10EFB8001A49012207F0CEFF4B204621184A0023A8
:10EFC800F7F700F91748FFF77FFF20B115481349F5
:10EFD800012207F0BFFF4B206921124A0023F7F7EF
:10EFE800F1F81148FFF770FF20B10F480B490122D3
:10EFF80007F0B0FF4B208C2100230B4AF7F7E2F80B
:10F008000A4B18880A4B1988BDE8084066E700BF14
:10F0180045A8050880B2050810260020C6A50508E1
:10F02800342600204A2C0020FC250020443A0020E9
:10F038000C3A002070B5044600200D461646F7F736
:10F0480089F80020F6F79AFF4FF4FC60F6F780FF86
:10F058002046294656BB1E4A3346F7F7B3F81D48E3
:10F06800FFF732FF20B11B481B49012207F072FF4E
:10F0780004F17006B6B230462946164A0023F7F75F
:10F08800A1F81648FFF720FF20B1144812490122C1
:10F0980007F060FF3235ADB220462946104A0023FA
:10F0A800F7F790F8304629460C4A07E00D4A002346
:10F0B800F7F788F832350B4AA9B220460023F7F74C
:10F0C80081F8094B1888094B1988BDE8704005E795
:10F0D80085B20508B03A0020E0A90508203A0020CA
:10F0E8008DB2050880AA0508443A00200C3A002091
:10F0F80030B5144D9DF80C402C70134D2880134DDD
:10F1080002FB04002980124D80B22880114D29800D
:10F11800114D2A80114A1380114B1880114B198008
:10F12800114B1249E2B21A7000230B7010490A7091
:10F138009DF810200134013254430E4A14700E4ACF
:10F14800137030BDC83B0020A83A0020EA370020E1
:10F15800443A00200C3A002068370020D43A0020B6
:10F168005A3600200C3800200E3A0020393600208C
:10F17800463A0020153600201436002038B50546DA
:10F1880000200C46F6F7E6FF0020F6F7F7FE4FF4EE
:10F19800FC60F6F7DDFE0B48FFF796FE28B109483C
:10F1A80009490A4B002207F0D5FE284621460023CC
:10F1B800044AF7F707F8064B1888064B1988BDE884
:10F1C80038408BE650360020A3AE05080000F03F1B
:10F1D800443A00200C3A0020114B1B68002B70B5F4
:10F1E80005460C4604DA5B420E480F492D2202E020
:10F1F8000C480D49202207F0ADFE0020F6F7AAFFC3
:10F208000020F6F7BBFE4FF4FC60F6F7A1FE054AB6
:10F21800284621460023BDE87040F6F7D3BF00BF5B
:10F22800403A00201838002095B205080F4B10B559
:10F2380019684FF4E170F8F730FC40F23D114FF4D3
:10F24800E070F8F70DFC0020F6F784FF0020F6F7D1
:10F2580095FE4FF4FC60F6F77BFE054A1920642101
:10F268000023BDE81040F6F7ADBF00BF403A0020CC
:10F278009DB2050808B54FF4E070F8F7FFFB40F2BF
:10F288003D13984205D14FF4E170BDE80840F8F706
:10F298001DBC002008BD38B5054600200C46F6F711
:10F2A80059FF0020F6F76AFE4FF4FC60F6F750FEAF
:10F2B8000B48FFF709FE28B109480A490A4B002202
:10F2C80007F048FE284621460023054AF6F77AFF4C
:10F2D800064B1888064B1988BDE83840FEE500BF84
:10F2E8002C360020A3AE05080000F03F443A002069
:10F2F8000C3A002038B5C501ADB20024601980B2BF
:10F30800F9F7F8FB0134C0B2FBF724FEA4B24FF4BE
:10F318007A70F9F7A7FD802CF0D138BD73B5104D80
:10F3280000240E20FBF716FE002609E00DF1070069
:10F33800FBF721FE20B19DF80730AB550136F6B238
:10F348003306F3D5E00180B205498022F9F72AFE99
:10F3580000B1FEE70134A4B2B4F5007FE1D17CBD71
:10F368006A37002007EE100AF8EE477A7FB517EEE5
:10F37800900A02F05DFF02460B4601A8054907F016
:10F38800E9FD0A20962101AA0023F6F71BFF07B022
:10F3980000BD00BFA4B205080EB403B070470A2828
:10F3A80010B5044602D10D20FFF7F9FF064A13688D
:10F3B8001BB103F8014B136010BD044B1B680BB164
:10F3C8002046984710BD00BFD80D0020CC3B002038
:10F3D80010B5044601E0FFF7E2FF14F8010B00281E
:10F3E800F9D110BD2DE9F04F044685B00D464FF018
:10F3F8000A0A00E035462078002800F0C480252855
:10F4080001D0013467E06078302803D1A078012367
:10F41800033407E02D2802D00234002302E0A0784C
:10F42800022303344FF0000805E00AFB080814F82B
:10F43800010BA8F13008A0F13002D2B2092AF4D9A0
:10F448006C2801D04C2803D114F8010B43F00403B5
:10F45800002800F09880602886BFA0F12002D2B270
:10F4680002464F2A3DD006D8432A2DD0442A09D037
:10F47800422A30D133E0552A04D0582A29D0532AB9
:10F4880029D101E00A272DE02E1D2F68002500E074
:10F4980001357A5D002AFBD104E02020FFF77FFFC9
:10F4A8004D4601E0980704D4454505F10109F4D318
:10F4B8004D463846FFF78CFF03E02020FFF76FFF2B
:10F4C80001354545F9D395E728782E1DFFF767FFE5
:10F4D80090E7102706E0FFF762FF2E468AE702272B
:10F4E80000E008272E1D442A296804D1002902DAE1
:10F4F800494243F00803002200E02A46B1FBF7FE28
:10F5080007FB1E11CDB2092D714607D9782814BF03
:10F518004FF0070C4FF0270C6544EDB230350DF86D
:10F528000250551CBEF1000F02D0102DE5D10F225C
:10F53800190705D504A94D192D2105F8101C951C8E
:10F5480013F0010F0CBF4FF0200B4FF0300B9B074F
:10F558002F4604D508E05846FFF721FF4F46474598
:10F5680007F10109F7D34F46013D1DF80500FFF7E4
:10F5780016FF002DF8D103E02020FFF710FF013718
:10F588004745F9D336E705B0BDE8F08F70B5064DAD
:10F598000C462E68286001E0FFF701FF14F8010B04
:10F5A8000028F9D12E6070BDCC3B00200FB407B500
:10F5B80004A951F8040B0191FFF714FFBDE80E40B0
:10F5C80004B070470EB417B505A9084C51F8043BB0
:10F5D800206018460191FFF705FF22680023137089
:10F5E8002360BDE81E4003B0704700BFD80D00205F
:10F5F8000EB433B505A9074C51F8043B25682060C3
:10F6080018460191FFF7EEFE2560BDE83C4003B0C7
:10F61800704700BFCC3B002070B51E4604461C480E
:10F628001546FFF7C3FF022E1FD0042E25D0012E4A
:10F638002AD105E0A15D1748FFF7B8FF013600E0C1
:10F648000026AE42F6DB2020FFF7A9FE002609E0DF
:10F65800A05DA0F12003DBB25E2B88BF2E20FFF750
:10F668009EFE0136AE42F3DB0EE034F8021B0A4878
:10F67800FFF79CFF013DF8D106E054F8041B07484A
:10F68800FFF794FF013DF8D10A20BDE8704086E6F7
:10F69800ABB20508B2B20508B8B20508BEB2050893
:10F6A80008B501214FF4807001F07CFA4FF48070A6
:10F6B8000021BDE8084001F075BA43680A6823F0E4
:10F6C800407323F4807313430A7943EA02234360A7
:10F6D800CA680B6930B51A4384688D68084B2A4399
:10F6E800234013434A7943EA420383600B7DC26A8D
:10F6F800013B22F47002DBB242EA0353C36230BD1D
:10F70800FDF7FFC000230360037143718360C3608A
:10F718000361012303757047074A084B516810B508
:10F728000B4090E8120021438468C06821430143DC
:10F738000B43536010BD00BF00230140E030FCFFC5
:10F748000023036043608360C3607047836811B11E
:10F7580043F0010301E023F001038360704743682D
:10F7680023F4400323F400730B4343607047416262
:10F7780082627047436823F01F030B43436070475E
:10F78800044B5A6810B142F4000201E022F400026E
:10F798005A60704700230140044B5A6810B142F484
:10F7A800800201E022F480025A6070470023014081
:10F7B800092970B50CB20CD904EB44041E3CC66888
:10F7C8000725A54026EA0505A34045EA0304C460C9
:10F7D8000AE0066904EB44040725A54026EA050566
:10F7E80013FA04F42C430461062A0CD80523013AC1
:10F7F8005A43446B1F23934024EA0303914043EA8E
:10F808000102426370BD0C2A12B20CD802EB8202CC
:10F81800233A046B1F23934024EA0303914043EAED
:10F828000102026370BD02EB8202413AC46A1F23DF
:10F83800934024EA0303914043EA0102C26270BD87
:10F84800836843F08043836070478068C0F38050CA
:10F858007047836811B143F4806301E023F4806347
:10F8680083607047836811B143F0020301E023F01D
:10F878000203836070474368013923F4604343EA15
:10F88800413343607047436811B143F4006301E0BA
:10F8980023F4006343607047C06C80B27047014B2B
:10F8A8001868704708230140836811B143F48073D6
:10F8B80001E023F4807383607047836811B143F4D7
:10F8C800007301E023F4007383607047044B5A68A7
:10F8D80010B142F4005201E022F400525A6070471D
:10F8E80000230140092970B50CB20CD904EB44047B
:10F8F8001E3CC6680725A54026EA0505A34045EA3B
:10F908000304C4600AE0066904EB44040725A54023
:10F9180026EA050513FA04F42C430461836BC3F348
:10F928000154121B0232D2B202EB82021F2494400D
:10F9380023EA040391400B43836370BD836B013951
:10F9480023F4401343EA01538363704782B00023D2
:10F9580001930190019BCB180193019B1A6002B09F
:10F968007047836823F470230B4383607047836870
:10F9780023F440130B4383607047836843F4800388
:10F98800836070478068C0F380507047436811B146
:10F9980043F4806301E023F4806343607047436865
:10F9A80011B143F4805301E023F48053436070475E
:10F9B80082B0002301930190019B28335B180193C7
:10F9C800019B186880B202B070470123C9B213FACC
:10F9D80001F143680AB1194301E023EA01014160DA
:10F9E8007047036819420CBF002001207047C943C3
:10F9F800016070474368006810EA112007D00122AF
:10FA0800C9B212FA01F119420CBF00200120704757
:10FA18006FEA112101607047036823F00103036056
:10FA28000023036043608360C36003612123436153
:10FA38002C4B98421CD02C4B984220D02B4B9842F0
:10FA480025D02B4B98422AD02A4B98422FD02A4BAC
:10FA5800984233D0294B984237D0294B984204D149
:10FA68004FF03D5243F8AC2C7047264B984203D1D7
:10FA78003D2243F8082C7047234B984204D14FF499
:10FA8800746243F8202C7047204B984204D14FF4FD
:10FA9800741243F8382C70471D4B984204D14FF02C
:10FAA800746243F8502C70471A4B984203D11A4A93
:10FAB80043F8642C7047194B984203D1184A43F80D
:10FAC8007C2C7047174B984203D1174A43F8942C63
:10FAD8007047164B984204BF4FF03D5243F8AC2C88
:10FAE800704700BF1060024028600240406002403A
:10FAF800586002407060024088600240A060024086
:10FB0800B860024010640240286402404064024029
:10FB180058640240706402403D000020886402403E
:10FB2800400F0020A064024000003D20B86402405D
:10FB38000268134B10B51340CC680A6822434C691D
:10FB480022438C692243CC6922430C6A22434C6AC3
:10FB580022438C6A22434C6B22438C6B224313430F
:10FB6800036042690C6BCB6A22F0070223431343FC
:10FB780043610B6943604B6883608B68C36010BD49
:10FB88003F801CF00023036043608360C36003610F
:10FB980043618361C361036243628362C362036337
:10FBA800436383637047036811B143F0010301E0C5
:10FBB80023F0010303607047036811B143F4004365
:10FBC80001E023F4004303607047036811B143F078
:10FBD800200301E023F02003036070474160704771
:10FBE800406880B27047036812B143F4002301E013
:10FBF80023F40023036001617047036811B143F4E3
:10FC0800802301E023F48023036070470AB1016177
:10FC18007047C16070470068C0F3C0407047006813
:10FC280000F001007047406900F0380070470A4A48
:10FC38000A4B10B50A4CA04288BF13468A004CBF35
:10FC48005B681B6821F0F02121F0821119420CBF7A
:10FC58000020012010BD00BF006402400060024087
:10FC68000F64024010B5084B084A094CA04288BFEF
:10FC7800134611F0005F21F0F02121F0821114BF2A
:10FC8800D960996010BD00BF006002400064024066
:10FC98000F6402400B0607D5436912B143F0800395
:10FCA80001E023F080034361802909D001F01E019F
:10FCB800036812B119430160704723EA010101602A
:10FCC8007047124B124A10B5124CA0428CBF144612
:10FCD8001C4621F0F02323F0C3132BB1026802F075
:10FCE8001E0202EAD12202E0426902F08002880084
:10FCF8004CBF6368236821F0F02121F0821018407E
:10FD080002D0101C18BF012010BD00BF00600240C7
:10FD1800006402400F64024010B5084B084A094CC1
:10FD2800A04288BF134611F0005F21F0F02121F0B6
:10FD3800821114BFD960996010BD00BF00600240F5
:10FD4800006402400F640240044B00221A605A60AB
:10FD58009A60DA60024A5A61704700BF003C01406D
:10FD6800FFFF7F00837910B5002B29D01A4B01685B
:10FD78001C68CA4314401C605C6822405A600279BF
:10FD880002F1804202F59E32146821431160026834
:10FD98009C68D1430C409C60DC682140D960417963
:10FDA800102906D1996811439960D9680A43DA6025
:10FDB80010BD01F1804303F59E3319680A4308E03A
:10FDC8000379016803F1804303F59E331A6822EA38
:10FDD80001021A6010BD00BF003C014000230C2244
:10FDE80003600371427183717047024B1A690243C1
:10FDF8001A617047003C0140034B5B6918420CBF15
:10FE080000200120704700BF003C0140014B5861B1
:10FE1800704700BF003C0140054B1A685B6903400E
:10FE280004D010420CBF00200120704718467047CC
:10FE3800003C0140014B5861704700BF003C014045
:10FE48004FF0204318B943F2DB021A6003E043F293
:10FE5800D20243F820204FF02042411C6FF070433B
:10FE680042F8213002F5827242F82030704770B5AE
:10FE780084684568C368C16A026825431D430369ED
:10FE88001D4343691D4383691D43C3691D43036AB9
:10FE98001D43436A1D43836A1D43036B0D431D4382
:10FEA8004FF02043082C43F8225005D153F8224044
:10FEB80044F0400443F82240436B9E691D68354373
:10FEC8005E6845EA06159E6845EA0625DE6845EA45
:10FED80006451E695B6945EA0655541C45EA0365F3
:10FEE8004FF02043B1F5804F43F8245010D1836B75
:10FEF800986919680143586841EA0011986841EA0D
:10FF0800002118695B6941EA005141EA036101E097
:10FF18006FF07041014B43F8221070BD040100A03E
:10FF2800022242604FF480524262416B4FF4005209
:10FF380010B5826200230F22FF2403608360C36030
:10FF4800036143618361C3610362C36203630A603F
:10FF58004A608C60CA600A614A618B61816B0A6081
:10FF68004A608C60CA600A614A618B6110BD4FF0BB
:10FF7800204321B153F8202042F0010203E053F856
:10FF88002010024A0A4043F820207047FEFF0F0065
:10FF980010280CBF064B074B4FF040024FF01801DA
:10FFA80019605A604FF0FC329A60DA60704700BFFF
:10FFB800600000A0800000A030B5836844681C433E
:10FFC800C36844F008041C4303691C43436944EABA
:10FFD8004324836944EA4334C36999685A68090425
:10FFE80041EA02211A68DB68114341EA0361036AA6
:08FFF8009A685D68120442EAF8
:020000040801F1
:1000000005221D68DB682A4342EA03620368102B5D
:100010000CBF034B034B1C609960DA6030BD00BF1E
:10002000600000A0800000A010230360C2690023CC
:1000300043608360C360036143618361FC23136099
:1000400053609360D360026A136053609360D3601F
:10005000704741B110280CBF074B084B1A6842F09B
:1000600004021A60704710280CBF034A034A044B6D
:1000700011680B4013607047600000A0800000A072
:10008000FBFF0F0041B110280CBF084B084B1A684A
:1000900042F040021A60704710280CBF034A044A1D
:1000A000044B11680B401360704700BF600000A054
:1000B000800000A0BFFF0F00102802D1024B58693A
:1000C0007047024B58697047600000A0800000A094
:1000D000054B18221A6000225A604FF0FC329A60D9
:1000E000DA601A61704700BFA00000A00268436890
:1000F00042F0100242EA4322836842EA4332144B40
:1001000010B51A60C26891685468090441EA042174
:100110001468D268214341EA02629A6002699168D8
:100120005468090441EA04211468D268214341EA71
:100130000262DA60426991685068090441EA00216C
:100140001068D268014341EA02621A6110BD00BF23
:10015000A00000A0C2680023036043608360FC230A
:10016000136053609360D3600269136053609360BF
:10017000D3604269136053609360D3607047054B4E
:1001800018B11A6842F0040202E01968024A0A40F3
:100190001A607047A00000A0FBFF0F0062B110289A
:1001A00001D10E4B03E0B0F5807F03D10C4B5A68B0
:1001B000114311E00B4BFAE7102804D1074B5A68A2
:1001C00022EA010108E0B0F5807F0CBF044B054B2B
:1001D0005A686FEA0101114059607047600000A041
:1001E000800000A0A00000A0102801D1064B04E070
:1001F000B0F5807F0CBF054B054B5B680B420CBF15
:1002000000200120704700BF600000A0800000A017
:10021000A00000A0102804D1074B5A6822EA01016F
:1002200008E0B0F5807F0CBF044B054B5A686FEABD
:100230000101114059607047600000A0800000A0DB
:10024000A00000A0102801D1084B04E0B0F5807F89
:100250000CBF074B074B5B6813EA010004D013EA9D
:10026000D1010CBF00200120704700BF600000A03A
:10027000800000A0A00000A0102804D1084B5A68FC
:1002800022EAD10109E0B0F5807F0CBF054B064B97
:100290005A684FEAD10122EA01015960704700BF54
:1002A000600000A0800000A0A00000A008B52C4BBA
:1002B000984205D10120014600F048FC012048E0A9
:1002C000284B984205D10220012100F03FFC02207A
:1002D0003FE0254B984205D10420012100F036FC77
:1002E000042036E0214B984205D10820012100F07E
:1002F0002DFC08202DE01E4B984205D11020012135
:1003000000F024FC102024E01A4B984205D1202054
:10031000012100F01BFC20201BE0174B984205D167
:100320004020012100F012FC402012E0134B9842C3
:1003300005D18020012100F009FC802009E0104B4C
:1003400098420BD14FF48070012100F0FFFB4FF475
:1003500080700021BDE8084000F0F8BB08BD00BF78
:10036000000002400004024000080240000C02406D
:10037000001002400014024000180240001C02401D
:10038000002002402DE9F0470023D1F800801A46F2
:100390004FF0010C03270CFA02F404EA0805A54209
:1003A0002ED1066817FA03F4E443264006600E795E
:1003B000D0F8009006FA03FA013E4AEA0909012E34
:1003C000C0F8009014D8866891F8059026408660A1
:1003D000866809FA03F949EA06068660466826EA4D
:1003E000050545608D7946689540ADB23543456059
:1003F000C5682C40C460CC79C5689C402C43C4605F
:1004000001320233102AC6D1BDE8F0874FF6FF73E0
:1004100003600023037143718371C371704782B01D
:100420004FF480330193019B0B430193019BC36104
:10043000C161019BC361C3690193C369019302B0A8
:100440007047036919420CBF002001207047006902
:1004500080B27047436919420CBF002001207047E9
:10046000406980B2704701837047418370470AB189
:1004700001837047418370474161704743694B4036
:100480004361704701F00703C908083130B59B008C
:1004900050F821500F249C4025EA040440F82140E4
:1004A00050F8214012FA03F31C4340F8214030BDBC
:1004B00008B5134B984207D14FF40010012100F00A
:1004C00069FB4FF4001014E00E4B984207D14FF433
:1004D0008000012100F05EFB4FF4800009E00A4B30
:1004E00098420BD14FF40000012100F053FB4FF470
:1004F00000000021BDE8084000F04CBB08BD00BF73
:100500000054004000580040005C00407FB50446A5
:10051000868868460D4600F06DFA02992C482B68D3
:1005200026F03F063604B1FBF0F0360C80B20643ED
:10053000A680228822F001021204120C2280254A91
:1005400093420AD85B00B1FBF3F301309BB280B257
:100550002084032B98BF042321E0EE884BF6FF7222
:10056000964205D103225343B1FBF3F39BB206E05D
:1005700019225343B1FBF3F39BB243F480431A05B2
:100580004FF4967208BF43F0010350434FF47A7260
:1005900090FBF2F0013080B243F400432084A38347
:1005A00023886989AA889BB243F0010323802388AA
:1005B00023F4816323F002031B040A431B0C13433F
:1005C0009BB223802A89AB8913439BB223817FBDD1
:1005D00040420F00A086010041F2883303600023EF
:1005E00083804BF6FF72038143814FF48043C280C6
:1005F00083817047038819B19BB243F0010303E084
:1006000023F001031B041B0C03807047038819B1FE
:100610009BB243F4807303E023F480731B041B0C30
:1006200003807047038819B19BB243F4007303E061
:1006300023F400731B041B0C0380704712B141F0BC
:10064000010101E001F0FE0101827047038819B148
:100650009BB243F4806303E023F480631B041B0C10
:100660000380704783899BB201F0FE0123F0FE03F3
:100670000B4383817047838919B19BB243F0010317
:1006800003E023F001031B041B0C838170470388E4
:1006900019B19BB243F0400303E023F040031B0475
:1006A0001B0C03807047038829B16FEA43436FEA4C
:1006B00053439BB201E05B045B0C038070470388EB
:1006C00019B99BB243F0800303E023F080031B04BD
:1006D0001B0C03807047B1F5804F838B04D023F44B
:1006E00080431B041B0C02E09BB243F480438383D2
:1006F0007047B1F5006F038803D19BB243F40063E8
:1007000003E023F400631B041B0C03807047B1F566
:10071000005F038803D19BB243F4005303E023F44A
:1007200000531B041B0C03807047038819B19BB254
:1007300043F0100303E023F010031B041B0C0380A1
:10074000704701827047008AC0B27047038819B1B0
:100750009BB243F4805303E023F480531B041B0C2F
:1007600003807047B1F5006F038803D19BB243F457
:10077000006303E023F400631B041B0C0380704739
:10078000038819B19BB243F0200303E023F0200358
:100790001B041B0C03807047008BC0F307207047BD
:1007A000838819B19BB243F4006303E023F4006330
:1007B0001B041B0C83807047838819B19BB243F4E0
:1007C000805303E023F480531B041B0C8380704789
:1007D00082B0002301930190019BCB180193019BF0
:1007E000188880B202B0704783889BB20AB119435F
:1007F00001E023EA010181807047838A008B9BB26C
:1008000043EA0040084020F07F40431A584240EB42
:1008100003007047838A008B9BB243EA004020F0BC
:100820007F40704782B00023009301930B0F01902B
:100830000093009B21F07F4113B1019B143302E030
:10084000019B090C18330193019B1B6819420CBFD3
:100850000020012002B07047C94389B281827047ED
:100860008388808A80B208409BB206D001F0E061A4
:1008700013EA11410CBF002001207047C94389B21F
:10088000818270470A4B1A6842F001021A60002206
:100890009A60196821F0847121F48031196005494A
:1008A0005960196821F480211960DA60704700BF2F
:1008B0000038024010300024024B00221A701870D9
:1008C000704700BF02380240034B1A6822F0F8025A
:1008D00042EAC0021A60704700380240014B1860BB
:1008E000704700BF00004742064B002201281A70E3
:1008F0001A7002D0042804D101E018707047052254
:100900001A70704770380240014B1860704700BF82
:10091000800E4742014341EA821200995B08013B85
:1009200042EA016141EA0341014B5960704700BF4F
:1009300000380240014B1860704700BF600047421A
:100940008001034B40EA0171C3F88410704700BF77
:1009500000380240014B1860704700BF68004742F2
:10096000014B1860704700BF4C004742034B9A6828
:1009700022F0EC6202430A439A607047003802405A
:10098000034B9A6822F0784202430A439A60704708
:1009900000380240034B9A6822F0030202439A6037
:1009A000704700BF00380240024B986800F00C000E
:1009B000704700BF00380240034B9A6822F0F002F3
:1009C00002439A60704700BF00380240034B9A68A8
:1009D00022F4E05202439A60704700BF00380240A0
:1009E000034B9A6822F4604242EAC0029A60704760
:1009F000003802401E4B9A6802F00C02042A10B51F
:100A000003D0082A03D01B4B18E01B4B16E0596893
:100A10005A6811F4800F596814BF174B154B02F038
:100A20003F02B3FBF2F3124A5268C2F30142C1F330
:100A3000881101324B435200B3FBF2F30C490360BF
:100A40008B680E4A0468C3F30313D35C34FA03F3D0
:100A500043608C68C4F38224145D33FA04F4846028
:100A60008968C1F34231525CD340C36010BD00BFFE
:100A7000003802400024F40000127A003403002001
:100A800000F44073B3F5407F084B08D1996820F01B
:100A9000704221F4F81122F440720A439A601A6FEE
:100AA000000542EA10501867704700BF0038024046
:100AB000014B1860704700BF3C0E4742014B186065
:100AC000704700BF400E4742014B1860704700BF9F
:100AD0005C014742044B1A6B09B1104301E022EA62
:100AE00000001863704700BF00380240044B5A6B87
:100AF00009B1104301E022EA00005863704700BFCB
:100B000000380240044B9A6B09B1104301E022EA1D
:100B100000009863704700BF00380240044B1A6C15
:100B200009B1104301E022EA00001864704700BFD9
:100B300000380240044B5A6C09B1104301E022EA2C
:100B400000005864704700BF00380240044B1A6927
:100B500009B1104301E022EA00001861704700BFAC
:100B600000380240044B5A6909B1104301E022EAFF
:100B700000005861704700BF00380240044B9A697A
:100B800009B1104301E022EA00009861704700BFFC
:100B900000380240044B1A6A09B1104301E022EA0E
:100BA00000001862704700BF00380240044B5A6AC8
:100BB00009B1104301E022EA00005862704700BF0B
:100BC00000380240044B1A6D09B1104301E022EADB
:100BD00000001865704700BF00380240044B5A6D92
:100BE00009B1104301E022EA00005865704700BFD8
:100BF00000380240044B9A6D09B1104301E022EA2B
:100C000000009865704700BF00380240044B1A6E20
:100C100009B1104301E022EA00001866704700BFE6
:100C200000380240044B5A6E09B1104301E022EA39
:100C300000005866704700BF00380240044B1A7825
:100C400009B1104301E022EA00001870704700BFAC
:100C50000D3802404309012B074A01D1136803E014
:100C6000022B0CBF136F536F00F01F0033FA00F01C
:100C700000F00100704700BF0038024007B50023B4
:100C800001933120FFF7E6FF019B01330193019BA4
:100C9000B3F5A06F01D00028F3D03120FFF7DAFFC1
:100CA000003018BF01200EBD024B5A6F42F0807217
:100CB0005A67704700380240034BDB6818420CBF8C
:100CC00000200120704700BF00380240014B18701F
:100CD000704700BF0E38024008B5154B98420BD143
:100CE00001214FF48050FFF761FF4FF48050002145
:100CF000BDE80840FFF75ABF0E4B984207D14FF4AA
:100D000080400121FFF746FF4FF4804009E00A4B85
:100D100098420BD14FF400400121FFF73BFF4FF405
:100D200000400021BDE80840FFF734BF08BD00BF08
:100D30000030014000380040003C00400B88028831
:100D400010B54C8823438C882343CC8823430C89DB
:100D500023434C8923438C892343CC8902F4415299
:100D6000234313439BB20380838B23F400631B0450
:100D70001B0C83830B8A038210BD838B23F47B635C
:100D800023F00F031B041B0C8383022303848B6853
:100D9000F0B5858B022BADB238D0294A8E88946885
:100DA000002E14BF02260126240203D5946824F4E1
:100DB00000049460D2F88440D2F884705268DFF85E
:100DC00084C002F03F02BCFBF2F2C4F38814544327
:100DD000C7F30272B4FBF2F4CA88B2F5007F4FF099
:100DE0000A0201D1240A02E07601B4FBF6F4624360
:100DF000B2FBF3F305330A229BB2B3FBF2F303F029
:100E000001021202C3F34F0392B200E000229C1EC3
:100E1000A4B2FE2C28BF0022CC8828BF0223134393
:100E200023439BB203840B884A882B4343F400631B
:100E300013438A8813438A8913439BB28383F0BD8B
:100E40000038024000127A00002303804380838030
:100E5000C380038143818381C38107230382704759
:100E600000230222038043808380C38082608381C9
:100E70007047038819B19BB243F0400303E023F0AD
:100E800040031B041B0C03807047838B19B19BB27A
:100E900043F4806303E023F480631B041B0C83830F
:100EA0007047038823F400631B041B0C0380038832
:100EB0009BB20B4303807047B1F5804F038803D189
:100EC0009BB243F4804303E023F480431B041B0CD8
:100ED000038070474FF6FF639942038803D09BB2AB
:100EE00043F4807303E023F480731B041B0C038022
:100EF0007047838819B19BB243F0040303E023F0E9
:100F000004031B041B0C83807047838819B19BB2B8
:100F100043F0100303E023F010031B041B0C838039
:100F20007047838B23F47B6323F00F031B041B0C9C
:100F30008383022303840B88828BB3F5007F10B573
:100F400092B205D0002B0CBF4FF48073002301E058
:100F50004FF480734C8822438C88898942F4006264
:100F600022430A4392B21343838310BD808980B227
:100F7000704781817047038819B19BB243F40053D5
:100F800003E023F400531B041B0C03807047038809
:100F90009BB243F4805303807047012902D0008B39
:100FA00080B27047808A80B27047008A80B27047F2
:100FB00083889BB20AB1194301E023EA01018180D1
:100FC0007047090901238B409BB21AB1828892B203
:100FD000134303E0828892B222EA030383807047BE
:100FE000038919420CBF002001207047C94389B210
:100FF0000181704710B584880089012301F00F0238
:1010000080B213FA02F21040A4B205D009098B4055
:101010001C420CBF0020012010BD01F00F01012374
:101020008B40DB439BB20381704700BF08B50121B1
:101030004FF48040FFF7BAFD4FF480400021BDE837
:101040000840FFF7B3BD014B1860704700380140FE
:1010500001F0030289080A4B023130B5920053F8BF
:1010600021500F24944025EA040443F8214053F80A
:10107000214010FA02F2144343F8214030BD00BF72
:1010800000380140014B1860704700BFDC00274268
:10109000014B1860704700BF00042742024B186ADA
:1010A000C0F30020704700BF0038014030B5048C09
:1010B00024F001042404240C0484058B048CADB2B8
:1010C000A4B225F0F305154324F00A0445EA0315FC
:1010D00044F00104ADB20C430583048430BD30B547
:1010E000048C24F010042404240C0484048B058C48
:1010F00024F44074ADB22405240D25F0A00544EA83
:10110000022445F0100544EA033445EA0115A4B26F
:10111000ADB20483058430BD08B5474B984205D174
:1011200001200146FFF742FD01203DE0B0F1804F74
:1011300005D101200146FFF72DFD012076E03F4B50
:10114000984205D102200121FFF724FD02206DE025
:101150003B4B984205D104200121FFF71BFD0420E1
:1011600064E0384B984205D108200121FFF712FDB9
:1011700008205BE0344B984205D110200121FFF795
:1011800009FD102052E0314B984205D12020012169
:10119000FFF700FD202049E02D4B984209D10220A5
:1011A0000121FFF703FD02200021BDE80840FFF701
:1011B000FDBC284B984207D14FF480300121FFF746
:1011C000F5FC4FF48030EFE7234B984207D14FF402
:1011D00000300121FFF7EAFC4FF40030E4E71F4B39
:1011E000984207D14FF480200121FFF7DFFC4FF434
:1011F0008020D9E71A4B984205D140200121FFF702
:10120000C9FC402012E0174B984205D180200121F3
:10121000FFF7C0FC802009E0134B98420BD14FF43C
:1012200080700121FFF7B6FC4FF480700021BDE80B
:101230000840FFF7AFBC08BD0000014000040040BB
:1012400000080040000C0040001000400014004066
:1012500000040140004001400044014000480140BA
:1012600000180040001C0040002000401C4A038879
:1012700090429BB212D002F5806290420ED0B0F143
:10128000804F0BD0A2F58032904207D002F58062E9
:10129000904203D002F58062904203D14A8823F045
:1012A000700313430F4A904208D002F580629042C7
:1012B00004D023F440730A899BB2134303804B6824
:1012C000C3620B880385064B984203D003F5806305
:1012D000984201D18B7A038601238382704700BF35
:1012E00000000140001000404FF0FF334360002336
:1012F0000380038143808372704701858282704737
:10130000038823F070031B041B0C0B4303807047FE
:1013100041627047C1627047406A7047008D80B279
:101320007047038819B19BB243F0020303E023F036
:1013300002031B041B0C03807047038819B19BB286
:1013400043F0040303E023F004031B041B0C03809D
:101350007047038819B19BB243F0800303E023F088
:1013600080031B041B0C03807047038823F00803D1
:101370001B041B0C038003889BB20B430380704744
:10138000038823F440731B041B0C038003889BB267
:101390000B4303807047038819B19BB243F00103EC
:1013A00003E023F001031B041B0C03807047038C34
:1013B00023F001031B041B0C038470B5038C848889
:1013C000028B0D884E8822F073021204120C2A43FD
:1013D0008D8923F002031B0435431B0CADB22B4354
:1013E0000E4DA842A4B203D005F58065A8420ED1E7
:1013F000CD894E8A23F008032B438D8823F0040304
:101400002B430D8A354324F44074ADB22C438480C1
:1014100002838A684263038470BD00BF00000140FC
:10142000038C23F010031B041B0C0384038C8288A1
:1014300030B5048B0D8824F4E6442404240C23F0F6
:10144000200344EA05241B048D891B0C43EA051381
:101450004D8843EA0513134DA84292B2A4B29BB241
:1014600003D005F58065A84215D1CD8923F080030E
:101470009BB243EA05134FF6BF751D408B8845EAC2
:1014800003130D8A22F4406242EA85024D8A42EA41
:1014900085029BB292B282808A680483826303844D
:1014A00030BD00BF00000140038C23F480731B0497
:1014B0001B0C0384038C828830B5848B0D8824F048
:1014C00073042404240C23F400731B042C438D891F
:1014D0001B0C43EA05234D8843EA0523124DA8421D
:1014E00092B29BB203D005F58065A84215D1CD8993
:1014F00023F400639BB243EA05234FF6FF351D40FA
:101500008B8845EA03230D8A22F4405242EA0512F1
:101510004D8A42EA05129BB292B282808A68848325
:10152000C263038430BD00BF00000140038C23F47C
:1015300080531B041B0C0384038C30B58488828B7E
:101540000D8822F4E6421204120C23F4005342EAFE
:1015500005221B048D891B0C43EA05334D8843EAA1
:1015600005330B4DA842A4B292B29BB203D005F54D
:101570008065A84205D10D8A24F4804444EA85148C
:10158000A4B2848082838A680264038430BD00BF71
:1015900000000140002303804380838083608381B7
:1015A000C38103824382704730B5058C0124ADB2FC
:1015B0008C4025EA040400F11803048409B10829C9
:1015C00007D149084FF68F70CC582040C850C858F2
:1015D0000AE00439C1F34E0148F6FF70CC582040B0
:1015E000C8501202C85892B20243CA5030BD41637B
:1015F000704781637047C163704701647047038B14
:1016000023F070031B041B0C0B4303837047038BF5
:1016100023F4E0431B041B0C43EA01239BB2038326
:101620007047838B23F070031B041B0C0B438383D5
:101630007047838B23F4E0431B041B0C43EA012314
:101640009BB283837047038B23F008031B041B0C9E
:101650000B4303837047038B23F400631B041B0CB1
:1016600043EA01239BB203837047838B23F0080373
:101670001B041B0C0B4383837047838B23F4006391
:101680001B041B0C43EA01239BB283837047038B2B
:1016900023F004031B041B0C0B4303837047038BD1
:1016A00023F480631B041B0C43EA01239BB20383D6
:1016B0007047838B23F004031B041B0C0B438383B1
:1016C0007047838B23F480631B041B0C43EA0123C4
:1016D0009BB283837047038B23F080031B041B0C96
:1016E0000B4303837047038B09025B0441EA5343B6
:1016F0009BB203837047838B23F080031B041B0C76
:101700000B4383837047838B09025B0441EA534395
:101710009BB283837047038C23F002031B041B0CD2
:101720000B4303847047038C23F008031B041B0C3A
:101730000B4303847047038C23F020031B041B0C12
:1017400043EA01139BB203847047038C23F08003A8
:101750001B041B0C43EA01139BB203847047038CE8
:1017600023F400731B041B0C43EA01239BB2038484
:101770007047038C23F400631B041B0C43EA012312
:101780009BB203847047038C23F400531B041B0C8F
:1017900043EA01339BB20384704710B5048C0123E4
:1017A0008B40A4B224EA03030384038C12FA01F1F0
:1017B0000B439BB2038410BD10B5048C04238B40F3
:1017C000A4B224EA03030384038C12FA01F10B434D
:1017D0009BB2038410BD00230122038043808280DA
:1017E000C38003817047406B7047806B7047C06B4C
:1017F0007047006C7047038B23F00C031B041B0C19
:101800000383038B9BB20B4303837047038B23F447
:1018100040631B041B0C0383038B9BB243EA01232D
:101820009BB203837047F8B50C464988A288B4F888
:1018300000E02389054600290CBF02270027012A62
:1018400014BF01260226BEF1000F10D1FFF72EFCB7
:101850002846E188FFF7CFFF2846394632462389DC
:10186000FFF73DFCE1882846BDE8F840CEE7FFF7EA
:1018700036FC2846E188FFF7C9FF2846394632463C
:101880002389FFF713FCE1882846BDE8F840B2E75A
:10189000838B23F00C031B041B0C8383838B9BB271
:1018A0000B4383837047838B23F440631B041B0C1F
:1018B0008383838B9BB243EA01239BB2838370476C
:1018C000F8B50D460B88AA88498804463BB92B8990
:1018D000FFF7ECFBE9882046BDE8F8408BE7042BD6
:1018E00007D12B89FFF7FBFBE9882046BDE8F840CC
:1018F0008CE7082BB5F808C0078C1DD127F480773A
:101900003F043F0C0784868B038CB6B29BB226F053
:10191000F30623F4206346EA0C1C43EA01211FFA74
:101920008CFC89B24CEA020241F48071828301840A
:10193000E988BDE8F840ABE727F480573F043F0C47
:101940000784868B038C26F4407623F400533605F7
:101950005B04360D5B0C46EA022243EA013342EA9D
:101960000C329BB2E98892B243F4805382830384A1
:10197000BDE8F84097E74A880B8813438A881343E9
:10198000CA8813430A8913434A8913438A89134334
:101990009BB2A0F8443070470023038043808380CB
:1019A000C3800381438183817047B0F8443029B1FB
:1019B0006FEA43436FEA53439BB201E05B045B0C65
:1019C000A0F844307047838819B19BB243F00403F8
:1019D00003E023F004031B041B0C838070478388FF
:1019E00019B19BB243F0010303E023F001031B0490
:1019F0001B0C8380704783899BB20AB1194301E0B5
:101A000023EA01018181704781827047038A19426C
:101A10000CBF002001207047C94389B20182704782
:101A2000038A828911EA030092B203D011420CBFEB
:101A3000002001207047C94389B2018270470A43E0
:101A4000A0F84820704783899BB20AB1194301E08E
:101A500023EA010181817047838819B19BB243F069
:101A6000080303E023F008031B041B0C838070476A
:101A7000038923F007031B041B0C038170470389B0
:101A800023F070031B041B0C0B43038103899BB2DF
:101A900043F007030381704738B50D461146012214
:101AA000602D044602D1FFF71AFB01E0FFF7FEFAB2
:101AB000238923F070031B041B0C1D4325812389FC
:101AC0009BB243F00703238138BD038923F07003E1
:101AD0001B041B0C0B4303817047838823F07003A6
:101AE0001B041B0C838083889BB20B43838070474D
:101AF000038923F007031B041B0C038103899BB29A
:101B00000B4303817047038923F080031B041B0CE4
:101B1000038103899BB20B430381704710B504898D
:101B2000E4B20C43144344EA0324A4B2048110BD7C
:101B300010B50446FFF7F2FF23899BB243F48043BC
:101B4000238110BD10B50446FFF7E8FF238923F079
:101B500077031B041B0C43F07703238110BD70B582
:101B60000489068B058C26F44076ADB226F0030678
:101B700024F00704360425F022052404360C15430E
:101B8000240C46F4807645EA0315214346F001060D
:101B9000ADB201810683058470BD838819B19BB203
:101BA00043F0800303E023F080031B041B0C8380BD
:101BB0007047A0F85010704708B5234B984205D1E4
:101BC00010200121FEF7F2FF102037E01F4B984252
:101BD00007D14FF400300121FEF7DCFF4FF4003055
:101BE00009E01B4B98420BD14FF480200121FEF7F6
:101BF000D1FF4FF480200021BDE80840FEF7CABFA6
